:100000000C94380F0C94650F0C94650F0C94650FCD
:100010000C94650F0C94650F0C94650F0C94650F90
:100020000C94650F0C94650F0C94650F0C94650F80
:100030000C94650F0C9490E50C94650F0C94650F6F
:100040000C94650F0C94F4830C94650F0C94650F5D
:100050000C94650F0C94650F0C94B08C0C94DBE140
:100060000C94650F0C94B6270C94650F0C94650FD7
:100070000C94650F0C94650F0C94650F0C94650F30
:100080000C9491820C94650F0C94650F0C94650F81
:100090000C94650F0C94650F0C94650F0C9462DE44
:1000A0000C94650F0C94650F0C9464820C94650F8E
:1000B0000C94650F0C94650F0C94650F0C943782AB
:1000C0000C94650F0C94650F0C94650F0C94650FE0
:1000D0000C94650F0C94650F0C94650F0C94650FD0
:1000E0000C94650F084AD73B3BCE016E84BCBFFD24
:1000F000C12F3D6C74319ABD56833DDA3D00C77FF8
:1001000011BED9E4BB4C3E916BAAAABE0000008090
:100110003F05A84CCDB2D44EB93836A9020C50B91F
:10012000918688083CA6AAAA2ABE000000803F4DFE
:10013000383420582059205A20450043616E6E6F94
:100140007420656E746572207375626469723A20FA
:10015000004D3234004D3233202573006175746FC9
:1001600025692E67006572726F72207772697469F3
:100170006E6720746F2066696C65004E6F74205343
:1001800044207072696E74696E67002F00534420BA
:100190007072696E74696E67206279746520002ED2
:1001A0000044656C6574696F6E206661696C656496
:1001B0002C2046696C653A200046696C65206465B0
:1001C0006C657465643A002E006F70656E20666120
:1001D000696C65642C2046696C653A200057726929
:1001E00074696E6720746F2066696C653A20002E12
:1001F000006F70656E206661696C65642C204669CD
:100200006C653A20002E006F70656E206661696C27
:1002100065642C2046696C653A200046696C65204F
:1002200073656C6563746564002053697A653A2070
:100230000046696C65206F70656E65643A20002E1B
:10024000006F70656E206661696C65642C2046697C
:100250006C653A20004E6F77206672657368206681
:10026000696C653A20004E6F7720646F696E672075
:1002700066696C653A20002220706F73002220703E
:100280006172656E743A2200535542524F5554497B
:100290004E452043414C4C207461726765743A228C
:1002A00000747279696E6720746F2063616C6C20D2
:1002B0007375622D67636F64652066696C65732072
:1002C0007769746820746F6F206D616E79206C653A
:1002D00076656C732E204D4158206C6576656C20D8
:1002E00069733A0053442063617264206F6B006F3E
:1002F00070656E526F6F74206661696C656400761C
:100300006F6C756D652E696E6974206661696C65C8
:100310006400534420696E6974206661696C00480A
:10032000617264636F6465642044656661756C74B2
:100330002053657474696E6773204C6F61646564E3
:10034000002044002049002020204D33303120502F
:10035000005049442073657474696E67733A0020D5
:100360005A0020590020204D323036205800486F66
:100370006D65206F666673657420286D6D293A007F
:10038000204500205A002058002042002054002020
:10039000204D323035205300416476616E636564D0
:1003A000207661726961626C65733A20533D4D69D4
:1003B0006E20666565647261746520286D6D2F73AB
:1003C000292C20543D4D696E2074726176656C2035
:1003D000666565647261746520286D6D2F73292CC4
:1003E00020423D6D696E696D756D207365676D6541
:1003F0006E742074696D6520286D73292C20583D1A
:100400006D6178696D756D205859206A65726B2031
:10041000286D6D2F73292C20205A3D6D6178696DF0
:10042000756D205A206A65726B20286D6D2F7329B7
:100430002C2020453D6D6178696D756D2045206AE1
:1004400065726B20286D6D2F7329002054002020C9
:100450004D323034205300416363656C65726174C2
:10046000696F6E3A20533D616363656C65726174B8
:10047000696F6E2C20543D726574726163742061E3
:100480006363656C65726174696F6E00204500205E
:100490005A0020590020204D3230312058004D6143
:1004A00078696D756D20416363656C65726174690F
:1004B0006F6E20286D6D2F7332293A002045002081
:1004C0005A0020590020204D3230332058004D6111
:1004D00078696D756D2066656564726174657320F9
:1004E000286D6D2F73293A00204500205A002059AD
:1004F0000020204D393220580053746570732070ED
:10050000657220756E69743A004572726F723A00B6
:100510006563686F3A0053544F5050452E00507237
:10052000696E7465722073746F7070656420647591
:100530006520746F206572726F72732E2046697821
:1005400020746865206572726F7220616E64207518
:100550007365204D39393920746F20726573746169
:1005600072742E202854656D7065726174757265A1
:100570002069732072657365742E20536574206939
:100580007420616674657220726573746172746937
:100590006E6729004D69736520C3A0206C276172C6
:1005A0007265742E005072696E7465722068616C99
:1005B0007465642E206B696C6C28292063616C6CF7
:1005C000656421006F6B00526573656E643A2000AC
:1005D0002200556E6B6E6F776E20636F6D6D616E6E
:1005E000643A2022004368616E6765722066696C18
:1005F000616D656E74004F6666736574205A203AAB
:1006000020007A5F6D61783A20007A5F6D696E3AFA
:1006100020004F6666736574205A004F66667365E6
:1006200074205A206F6B00486F74656E64206F668B
:1006300066736574733A007A5F6D696E3A2000796B
:100640005F6D61783A2000785F6D696E3A20002016
:100650005A3A0020593A0020436F756E7420583A78
:10066000200020453A00205A3A0020593A00583AD2
:10067000004649524D574152455F4E414D453A4D16
:1006800061726C696E2056312E302E323B205370D1
:1006900072696E7465722F6772626C206D61736827
:1006A000757020666F722067656E36204649524D20
:1006B000574152455F55524C3A68747470733A2FE3
:1006C0002F6769746875622E636F6D2F4D61726C50
:1006D000696E4669726D776172652F4D61726C69E2
:1006E0006E2050524F544F434F4C5F564552534922
:1006F0004F4E3A312E30204D414348494E455F54CC
:100700005950453A45787033442045585452554421
:1007100045525F434F554E543A3220555549443A5D
:1007200030303030303030302D303030302D3030CF
:1007300030302D303030302D3030303030303030BF
:10074000303030300A004578703344204172726591
:10075000742E0045787033442070726574652E00E5
:1007600054656D70206C6974204F4B2E0020423A06
:100770000020453A00543A004C697420656E2063AD
:100780006861756666650054656D70206275736595
:10079000204F4B0020573A0020453A00543A00427F
:1007A00075736520656E20636861756666650020F7
:1007B00042403A0020403A00202F003A00205400E6
:1007C000202F0020423A00202F006F6B20543A0067
:1007D0002569206D696E2C202569207365630045AD
:1007E0006E642066696C65206C697374004265678D
:1007F000696E2066696C65206C697374004175636D
:10080000756E206D6F7576656D656E742E0045781A
:100810007033442070726574652E00526570726981
:100820002E206465206C27696D70722E00457870EB
:1008300033442070726574652E0052657072692EA3
:10084000206465206C27696D70722E004174746598
:100850006E2E206465206C277574696C2E005265BD
:10086000706F732E2E2E00706F733A2000FF01FF01
:100870000000964300005243000039430000A040AE
:100880000000A040000000400000000000005243B3
:100890000000000000000000000000000000000058
:1008A0000000964300005243000039432569206848
:1008B000202569206D696E00446F6E652070726935
:1008C0006E74696E672066696C650053544F5050B2
:1008D000452E005072696E7465722073746F70706B
:1008E00065642064756520746F206572726F727321
:1008F0002E2046697820746865206572726F7220B8
:10090000616E6420757365204D39393920746F200C
:10091000726573746172742E202854656D706572EF
:1009200061747572652069732072657365742E2019
:1009300053657420697420616674657220726573F2
:1009400074617274696E6729004E6F204C696E6520
:10095000204E756D626572207769746820636865E2
:10096000636B73756D2C204C617374204C696E65DC
:100970003A20004E6F20436865636B73756D207776
:10098000697468206C696E65206E756D6265722C85
:10099000204C617374204C696E653A200063686571
:1009A000636B73756D206D69736D617463682C2062
:1009B0004C617374204C696E653A20004C696E6519
:1009C000204E756D626572206973206E6F74204CC5
:1009D000617374204C696E65204E756D6265722B73
:1009E000312C204C617374204C696E653A20004DA7
:1009F00031313000446F6E6520736176696E672017
:100A000066696C652E006F6B004D323900202050F6
:100A10006C616E6E65724275666665724279746568
:100A2000733A20002046726565204D656D6F7279BE
:100A30003A2000466562203232203230313700439E
:100A40006F6D70696C65643A2000286E6F6E652C5E
:100A50002064656661756C7420636F6E66696729D2
:100A600000207C20417574686F723A2000466562F0
:100A700020323220323031372031383A35393A306D
:100A80003300204C61737420557064617465643A5E
:100A90002000312E302E32004D61726C696E0020C4
:100AA000536F6674776172652052657365740020B8
:100AB0005761746368646F672052657365740020C2
:100AC00042726F776E206F75742052657365740083
:100AD0002045787465726E616C2052657365740090
:100AE000506F7765725570007374617274002200E4
:100AF000656E717565696E672022002200656E71F2
:100B00007565696E672022007C3C3E5E2B3D3F2F61
:100B10005B5D3B2C2A225C0045303A20005A3A208B
:100B200000593A2000583A20004D53312C4D533291
:100B30002050696E730A0024F404D9201BC40C5C95
:100B40000E9804C4095F0265077101F405F900FB02
:100B500004B30048048700C103690058035500032B
:100B6000034500BE023A008402310053022A0029E4
:100B700002250004022000E4011C00C8011900AF96
:100B80000117009801140084011300710110006125
:100B900001100051010E0043010D0036010B002B26
:100BA000010B0020010B00150109000C01090003D5
:100BB000010800FB000800F3000800EB000700E458
:100BC000000600DE000600D8000600D2000600CCB9
:100BD000000500C7000500C2000500BD000400B903
:100BE000000400B5000400B1000400AD000400A939
:100BF000000400A5000300A20003009F0004009B66
:100C00000003009800030095000200930003009089
:100C10000003008D0002008B0003008800020086A4
:100C200000020084000300810002007F0002007DBA
:100C30000002007B000200790002007700010076CC
:100C40000002007400020072000100710002006FD7
:100C50000002006D0001006C0002006A00010069E2
:100C600000020067000100660001006500010064E9
:100C70000002006200010061000100600001005FED
:100C80000002005D0001005C0001005B0001005AF1
:100C900000010059000100580001005700010056F2
:100CA00000010055000100540001005300000053F2
:100CB0000001005200010051000100500001004FEE
:100CC0000001004E0000004E0001004D0001004CEC
:100CD0000001004B0000004B0001004A00010049E8
:100CE00000010048000000480001004700010046E4
:100CF00000000046000100450000004500010044DE
:100D000000010043000000430001004200000042D7
:100D10000001004100000041000100400001003FCF
:100D20000000003F0001003E0000003E0001003DC9
:100D30000000003D0001003C0000003C0000003CC1
:100D40000001003B0000003B0001003A0000003AB7
:100D500000010039000000390001003800000038AF
:100D600000000038000100370000003700010036A5
:100D7000000000360000003600010035000000359C
:100D80000000003500010034000000340000003491
:100D90000001003300000033000000330001003286
:100DA000000000320000003200010031000000317C
:100DB0000000003100010030000000300000003071
:100DC0000001002F0000002F0000002F0000002F66
:100DD0000001002E0000002E0000002E0001002D5A
:100DE0000000002D0000002D0000002D0001002C4F
:100DF0000000002C0000002C0000002C0001002B43
:100E00000000002B0000002B0000002B0001002A36
:100E10000000002A0000002A0000002A000100292A
:100E2000000000290000002900000029000000291E
:100E30000001002800000028000000280000002811
:100E40000000002800010027000000270000002704
:100E500000000027000000270001002600000026F7
:100E600000000026000000260000002600010025EA
:100E700000000025000000250000002500000025DE
:100E800000000025000100240000002400000024D0
:100E900000000024000000240001002300000023C3
:100EA00000000023000000230000002300000023B6
:100EB00000000023000100220000002200000022A8
:100EC000000000220000002200000022000100219A
:100ED000000000210000002100000021000000218E
:100EE000000000210000002100010020000000207F
:100EF0000000002000000020000000200000002072
:100F000000000020000000200001001F0000001F62
:100F10000000001F0000001F0000001F0000001F55
:100F20000000001F0001001E0000001E0000001E47
:100F30000000001E00000024F4D43050C38E20C2F4
:100F4000A24017828B7011127A910D816CD90AA878
:100F500061E108C7586607615143061E4B5D05C134
:100F600045A7041A411104093D9803713931034022
:100F700036DB0265339102D4305402802E1D0263A9
:100F80002CEE01752AC501B028A001102781018F20
:100F90002564012B244B01E0223401AC211F018D7B
:100FA000200D01801FFC00841EED00971DDF00B89E
:100FB0001CD200E61BC600201BBC00641AB200B2A3
:100FC00019A8000A19A0006A189900D117910040C9
:100FD000178B00B516840031167E00B31579003AE0
:100FE000157300C7146F0058146A00EE136600886A
:100FF00013630025135E00C7125B006C12570015C7
:10100000125400C111510070114F0021114B00D634
:101010001049008D1047004610440002104200C0E5
:101020000F4000800F3E00420F3C00060F3B00CBFC
:101030000E3800930E37005C0E3500270E3400F397
:101040000D3200C10D3100900D3000600D2E0032C8
:101050000D2D00050D2C00D90C2B00AE0C290085A0
:101060000C29005C0C2700350C27000E0C2600E82C
:101070000B2400C40B2400A00B23007D0B23005A7B
:101080000B2100390B2100180B2000F80A1F00D992
:101090000A1E00BB0A1E009D0A1D00800A1D006377
:1010A0000A1C00470A1B002C0A1B00110A1A00F731
:1010B000091A00DD091900C4091900AB09190092C9
:1010C0000917007B091800630917004C0916003640
:1010D000091600200916000A091500F5081500E098
:1010E000081400CC081400B8081400A408140090D8
:1010F0000813007D0812006B081300580812004600
:101100000812003408110023081100120811000110
:10111000081100F0071000E0071000D0071000C011
:10112000071000B0070F00A107100091070E008301
:10113000070F0074070F0065070E0057070E0049E0
:10114000070E003B070D002E070E0020070D0013B1
:10115000070D0006070D00F9060C00ED060D00E076
:10116000060C00D4060C00C8060C00BC060C00B02F
:10117000060C00A4060B0099060C008D060B0082DD
:10118000060B0077060B006C060B0061060A005781
:10119000060B004C060A0042060A0038060A002E1A
:1011A000060A0024060A001A060A001006090007AB
:1011B000060A00FD050900F4050900EB050900E237
:1011C000050900D9050900D0050900C7050900BEB9
:1011D000050900B5050800AD050800A50509009C36
:1011E000050800940508008C050800840508007CAB
:1011F000050800740508006C050700650508005D1A
:10120000050700560508004E050700470507004082
:1012100005080038050700310507002A05070023E7
:101220000507001C050600160507000F0507000846
:1012300005060002050700FB040600F5040700EEA2
:10124000040600E8040600E2040700DB040600D5FB
:10125000040600CF040600C9040600C3040600BD4E
:10126000040600B7040600B1040500AC040600A69D
:10127000040600A00405009B0406009504050090E8
:101280000406008A04050085040500800406007A2F
:1012900004050075040500700405006B0405006674
:1012A000040500610405005C0405005704050052B4
:1012B0000405004D04050048040500430405003EF4
:1012C0000404003A04050035040500300404002C31
:1012D00004050027040400230405001E0404001A6A
:1012E00004040016040500110404000D04040009A0
:1012F0000405000404040000040400FC030400F8D6
:10130000030400F4030400F0030400EC030400E809
:10131000030400E4030400E0030400DC030400D839
:10132000030400D4030400D0030400CC030400C869
:10133000030300C5030300656E6473746F7073204C
:101340006869743A205A00205A3A00656E647374D2
:101350006F7073206869743A20590020593A00650B
:101360006E6473746F7073206869743A205800203B
:10137000583A00656E6473746F7073206869743ACC
:1013800020004572723A204D415854454D5020423C
:1013900045440054656D70657261747572652068AE
:1013A000656174656420626564207377697463683D
:1013B0006564206F66662E204D415854454D50207F
:1013C00074726967676572656420212100457272D5
:1013D0003A204D494E54454D50003A20457874729C
:1013E00075646572207377697463686564206F66DD
:1013F000662E204D494E54454D50207472696767E2
:10140000657265642021004572723A204D4158543E
:10141000454D50003A2045787472756465722073AA
:1014200077697463686564206F66662E204D415845
:1014300054454D5020747269676765726564202158
:1014400000202D20496E76616C6964206578747285
:1014500075646572206E756D626572202100700181
:101460002C0190012701B0012201C0011D01F001F2
:1014700018011002130130020E01600209019002EE
:101480000401C002FF000003FA004003F5008003DE
:10149000F000D003EB002004E6007004E100E0045B
:1014A000DC004005D700C005D2004006CD00D006C4
:1014B000C8008007C3003008BE00F008B900C009AA
:1014C000B400B00AAF00B00BAA00D00CA500000E0B
:1014D000A000500F9B00C010960050129100001405
:1014E0008C00C0158700B0178200B0197D00D01B9A
:1014F0007800001E730040206E0090226900F024E6
:10150000640040275F0090295A00E02B5500102E00
:10151000500020304B0010324600E033410090353F
:101520003C001037370070383200A0392D00B03A37
:101530002800A03B2300603C1E00103D1900903D98
:101540001400103E0F00703E0A00C03E0500003F30
:101550000000504944204175746F74756E652066B3
:10156000696E6973686564212050757420746865BC
:10157000206C617374204B702C204B6920616E6469
:10158000204B6420636F6E7374616E747320667297
:101590006F6D2061626F766520696E746F20436F96
:1015A0006E66696775726174696F6E2E6800504966
:1015B00044204175746F74756E65206661696C6551
:1015C00064212074696D656F75740020403A006F66
:1015D0006B20543A006F6B20423A0050494420413E
:1015E00075746F74756E65206661696C6564212021
:1015F00054656D706572617475726520746F6F20CB
:101600006869676800204B643A2000204B693A20E3
:1016100000204B703A200020436C61737369632093
:1016200050494420002054753A2000204B753A2040
:1016300000206D61783A2000206D696E3A2000200C
:10164000643A200020626961733A20002D2D3A2D02
:101650002D002D2D2D0053440001200001200005F8
:101660002E2E004D656E75207072696E6369706113
:101670006C004D3234004D323320257300506173BD
:1016800020646520636172746500496D70722E205C
:1016900064657075697320534400417272657465A6
:1016A0007220696D70722E0052657072656E647280
:1016B0006520696D70722E00496E746572726F6D6F
:1016C00070726520696D70722E00436F6E74726F58
:1016D0006C6572005072657061726572005072655F
:1016E00063686175666661676520504C41005265AC
:1016F000676C6572005375727665696C6C65720013
:101700004D383420582059205A20450052657374B2
:1017100061757265722064656661757473004669EF
:101720006C616D656E74004D6F7576656D656E7478
:101730000054656D7065726174757265004D656EFB
:1017400075207072696E636970616C0046696C2EF9
:10175000204469612E20320046696C2E2044696164
:101760002E20320046696C2E204469612E20310003
:1017700046696C2E204469612E20310041727265E9
:1017800074004D6172636865200041727265740077
:101790004D617263686520004520696E206D6D3370
:1017A00000436F6E74726F6C657200457061732FC9
:1017B0006D6D00457061732F6D6D005A7061732FF0
:1017C0006D6D005A7061732F6D6D00597061732FCC
:1017D0006D6D00597061732F6D6D00587061732FBE
:1017E0006D6D00587061732F6D6D00412D726574C1
:1017F0007261637400412D7265747261637400419B
:101800006D6178206500416D6178206500416D61F2
:1018100078207A00416D6178207A00416D617820EE
:101820007900416D6178207900416D617820780000
:10183000416D6178207800566465706C206D696E2A
:1018400000566465706C206D696E00566D696E009F
:10185000566D696E00566D61786500566D617865EC
:1018600000566D61787A00566D61787A00566D6128
:10187000787900566D61787900566D6178780056F8
:101880006D6178780056652D6A65726B0056652D1E
:101890006A65726B00567A2D6A65726B00567A2DF6
:1018A0006A65726B005678792D6A65726B0056789E
:1018B000792D6A65726B00416363656C00416363F7
:1018C000656C00436F6E74726F6C65720052656771
:1018D0006C2E2070726563682E2041425300526561
:1018E000676C2E2070726563682E20504C4100504A
:1018F00049442D43005049442D43005049442D4450
:10190000005049442D44005049442D490050494459
:101910002D49005049442D50005049442D5000207D
:10192000022046616374657572002002204661637F
:1019300074657572002002204D6178002002204DF0
:101940006178002002204D696E002002204D696EF2
:10195000004172726574004D6172636865200041D8
:1019600072726574004D6172636865200054656D24
:10197000702E204175746F2E00566974652E207686
:10198000656E74696C617465757200566974652E54
:101990002076656E74696C617465757200506C6157
:1019A0007465617500506C61746561750042757392
:1019B0006532004275736532004275736500427589
:1019C000736500436F6E74726F6C657200506C616A
:1019D0007465617500506C61746561750042757362
:1019E00065004275736500566974652E2076656ED4
:1019F00074696C617465757200566974652E207621
:101A0000656E74696C61746575720054656D70659E
:101A100072617475726500506C6174656175005017
:101A20006C6174656175004275736500427573651C
:101A300000566974652E2076656E74696C617465F4
:101A4000757200566974652E2076656E74696C61D6
:101A5000746575720054656D706572617475726538
:101A6000004D36303200426F62696E65203120636E
:101A7000686172676565004465706C6163657220BA
:101A8000756E206178650047323700436861722EB9
:101A9000204F7269672E0047323600536175762EEB
:101AA000204F7269672E0047393220583020593054
:101AB000205A30004F726967696E6520696369005A
:101AC0004D38340041727265746572206D6F7465B3
:101AD0007572730047323800504F4D206175746F36
:101AE00000526566726F696469720050726563685E
:101AF0006175666661676520414253005072656397
:101B0000686175666661676520504C41004D656E81
:101B100075207072696E636970616C004176616EE8
:101B2000636520302E316D6D004176616E636520F6
:101B3000316D6D004176616E63652031306D6D00F1
:101B40005072657061726572004578747275646573
:101B500072004176616E6365205A004176616E6362
:101B6000652059004176616E6365205800446570B8
:101B70006C6163657220756E2061786500457874CC
:101B80007275646572005A0059005800507265639E
:101B9000682E2041425320506C617465617500507D
:101BA000726563682E2041425320546F7574005053
:101BB00072656368617566662E204142532032006B
:101BC0005072656368617566662E2041425320310C
:101BD0000050726570617265720050726563682EA4
:101BE00020504C4120506C617465617500507265E5
:101BF00063682E20504C4120546F757400507265FC
:101C00006368617566662E20504C41203200507228
:101C1000656368617566662E20504C412031005026
:101C200072657061726572004D36303000436861D4
:101C30006E6765722066696C616D656E7400466CD6
:101C40007578203100466C7578203100466C7578C7
:101C5000203000466C7578203000466C7578004660
:101C60006C757800566974652E2076656E74696CA3
:101C7000617465757200566974652E2076656E74A0
:101C8000696C617465757200506C61746561750092
:101C9000506C617465617500427573653200427500
:101CA0007365320042757365004275736500205696
:101CB0006974657373650020566974657373650094
:101CC0004D656E75207072696E636970616C00435A
:101CD0006172746520726574697265650043617232
:101CE000746520696E7365726565004D3330302010
:101CF000533639382050323030004D333030205395
:101D000036353920503230300000002100240027C1
:101D1000002A002D003000330001010000040107FB
:101D2000010A0100002200250028002B002E0031AE
:101D300000340002010000050108010B0100002031
:101D4000002300260029002C002F00320000010093
:101D50000003010601090105050505070508080836
:101D600008020202020A0A0808040404040101012C
:101D70000101010101030303030303030304070734
:101D8000070C0C0C0C0C0C0C0C02020202060606D2
:101D900006060606060B0B0B0B0B0B0B0B010210BA
:101DA0002020080810204010204080020102010875
:101DB0000402010102040810204080804020100825
:101DC000040201800402018040201008040201087E
:101DD00004020101020408102040800102040810DE
:101DE0002040800000090A02080B0C0D07060304BE
:101DF00001000000000000000000000000000000E2
:101E000000000000000000000000000000000011C1
:101E1000100F0000000000000000000000000000A3
:101E200000000000000000000002494E46494E49F3
:101E300054594E414ECDCCCC3D0AD7233C17B7D197
:101E40003877CC2B329595E6241FB14F0A0000203D
:101E5000410000C84200401C4620BCBE4CCA1B0EBC
:101E60005AAEC59D74004A28C12AF6D3D1DDBC2ADA
:101E700011241FBECFEFD1E2DEBFCDBF00E00CBF0B
:101E800015E0A0E0B2E0E6E3FDED01E00BBF02C02B
:101E900007900D92A838B107D9F71BBE12E1A8E848
:101EA000B5E001C01D92AE36B107E1F71EE1CEE606
:101EB000DEE104C02297FE010E9441EEC636D10742
:101EC000C9F70E94E9E40C948FEE0C940000A0E0A6
:101ED000B0E0EDE6FFE00C945EEEEC015B01611515
:101EE000710519F0FB0191838083F9908F2D90E0AB
:101EF0000E9445EE892BC9F7FDE2FF1621F4F99007
:101F0000EE24E39405C02BE2F21609F4F990EE24D6
:101F10008E0101501040C8016AE27EE143E050E0CA
:101F200072D2892BF9F48E010E5F1F4FC8016DE24A
:101F30007EE145E050E067D2892B19F48E01095FFC
:101F40001F4FA114B10419F0F50111830083E0FCC7
:101F500004C070E090E080E813C070E090E080E89A
:101F60006FEF07C1C80162E37EE143E050E04BD26E
:101F7000892B69F4A114B10429F470E090E080EC9D
:101F80006FE7F7C02296F501D183C083F6CF88248E
:101F9000992440E050E060E070E0EF2DE053EA303B
:101FA000A0F5F2E0EF2A8E2D90E09C0128703070B1
:101FB000E2FE06C0232B79F50894811C911C2BC0EE
:101FC000232B19F0089481089108DB01CA0112E063
:101FD000880F991FAA1FBB1F1A95D1F7480F591FC9
:101FE0006A1F7B1F440F551F661F771F4E0F511D21
:101FF000611D711D483929E9520729E9620729E164
:10200000720748F084E0E82A06C0EE3F31F4E3FCB2
:1020100039C098E0E92AF990C0CFE53311F0E531F5
:1020200089F529912D3219F4E0E1EE2A05C02B3211
:1020300019F081E090E003C0299182E090E0E22F66
:10204000E053EA3018F0C81BD90B1CC020E030E088
:10205000FCE020383F075CF4C901880F991F880F06
:10206000991F280F391F220F331F2E0F311DE991A1
:10207000E053EA3068F3E4FE03C0309521953F4F0A
:10208000820E931ECE2CDD24E1FE07C0A114B10404
:1020900021F02197F501D183C083CB01BA010E94C1
:1020A0009EEA7B018C01F3E0CF22DD2423E0C216FF
:1020B000D10421F417FB109517F910955701680109
:1020C000C801B70120E030E040E050E00E94FEE9A6
:1020D000882309F44AC097FE0DC029E4E22E2EE1C0
:1020E000F22E9094819491089394C0E2D0E000E0A5
:1020F00010E012C091E6E92E9EE1F92EF6CFF7012D
:102100002591359145915491C601B5010E94DEECAF
:102110005B016C018C1A9D0A8C169D0684F7D5957F
:10212000C7950F5F1F4F0630110529F08CEF9FEF09
:10213000E80EF91EF1CFC501D6017C018D018C2D71
:10214000880F8D2D881F8F3F51F0C601B50120E00B
:1021500030E040E050E00E94FEE9882331F482E262
:1021600090E090936D1280936C127E2D9F2D802FA6
:10217000612F272F392F482F562FB901CA01CDB70C
:10218000DEB7ECE00C947AEE2F923F925F926F9262
:102190007F928F929F92AF92BF92CF92DF92EF92F7
:1021A000FF920F931F93CF93DF938C011B01EA01E2
:1021B0006115710519F0FB0191838083209749F027
:1021C000CE010297839728F020E030E040E050E015
:1021D000F6C0F801A1908F018A2D90E00E9445EE93
:1021E000892BB9F7FDE2AF1631F4F801A1908F0108
:1021F0005524539407C0FBE2AF1619F4F801A190DF
:102200008F015524209719F0C031D105C1F4F0E3B6
:10221000AF1679F4F8018081883711F0883549F4D8
:10222000F801A1800E5F1F4FF2E05F2AC0E1D0E00D
:1022300006C0209721F480E3A816E9F427C0C8302F
:10224000D10531F1C930D10524F4C230D10531F5C1
:102250000CC0CA30D10589F0C031D105F9F4C12CC8
:10226000D12CE12CB8E0FB2E28C0C12CD12CE12CC4
:10227000A0E4FA2E22C0CAE0D0E0FCECCF2EFCECA9
:10228000DF2EFCECEF2EFCE0FF2E17C0C8E0D0E004
:10229000C12CD12CE12CE0E1FE2E0FC09E01442781
:1022A00037FD4095542F60E070E080E090E80E9498
:1022B00002EEC901DA016C017D0120E030E040E06E
:1022C00050E060E03E01882477FC8094982C70ED0B
:1022D000B72EBA0CE9E0EB1570F48A2D81548A31DF
:1022E00018F499ECB92E06C08A2D81568A3150F522
:1022F00089EAB82EBA0C8B2D90E08C179D0714F547
:102300006F3FE1F0C216D306E406F506B0F0CA014D
:10231000B901A40193010E94B0ED9B01AC012B0D0A
:10232000311D411D511D2130F0E03F07F0E04F0706
:10233000F0E85F0710F461E001C06FEFF801A190D1
:102340008F01C5CF2114310481F0662331F0015093
:102350001040F1011183008308C051FE1AC00250E1
:102360001040F1011183008314C067FF12C050FCBC
:1023700005C02FEF3FEF4FEF5FE704C020E030E0F4
:1023800040E050E882E290E090936D1280936C12EE
:1023900016C050FE08C050954095309521953F4F8E
:1023A0004F4F5F4F0CC057FF0AC082E290E09093FE
:1023B0006D1280936C122FEF3FEF4FEF5FE7B90183
:1023C000CA01DF91CF911F910F91FF90EF90DF90A5
:1023D000CF90BF90AF909F908F907F906F905F90C5
:1023E0003F902F900895FB01DC0105900D92002095
:1023F000E1F70895FC0105900020E9F7809590959C
:102400008E0F9F1F0895FB01DC014150504088F062
:102410008D9181341CF08B350CF4805E65916134B4
:102420001CF06B350CF4605E861B611171F3990B27
:102430000895881BFCCFFB01DC014150504048F05F
:1024400005900D920020C9F701C01D9241505040E7
:10245000E0F70895FB0155915523A9F0BF01DC0178
:102460004D9145174111E1F759F4CD010590002038
:1024700049F04D9140154111C9F3FB014111EFCFD6
:1024800081E090E001970895FB01DC0104C08D918B
:102490000190801921F441505040C8F7881B990BD6
:1024A0000895FB01DC0102C001900D9241505040A3
:1024B000D8F70895FB01DC018D9181341CF08B3538
:1024C0000CF4805E619161341CF06B350CF4605E3D
:1024D000861B611189F3990B0895FB01DC010D90B6
:1024E0000020E9F7119701900D920020E1F708957F
:1024F000FC018191861721F08823D9F79927089547
:102500003197CF010895FB01DC018D910190801975
:102510000110D9F3990B0895FB01DC0101900D9294
:102520000020E1F70895FB01DC014150504030F0FC
:102530008D910190801919F40020B9F7881B990B2F
:102540000895FB01DC014150504048F001900D928C
:102550000020C9F701C01D9241505040E0F7089596
:10256000AEE0B0E0E6EBF2E10C9466EE0E891F8976
:102570008EE08C831A8309838FEF9FE79E838D8380
:102580009E01265E3F4FCE010196688D798DA9018F
:102590000AD02F813885020F131FF80110822E9662
:1025A000E4E00C9482EEABE0B0E0E9EDF2E10C94F3
:1025B00058EE3C012B015A01FC01178216828381DF
:1025C00081FD03C06FEF7FEFB9C19AE0892E1E0134
:1025D0000894211C311CF3012381F20123FD859114
:1025E00023FF81912F01882309F4A5C1853239F495
:1025F00023FD859123FF81912F01853221F490E005
:10260000B301B7D1E8CF982FFF24EE249924FFE13E
:10261000FF15D0F09B3269F09C3228F4903259F0CB
:10262000933291F40EC09D3249F0903369F441E049
:1026300024C052E0F52A84E0F82A28C098E0F92A5C
:1026400025C0E0E1FE2A22C0F7FC29C0892F805373
:102650008A3070F4F6FE05C0989C902C1124980ED8
:1026600015C0E89CE02C1124E80EF0E2FF2A0EC011
:102670009E3229F4F6FC5FC140E4F42A07C09C3680
:1026800019F450E8F52A02C0983649F4F20123FD06
:10269000959123FF91912F01992309F0B8CF892FAC
:1026A0008554833018F08052833038F444E050E091
:1026B000A40EB51E5FE359830FC0933631F09337F4
:1026C00079F0933509F052C01FC0F50180818983EC
:1026D00042E050E0A40EB51E610101E010E011C01F
:1026E000F501C080D180F6FC03C06FEF7FEF02C020
:1026F000692D70E042E050E0A40EB51EC6012ED157
:102700008C015FE7F52213C0F501C080D180F6FC93
:1027100003C06FEF7FEF02C0692D70E042E050E030
:10272000A40EB51EC6010FD18C0150E8F52AF3FEA8
:1027300006C018C080E290E0B3011BD1EA948E2D50
:1027400090E008171907B0F30DC0F601F7FC85916A
:10275000F7FE81916F0190E0B3010BD1E110EA9493
:10276000015010400115110581F7E2C0943611F0B7
:10277000993661F5F7FE08C0F5012081318142816B
:10278000538184E090E00AC0F501808191819C0131
:10279000442737FD4095542F82E090E0A80EB91EE3
:1027A0009FE6F92257FF09C0509540953095219535
:1027B0003F4F4F4F5F4FE0E8FE2ACA01B901A10128
:1027C0002AE030E002D1D82ED2183FC0953729F444
:1027D0001F2D1F7E2AE030E01DC01F2D197F9F3660
:1027E00061F0903720F4983509F0A5C00FC09037FC
:1027F00039F0983709F09FC004C028E030E00AC0E3
:10280000106114FD146020E130E004C014FD166076
:1028100020E132E017FF08C0F501608171818281FB
:10282000938144E050E008C0F50180819181BC01B2
:1028300080E090E042E050E0A40EB51EA101C5D0BA
:10284000D82ED2188FE7F82EF122F6FE0BC05EEFDD
:10285000F522D91438F4F4FE07C0F2FC05C08FEE5F
:10286000F82202C01D2D01C0192DF4FE0DC0FE017D
:10287000ED0DF11D8081803319F499EEF92208C025
:102880001F5FF2FE05C003C08F2D867809F01F5F21
:102890000F2DF3FC13C0F0FE0EC01E1510F09D2C82
:1028A0000AC09D2C9E0C911A1E2D05C080E290E05E
:1028B000B3015FD01F5F1E15C8F304C01E1510F4CE
:1028C000E11A01C0EE2404FF0EC080E390E0B301E2
:1028D00050D002FF1BC001FD03C088E790E00EC08E
:1028E00088E590E00BC0802F867881F001FF02C060
:1028F0008BE201C080E2F7FC8DE290E0B30139D0B9
:1029000005C080E390E0B30134D09A94D914C8F3A1
:10291000DA94F101ED0DF11D808190E0B30129D031
:10292000DD20B1F705C080E290E0B30122D0EA9447
:10293000EE20C9F750CEF30166817781CB012B964B
:10294000E2E10C9474EEFC010590615070400110BE
:10295000D8F7809590958E0F9F1F0895FC016150C8
:10296000704001900110D8F7809590958E0F9F1FB1
:1029700008950F931F93CF93DF938C01EB018B810D
:1029800081FF1BC082FF0DC02E813F818C819D8104
:102990002817390764F4E881F9810193F983E88302
:1029A00006C0E885F985802F1995892B31F48E8131
:1029B0009F8101969F838E8302C00FEF1FEFC80196
:1029C000DF91CF911F910F910895FA01AA27283026
:1029D00051F1203181F1E8946F936E7F6E5F7F4FEC
:1029E0008F4F9F4FAF4FB1E03ED0B4E03CD0670F68
:1029F000781F891F9A1FA11D680F791F8A1F911DBB
:102A0000A11D6A0F711D811D911DA11D20D009F40A
:102A100068943F912AE0269F11243019305D31934C
:102A2000DEF6CF010895462F4770405D4193B3E035
:102A30000FD0C9F7F6CF462F4F70405D4A3318F0DC
:102A4000495D31FD4052419302D0A9F7EACFB4E08D
:102A5000A6959795879577956795BA95C9F7009745
:102A60006105710508959B01AC010A2E06945795E6
:102A7000479537952795BA95C9F7620F731F841F3D
:102A8000951FA01D0895FC01128213820895FC0178
:102A90008381882311F081E082830895FC01828183
:102AA000811112820895CF93DF93DC01FC01EB5575
:102AB000FE4F808191810097C9F1019791838083B6
:102AC000ED01CC5ADF4FFD01ED58FF4F8BE1019036
:102AD00009928150E1F7FD01EE5AFF4FAF58BF4F09
:102AE0008D919C911197A157B04091838083FD01F6
:102AF000ED58FF4F20E030E0AD014B555E4F10C068
:102B00002F5F3F4FEF01DF015F968BE10D90099240
:102B10008150E1F7858D968D329791838083B196B0
:102B2000DA018D919C912817390750F3DF91CF91ED
:102B30000895FC018DE095E091838083878188234F
:102B400021F0CF0104960C94E4720895CF92DF92A5
:102B5000EF92FF920F931F93DF93CF93CDB7DEB722
:102B60006F970FB6F894DEBF0FBECDBF8C016B011F
:102B7000095A1F4FD8018C9107551040882321F422
:102B80002FE2E22EF12C03C090E5E92EF12CE00EAD
:102B9000F11E8DE095E09A8389831C821B82188642
:102BA0001D82B7016C5F7F4FCE010596A60121E023
:102BB0000E94D079882391F5E0E1F5E0949108C076
:102BC0008091C00085FFFCCF9093C6003196949110
:102BD0009923B1F7EBE3F1E0949108C08091C00034
:102BE00085FFFCCF9093C600319694919923B1F75D
:102BF00009C08091C00085FFFCCF0894C11CD11C86
:102C00009093C600F6019081992399F78091C000B6
:102C100085FFFCCF8AE08093C6005AC0F801EB55CF
:102C2000FE4F208131812A30310508F040C02F5FEE
:102C30003F4F3183208321503040F90185E0EE0F72
:102C4000FF1F8A95E1F7E21BF30BED58FF4FE00FF2
:102C5000F11F13C0AF01415E5F4FBF018BE1DB018C
:102C60000D90BD01DA010D92AD018150C1F7929135
:102C700082913296968F858F7F9721503040BFEF9B
:102C80002E3F3B0739F7D801AD58BF4FF7013496B7
:102C90008BE101900D928150E1F70F581F4FF70122
:102CA00082819381D8018D939C9301571040D80164
:102CB000AC5ABF4FFE0135968BE101900D928150C9
:102CC000E1F70E5A1F4F8B819C81F801918380831D
:102CD000CE0101962EDF6F960FB6F894DEBF0FBEC1
:102CE000CDBFCF91DF911F910F91FF90EF90DF90BB
:102CF000CF900895EF92FF920F931F938C013EECBB
:102D0000E32E31E0F32EE80EF91EC7010E94977200
:102D1000C7010E94E472F801108211821F910F9185
:102D2000FF90EF900895CF92DF92EF92FF920F9372
:102D30001F93CF93DF937C016B01DB010D9000208B
:102D4000E9F78D0101501040061B170BEEECF1E086
:102D5000EE0EFF1ED7011C92E2E3FEEFEE0EFF1E09
:102D6000CB016EE470E0C4DBEC01009731F4F801B4
:102D70003197EC0DFD1D86010CC060E270E0B8DB00
:102D80008C010F5F1F4FCE016AE270E0B1DBFC01E6
:102D900031978DE081838AE082831382C701865355
:102DA0009E4FB8010E94E17A8EEC91E0E80EF91E88
:102DB000D7018C91882319F1E9E0F5E0949108C0DE
:102DC0008091C00085FFFCCF9093C600319694910E
:102DD0009923B1F7E5E6F1E0949108C08091C00035
:102DE00085FFFCCF9093C600319694919923B1F75B
:102DF0008091C00085FFFCCF8AE08093C600DF9100
:102E0000CF911F910F91FF90EF90DF90CF90089599
:102E1000CF93DF93EC018B81882309F43BC0EDE86D
:102E2000F1E0949108C08091C00085FFFCCF9093A1
:102E3000C600319694919923B1F7CD57DD4F488163
:102E400059816A817B81C358D2408CE096E02AE0A8
:102E500030E00E94E328EBE8F1E0949108C0809113
:102E6000C00085FFFCCF9093C600319694919923C2
:102E7000B1F7C558DD4F488159816A817B818CE06B
:102E800096E02AE030E00E94E3288091C00085FFB0
:102E9000FCCF12C0EBE7F1E0949108C08091C00034
:102EA00085FFFCCF9093C600319694919923B1F79A
:102EB0008091C00085FFFCCF8AE08093C600DF913F
:102EC000CF9108952F923F924F925F926F927F928F
:102ED0008F929F92AF92BF92CF92DF92EF92FF922A
:102EE0000F931F93DF93CF93CDB7DEB7AC970FB699
:102EF000F894DEBF0FBECDBF5C014B01FC018381A6
:102F0000882309F43BC1C50182539E4F0E94E4729D
:102F1000F50112821A8A1D8A198A188A8DE095E0B5
:102F20009F878E875EE4C52ED12CCA0CDB1C2FE256
:102F300030E0A20EB31EF601B182A08221ED3FEF78
:102F4000A20EB31EF40180818F3209F08DC0C4013E
:102F50006FE270E0CDDA7C010894E11CF11C3E01C7
:102F60000894611C711C260142E1242E312C2C0E88
:102F70003D1E75C0C7016FE270E0BADA6C010097C0
:102F800009F480C0E816F90608F07CC08C010E191F
:102F90001F09C301B701A801D4DA060D171DF801F6
:102FA0001082F30107C08091C00085FFFCCF3196ED
:102FB0009093C60090819923B1F78091C00085FF5E
:102FC000FCCFFAE0F093C600F201608171816115D7
:102FD000710519F460E070E002C06C5F7F4FC101C1
:102FE000A30121E00E94D079882371F5E9ECF1E09A
:102FF000949108C08091C00085FFFCCF9093C600DB
:10300000319694919923B1F7FE01319607C08091D2
:10301000C00085FFFCCF31969093C6009081992324
:10302000B1F7E7ECF1E0949108C08091C00085FF12
:10303000FCCF9093C600319694919923B1F780917B
:10304000C00085FFFCCF94C02EE030E02C0F3D1F68
:10305000F2013183208376010894E11CF11CE11414
:10306000F10409F087CF0BC080E590E0A80EB91EEF
:10307000F601B182A08220EB3FEFA20EB31ED82C46
:10308000092D02C0DE2C0F2D8EE490E0A80EB91E93
:10309000F5018081918122EB3FEFA20EB31E0097D4
:1030A00019F480E090E001C004966D2D702F0E940D
:1030B0009C7A882371F1E9EBF1E0949108C080914A
:1030C000C00085FFFCCF9093C60031969491992360
:1030D000B1F78D2D902F9C01F90107C08091C000A0
:1030E00085FFFCCF31969093C60090819923B1F76C
:1030F0008091C00085FFFCCF8AE08093C60083E802
:1031000092E0A80EB91EF50110821182128213827C
:1031100032C0E1EAF1E0949108C08091C00085FFDF
:10312000FCCF9093C600319694919923B1F78D2DE1
:10313000902F9C01F90107C08091C00085FFFCCF52
:1031400031969093C60090819923B1F7EFE9F1E0B1
:10315000949108C08091C00085FFFCCF9093C60079
:10316000319694919923B1F78091C00085FFFCCFEF
:103170008AE08093C600CE010E96DBDCAC960FB6DB
:10318000F894DEBF0FBECDBFCF91DF911F910F919D
:10319000FF90EF90DF90CF90BF90AF909F908F9077
:1031A0007F906F905F904F903F902F900895BF92C7
:1031B000CF92DF92EF92FF920F931F93CF93DF9303
:1031C0008C01EB018FE28993EE24E394FF2475EAEE
:1031D000C72E71E0D72EC00ED11E6FE1B62E14C0DF
:1031E000FB9CC00111248D589F4F800F911FBE0181
:1031F0000E94F47202C02196E3948881882319F01A
:103200008CE88E15C0F7F3942F2D30E0F601808105
:1032100091812817390720F3E7FC07C0C8018253C2
:103220009E4FBE010E94F47201C01882DF91CF91BF
:103230001F910F91FF90EF90DF90CF90BF90089576
:10324000EF92FF920F931F93CF93DF938C01FC01BA
:10325000138286A9882321F0C801C3960E94E472D4
:10326000E7EAEE2EE1E0FE2EE00EF11EC70160E07F
:1032700045E30E949370882309F5E0E1F5E094911D
:1032800008C08091C00085FFFCCF9093C6003196A6
:1032900094919923B1F7E2E1F3E0949108C0809111
:1032A000C00085FFFCCF9093C6003196949199237E
:1032B000B1F78091C00085FFFCCF7DC0E801C45507
:1032C000DE4FCE01B70141E00E94727B882341F5B9
:1032D000CE01B70140E00E94727B882309F5E9E046
:1032E000F5E0949108C08091C00085FFFCCF9093D9
:1032F000C600319694919923B1F7EFEFF2E09491E3
:1033000008C08091C00085FFFCCF9093C600319625
:1033100094919923B1F78091C00085FFFCCF4BC0F9
:10332000C801C396BE010E94D675882309F5E9E05D
:10333000F5E0949108C08091C00085FFFCCF909388
:10334000C600319694919923B1F7EFEEF2E0949193
:1033500008C08091C00085FFFCCF9093C6003196D5
:1033600094919923B1F78091C00085FFFCCF23C0D1
:1033700081E0F8018383E0E1F5E0949108C0809159
:10338000C00085FFFCCF9093C6003196949199239D
:10339000B1F7E4EEF2E0949108C08091C00085FF9F
:1033A000FCCF9093C600319694919923B1F7809108
:1033B000C00085FFFCCF8AE08093C600D801AC5ADC
:1033C000BF4FF801F3968BE101900D928150E1F728
:1033D000F80181A992A90E5A1F4FF80191838083A9
:1033E00002551040C8018F96025B1F4FF801918370
:1033F0008083DF91CF911F910F91FF90EF900895FF
:103400002F923F924F925F926F927F929F92AF92D4
:10341000BF92CF92DF92EF92FF920F931F93DF93B1
:10342000CF93CDB7DEB7CC55D0400FB6F894DEBF02
:103430000FBECDBF6C01662311F527E832E0C20E46
:10344000D31ED6018C91E9E7FDEFCE0EDF1E882357
:1034500009F4E2C02FE732E0C20ED31ED601ED9090
:10346000FD900D911C91E1E8FDEFCE0EDF1E0E9454
:1034700023E2E616F7060807190708F4CDC027E887
:1034800032E0C20ED31ED6011C92E9E7FDEFCE0E4C
:10349000DF1ED60113968C91882339F4C601D0DE45
:1034A000F6018381882309F4B7C000D000D0EDB7BE
:1034B000FEB731967E010894E11CF11CADB7BEB792
:1034C0001296FC92EE9211978CE591E093838283A1
:1034D000D6019D968D919C919E979583848340D82B
:1034E0008701EDB7FEB736960FB6F894FEBF0FBE54
:1034F000EDBF57010AC0D8018C91992787FD90959F
:103500000E944DEEF80181938F01F501019000209A
:10351000E9F73197EA19FB09802F8E198E175CF3B2
:1035200013E3A12EB12CAC0CBD1CC50140E050E052
:1035300060E070E00E94CD719924BDE3EB2EF12C88
:10354000EC0EFD1E2E010894411C511CAFE16A2EA9
:10355000712C6C0E7D1EF5E52F2EF1E03F2E42C042
:10356000D8018C9190E00E944DEEF80181938F017B
:10357000D7010D900020E9F71197AE19BF09802FF0
:103580008E198A176CF327968FAD27978E3751F1D6
:10359000C701B20145E050E00E949312009711F577
:1035A00000D000D0EDB7FEB73196ADB7BEB71296DA
:1035B0007C926E92119733822282558244820E94BD
:1035C000B012EDB7FEB736960FB6F894FEBF0FBE39
:1035D000EDBFC3010E94643681E591E00E94EB35A6
:1035E00099249394C501B70140E050E00E94F5741E
:1035F000181614F48701BCCF992041F48FEF9FEF88
:10360000D6019E969C938E939D9706C0F60185A544
:1036100096A5019696A785A7C45ADF4F0FB6F894D2
:10362000DEBF0FBECDBFCF91DF911F910F91FF90F5
:10363000EF90DF90CF90BF90AF909F907F906F9072
:103640005F904F903F902F9008952F923F924F920E
:103650005F926F927F928F929F92AF92BF92CF9222
:10366000DF92EF92FF920F931F93DF93CF93CDB72B
:10367000DEB7CF58D0400FB6F894DEBF0FBECDBF37
:103680008C012B016A01C757DF4F39832883C95842
:10369000D04084E090E0C80ED91EF8017196C95759
:1036A000DF4FF983E883C758D04044E0642E712C83
:1036B000600E711ECA57DF4F1882C658D04036E6DA
:1036C000E32EF12CEC0EFD1EC7010B96C557DF4F04
:1036D00099838883CB58D04028E8822E22E0922E0E
:1036E000800E911E9AE8A92E92E0B92EA00EB11E6E
:1036F00087E4282E312C2C0E3D1EF1013496C35741
:10370000DF4FF983E883CD58D040E0E1F5E08491C4
:10371000C157DF4F8883CF58D04053C1F70183850D
:10372000482F50E0BA01687170706031710509F07E
:1037300056C1F401208131812130310509F44FC196
:103740002230310509F44BC1F701DE011196908159
:10375000903239F08E2F8E19883011F48EE28D93CD
:103760009D933196C557DF4F88819981CB58D040C2
:10377000E817F90761F71C921E86F2018081882301
:1037800031F4CE010E9660E072E00E946D12CE011F
:103790000E96B2010E946D12CE010E96BE016F5FB1
:1037A0007F4F0E946D12CE010E9660E072E00E9483
:1037B0006D121CA61FA61BA61AA68DE095E099A760
:1037C00088A7CE018C96B601AE014F5F5F4F21E016
:1037D0000E94D079882309F03FC0F4018081918153
:1037E000892BD1F5C157DF4F9881CF58D040E0E108
:1037F000F5E008C08091C00085FFFCCF9093C60023
:10380000319694919923B1F7E2E0F2E007C08091FC
:10381000C00085FFFCCF31969093C600908199231C
:10382000B1F78091C00085FFFCCFFAE0F093C600AD
:10383000FE01319607C08091C00085FFFCCF319614
:103840009093C60090819923B1F78091C00085FFC5
:10385000FCCF8AE08093C600C357DF4FA881B981AF
:10386000CD58D040FE01BC968BE101900D92815065
:10387000E1F78AA59BA5F101938382838DE095E012
:1038800091838083C801BE01625F7F4FA10120E068
:1038900030E0DBDEC1014DD9CE0188964AD991C016
:1038A0009E3209F48EC09F3509F48BC0F8019189CE
:1038B0009E3209F486C09F3509F483C043FD81C060
:1038C00080E06031710509F481E0F80184A7882364
:1038D00049F4F7018085873409F073C081858E37FC
:1038E00009F46FC0D301F7018081803241F08E2F3F
:1038F0008E19883011F48EE28D9380818D933196EC
:10390000C557DF4F88819981CB58D040E817F90718
:1039100059F71C92F40180819181009701F5F20121
:1039200007C08091C00085FFFCCF31969093C60000
:1039300090819923B1F7F30107C08091C00085FF02
:10394000FCCF31969093C60090819923B1F7809176
:10395000C00085FFFCCFFAE0F093C60032C0813092
:10396000910539F4F50180819181019691838083DD
:1039700028C0029731F5C757DF4F88819981C95810
:10398000D040009731F0B3010E945A12892B71F494
:103990002BC0CA57DF4F9881C658D040292F30E03E
:1039A000F5018081918128173907F1F0CA57DF4F5F
:1039B000F881C658D040FF5FCA57DF4FF883C6581A
:1039C000D040C601B701C957DF4F48815981C75858
:1039D000D0400E94F57418160CF4A0CE05C0F70173
:1039E0009081992309F05CCFC157DF4F0FB6F8944F
:1039F000DEBF0FBECDBFCF91DF911F910F91FF9022
:103A0000EF90DF90CF90BF90AF909F908F907F907E
:103A10006F905F904F903F902F900895EF92FF929C
:103A20000F931F93DF93CF93CDB7DEB76F970FB68A
:103A3000F894DEBF0FBECDBF7C018C01025B1F4F2F
:103A4000805B9F4FF8019183808328E832E0E20E8B
:103A5000F31E21E030E0F701219331937F011182C1
:103A6000108226E73DEFE20EF31E049640E050E0A0
:103A700060E070E00E94CD71F80120813181DE01AB
:103A80001596F90134968BE101900D928150E1F782
:103A9000F901828193819C838B838DE095E09A83E9
:103AA0008983C70165E172E08E010F5F1F4FA80196
:103AB00020E030E0CADDC8013CD8F701E657FD4FF1
:103AC000808191816F960FB6F894DEBF0FBECDBF97
:103AD000CF91DF911F910F91FF90EF900895CF92BA
:103AE000DF92EF92FF920F931F93DF93CF93CDB7A7
:103AF000DEB76F970FB6F894DEBF0FBECDBF7C0167
:103B00006A018C01025B1F4F805B9F4FF80191831C
:103B1000808328E832E0E20EF31E22E030E0F70175
:103B2000219331937F017183608326E73DEFE20E9D
:103B3000F31E049640E050E060E070E00E94CD711A
:103B4000F80120813181DE011596F90134968BE16F
:103B500001900D928150E1F7F901828193819C835C
:103B60008B838DE095E09A838983C70165E172E0DC
:103B70008E010F5F1F4FA801960167DDC8010E94EB
:103B800099156F960FB6F894DEBF0FBECDBFCF91DB
:103B9000DF911F910F91FF90EF90DF90CF900895EC
:103BA0002F923F924F925F926F927F928F929F924D
:103BB000AF92BF92CF92DF92EF92FF920F931F933B
:103BC000DF93CF93CDB7DEB7AD970FB6F894DEBFD6
:103BD0000FBECDBF7C013B014DA7DC0113968C913C
:103BE000882309F450C3E1EDF1E0EE0EFF1ED7018A
:103BF0008C91EFE2FEEFEE0EFF1E882309F418C150
:103C0000222309F0E0C029EE31E0E20EF31ED701D5
:103C10008C91E7E1FEEFEE0EFF1E882371F1E9E0E3
:103C2000F5E0949108C08091C00085FFFCCF90938F
:103C3000C600319694919923B1F7E1EAF2E09491AC
:103C400008C08091C00085FFFCCF9093C6003196DC
:103C500094919923B1F78CE096E061E070E04AE03E
:103C600050E00E9432298091C00085FFFCCF8AE09D
:103C70008093C6000E94682B06C3E0E1F5E09491B2
:103C800008C08091C00085FFFCCF9093C60031969C
:103C900094919923B1F7E8E8F2E0949108C08091FB
:103CA000C00085FFFCCF9093C60031969491992374
:103CB000B1F7F30107C08091C00085FFFCCF3196BA
:103CC0009093C60090819923B1F7EDE7F2E09491CB
:103CD00008C08091C00085FFFCCF9093C60031964C
:103CE00094919923B1F7C7012EEE31E0E20EF31E55
:103CF000B7015DDA4BEF5FEFE40EF51ED7019C9143
:103D0000E7E1FEEFEE0EFF1E8DE8989FF001112413
:103D1000E251FE4FEE0DFF1D07C08091C00085FFF0
:103D2000FCCF31969093C60090819923B1F7E7E7D5
:103D3000F2E0949108C08091C00085FFFCCF909381
:103D4000C600319694919923B1F723E832E0E20E50
:103D5000F31ED7014D915D916D917C91EDE7FDEFE3
:103D6000EE0EFF1E8CE096E02AE030E00E94E32891
:103D70008091C00085FFFCCF8AE08093C600A70138
:103D800047515E4FDA012C91E22FF0E0EE0FFF1F5A
:103D9000EE0FFF1FEE0DFF1DE651FE4F83E892E090
:103DA000E80EF91ED701AD90BD90CD90DC908DE767
:103DB0009DEFE80EF91EA082B182C282D3822F5FEE
:103DC000DA012C932FC0E0E1F5E0949108C08091D6
:103DD000C00085FFFCCF9093C60031969491992343
:103DE000B1F7E6E6F2E0949108C08091C00085FF4B
:103DF000FCCF9093C600319694919923B1F7F301CB
:103E000007C08091C00085FFFCCF31969093C6001B
:103E100090819923B1F78091C00085FFFCCF8AE0A3
:103E20008093C600C70182539E4F0E94E47239C03E
:103E3000E9EEF1E0EE0EFF1ED7011C92E7E1FEEF86
:103E4000EE0EFF1EE0E1F5E0949108C08091C00005
:103E500085FFFCCF9093C600319694919923B1F7DA
:103E6000E5E5F2E0949108C08091C00085FFFCCFA9
:103E70009093C600319694919923B1F7F30107C04E
:103E80008091C00085FFFCCF31969093C600908151
:103E90009923B1F78091C00085FFFCCF8AE0809321
:103EA000C600D70112961C921A8A1D8A198A188A8E
:103EB0008DE095E09F878E876EE4A62EB12CAE0C28
:103EC000BF1CEFE2F0E0EE0EFF1ED501ED92FC927A
:103ED000E1EDFFEFEE0EFF1ED3018C918F3209F062
:103EE00090C0C3016FE270E00E9478126C010894E8
:103EF000C11CD11C4E010894811C911C250152E16A
:103F0000252E312C2C0E3D1E77C0C6016FE270E0CD
:103F10000E9478125C01009709F480C0C816D90687
:103F200008F07CC08C010C191D09C401B601A80160
:103F30000E94A112080D191DF8011082F40107C09A
:103F40008091C00085FFFCCF31969093C600908190
:103F50009923B1F78091C00085FFFCCFFAE0F09380
:103F6000C600D2016D917C916115710519F460E074
:103F700070E002C06C5F7F4FC101A40121E00E948C
:103F8000D079882371F5E1E4F2E0949108C0809142
:103F9000C00085FFFCCF9093C60031969491992381
:103FA000B1F7FE01319607C08091C00085FFFCCFBC
:103FB00031969093C60090819923B1F7EFE3F2E038
:103FC000949108C08091C00085FFFCCF9093C600FB
:103FD000319694919923B1F78091C00085FFFCCF71
:103FE00023C12EE030E02C0F3D1FF20131832083EE
:103FF00065010894C11CD11CC114D10409F085CFFE
:104000000BC040E550E0E40EF51ED501ED92FC92A8
:10401000E0EBFFEFEE0EFF1E830101C08601F7010A
:10402000E25BFF4F2DA5222309F4BFC0608171819F
:104030006115710519F460E070E002C06C5F7F4F9C
:10404000C70182539E4FA80121E00E94D0798823A6
:1040500009F47EC04FED51E0E40EF51ED7014D91FD
:104060005D916D917C91ECE9F0E0EE0EFF1ED701C1
:104070004D935D936D937C931397E5E8FDEFEE0E02
:10408000FF1EE1E3F2E0949108C08091C00085FF3B
:10409000FCCF9093C600319694919923B1F7F80123
:1040A00007C08091C00085FFFCCF31969093C60079
:1040B00090819923B1F7E9E2F2E0949108C08091F0
:1040C000C00085FFFCCF9093C60031969491992350
:1040D000B1F78CE096E02AE030E00E94E32880917E
:1040E000C00085FFFCCF8AE08093C60023E832E061
:1040F000E20EF31ED7011D921D921D921C92139782
:10410000EDE7FDEFEE0EFF1EEBE1F2E0949108C04B
:104110008091C00085FFFCCF9093C60031969491AA
:104120009923B1F78091C00085FFFCCF8AE080938E
:10413000C600C70160E070E0A801D1DCD70151964C
:104140008C91882309F498C087010F5E1F4F94C09B
:10415000E7E0F2E0949108C08091C00085FFFCCFB9
:104160009093C600319694919923B1F7F80107C056
:104170008091C00085FFFCCF31969093C60090815E
:104180009923B1F7E5E0F2E0949108C08091C00076
:1041900085FFFCCF9093C600319694919923B1F797
:1041A0008091C00085FFFCCF3FC0608171816115A7
:1041B000710519F460E070E002C06C5F7F4FC701C9
:1041C00082539E4FA80126E50E94D079882381F56D
:1041D000E1EFF1E0949108C08091C00085FFFCCF31
:1041E0009093C600319694919923B1F7F80107C0D6
:1041F0008091C00085FFFCCF31969093C6009081DE
:104200009923B1F7EFEEF1E0949108C08091C000DE
:1042100085FFFCCF9093C600319694919923B1F716
:104220008091C00085FFFCCF8AE08093C60027C044
:1042300081E0F7018083EDEDF1E0949108C0809179
:10424000C00085FFFCCF9093C600319694919923CE
:10425000B1F7F30107C08091C00085FFFCCF319614
:104260009093C60090819923B1F78091C00085FF9B
:10427000FCCF8AE08093C600C8010E9445D4CE01DD
:104280000E960E949915AD960FB6F894DEBF0FBE3C
:10429000CDBFCF91DF911F910F91FF90EF90DF90F5
:1042A000CF90BF90AF909F908F907F906F905F90D6
:1042B0004F903F902F900895EF92FF920F931F938E
:1042C000CF93DF93EC010E94D1838E0107511E4FE3
:1042D000D8018C91BEECEB2EB1E0FB2EEC0EFD1E56
:1042E000882399F1C7010E94E472F801608161504E
:1042F00060838DE8689FB001112462517E4F6C0F7E
:104300007D1FCE0141E021E04BDCD801EC91F0E0D3
:10431000EE0FFF1FEE0FFF1FEC0FFD1FE651FE4FCC
:104320004081518162817381CD57DD4F488359832C
:104330006A837B83C358D240C7010E94CD718B81B1
:10434000882389F181E08A832EC00E94AF83C70150
:104350000E94E4721A828FE291E00E94EB35809114
:104360004A0B882301F110924A0B8091EE08C82F66
:10437000D0E0CC0FDD1FCB56DF4E688179818827D6
:1043800077FD8095982F0E94A0EA209155043091E6
:10439000560440915704509158040E940CEC181692
:1043A00014F419821882DF91CF911F910F91FF9021
:1043B000EF900895FC0181E08183CF0140E021E08E
:1043C000EFCBEF92FF920F931F93DF93CF93CDB775
:1043D000DEB76F970FB6F894DEBF0FBECDBF7C017E
:1043E00088E892E0E80EF91EF7011182108288E752
:1043F0009DEFE80EF91E87010D5C1F4FC80140E0DC
:1044000050E060E070E00E94CD71DE011596F80189
:104410008BE101900D928150E1F7F70181A992A9FA
:104420009C838B838DE095E09A838983C70165E146
:1044300072E08E010F5F1F4FA80120E030E005D928
:10444000C8010E9499156F960FB6F894DEBF0FBE93
:10445000CDBFCF91DF911F910F91FF90EF90089505
:104460000F931F93CF93DF93DC01D3961C92D397C6
:10447000D6961C92D697D2961C921E92D1978DE01A
:1044800095E0D0969C938E939F97AC5ABF4F1C9209
:1044900013961C92A755B040FD01E05BFF4FAE5A4A
:1044A000BF4F11961C921E92A255B04091838083FB
:1044B000ED01C159DF4FFE0120E030E0482F1482AA
:1044C00017821382128240839183215E3F4F7F9631
:1044D00081E02633380799F7A855BE4F89E18C93C0
:1044E00013961C9258961C921B961C9213961C9223
:1044F000A15DB140FD01E653FE4FA453BE4F11969E
:104500001C921E9240839183A155BF4F1D921D9214
:104510001D921C92139718961D921D921D921C922B
:104520001397A358B24012961C92129713961C929E
:1045300013971C9211961C9211978D0101581D4FD3
:10454000F8011082118212821382AB55BE4F119670
:104550001C921E92AC5BBF4F1C92FE01C9011192CE
:104560000197E9F7A256BF4F81E08C93A758B2405C
:104570009E961C921E929D970E9423E268577C4E45
:104580008F4F9F4FF8016083718382839383DF9104
:10459000CF911F910F910895DF93CF93CDB7DEB7E1
:1045A000E0970FB6F894DEBF0FBECDBFDE011196C7
:1045B000E5EBF4E080E101900D928150E1F7DE013E
:1045C0005196E5EAF4E080E101900D928150E1F727
:1045D000DE019196E5E9F4E080E101900D928150D1
:1045E000E1F789819A81AB81BC818093EE0A909337
:1045F000EF0AA093F00AB093F10A89899A89AB89EE
:10460000BC898093DE0A9093DF0AA093E00AB093FE
:10461000E10A89A19AA1ABA1BCA18093FE0A909363
:10462000FF0AA093000BB093010B8D819E81AF8197
:10463000B8858093F20A9093F30AA093F40AB0939A
:10464000F50A8D899E89AF89B88D8093E20A90938F
:10465000E30AA093E40AB093E50A8DA19EA1AFA15D
:10466000B8A58093020B9093030BA093040BB09317
:10467000050B89859A85AB85BC858093F60A909356
:10468000F70AA093F80AB093F90A898D9A8DAB8D39
:10469000BC8D8093E60A9093E70AA093E80AB09352
:1046A000E90A89A59AA5ABA5BCA58093060B9093B2
:1046B000070BA093080BB093090B8D859E85AF85E2
:1046C000B8898093FA0A9093FB0AA093FC0AB093EE
:1046D000FD0A8D8D9E8DAF8DB8A18093EA0A9093CF
:1046E000EB0AA093EC0AB093ED0A8DA59EA5AFA5A9
:1046F000B8A980930A0B90930B0BA0930C0BB0936B
:104700000D0B0E948B5D80E090E8ABE3B5E48093F5
:10471000120B9093130BA093140BB093150B809373
:10472000160B9093170BA093180BB093190B20E066
:1047300030E040E050E020930E0B30930F0B40939D
:10474000100B5093110B80E29EE4A0E0B0E0809348
:10475000DA0A9093DB0AA093DC0AB093DD0A209377
:10476000260B3093270B4093280B5093290B80E0A6
:1047700090E0A0EAB1E480931A0B90931B0BA093F6
:104780001C0BB0931D0B8DEC9CECACECBEE380934A
:104790001E0B90931F0BA093200BB093210B80E076
:1047A00090E0A0EAB0E48093220B9093230BA093B7
:1047B000240BB093250B2093BB083093BC08409387
:1047C000BD085093BE082093B7083093B8084093B3
:1047D000B9085093BA082093B3083093B4084093B3
:1047E000B5085093B6088DEC90E090931711809324
:1047F000161182E390E090931911809318112FEF16
:1048000030E030931B1120931A118BEE90E09093BF
:104810001D1180931C1186E490E090931F118093EA
:104820001E11309321112093201189E29CE5A3E30E
:10483000B1E48093620490936304A0936404B09302
:1048400065046EEA77E481EE9EE30E94218C60931A
:10485000660470936704809368049093690461E729
:104860007DEB8EE892E40E942D8C60936A04709335
:104870006B0480936C0490936D040E941E8B80E007
:1048800090E0A0E8BFE380936E0490936F04A09340
:104890007004B09371041092A20880E090E0A0E44C
:1048A000B0E48093180490931904A0931A04B09371
:1048B0001B0480931C0490931D04A0931E04B093CA
:1048C0001F04A1D6E0E1F5E0949108C08091C000FA
:1048D00085FFFCCF9093C600319694919923B1F750
:1048E000EFE1F3E0949108C08091C00085FFFCCF18
:1048F0009093C600319694919923B1F78091C000AE
:1049000085FFFCCF8AE08093C600E0960FB6F8944E
:10491000DEBF0FBECDBFCF91DF910895CF93DF9360
:10492000C0E1D5E0FE01949108C08091C00085FFF0
:10493000FCCF9093C600319694919923B1F7E9EF9B
:10494000F4E0949108C08091C00085FFFCCF909363
:10495000C600319694919923B1F78091C00085FFEC
:10496000FCCF8AE08093C600FE019491E0E1F5E07F
:1049700008C08091C00085FFFCCF9093C60031969F
:1049800094919923B1F74091EE0A5091EF0A60910A
:10499000F00A7091F10A81EF94E00E94112E40918B
:1049A000F20A5091F30A6091F40A7091F50A8EEEC2
:1049B00094E00E94112E4091F60A5091F70A6091FE
:1049C000F80A7091F90A8BEE94E00E94112E409142
:1049D000FA0A5091FB0A6091FC0A7091FD0A88EE78
:1049E00094E00E94112EE6E1F2E007C08091C00041
:1049F00085FFFCCF31969093C60090819923B1F743
:104A00008091C00085FFFCCF8AE08093C600FE0144
:104A10009491E0E1F5E008C08091C00085FFFCCFF3
:104A20009093C600319694919923B1F7EEECF4E09F
:104A3000949108C08091C00085FFFCCF9093C60080
:104A4000319694919923B1F78091C00085FFFCCFF6
:104A50008AE08093C600FE019491E0E1F5E008C091
:104A60008091C00085FFFCCF9093C6003196949151
:104A70009923B1F74091DE0A5091DF0A6091E00A74
:104A80007091E10A85EC94E00E94112E4091E20AB7
:104A90005091E30A6091E40A7091E50A82EC94E097
:104AA0000E94112E4091E60A5091E70A6091E80AAF
:104AB0007091E90A8FEB94E00E94112E4091EA0A6E
:104AC0005091EB0A6091EC0A7091ED0A8CEB94E046
:104AD0000E94112EE6E1F2E007C08091C00085FF40
:104AE000FCCF31969093C60090819923B1F78091C5
:104AF000C00085FFFCCF8AE08093C600FE01949140
:104B0000E0E1F5E008C08091C00085FFFCCF909304
:104B1000C600319694919923B1F7EEE9F4E09491AF
:104B200008C08091C00085FFFCCF9093C6003196ED
:104B300094919923B1F78091C00085FFFCCF8AE062
:104B40008093C600FE019491E0E1F5E008C08091F9
:104B5000C00085FFFCCF9093C600319694919923B5
:104B6000B1F74091FE0A5091FF0A6091000B7091DD
:104B7000010B85E994E00E94232E4091020B509195
:104B8000030B6091040B7091050B82E994E00E9485
:104B9000232E4091060B5091070B6091080B7091EA
:104BA000090B8FE894E00E94232E40910A0B50914C
:104BB0000B0B60910C0B70910D0B8CE894E00E9434
:104BC000232EE6E1F2E007C08091C00085FFFCCF14
:104BD00031969093C60090819923B1F78091C000DF
:104BE00085FFFCCF8AE08093C600FE019491E0E14E
:104BF000F5E008C08091C00085FFFCCF9093C6000F
:104C0000319694919923B1F7E7E5F4E0949108C0C7
:104C10008091C00085FFFCCF9093C600319694919F
:104C20009923B1F78091C00085FFFCCF8AE0809383
:104C3000C600FE019491E0E1F5E008C08091C0005B
:104C400085FFFCCF9093C600319694919923B1F7DC
:104C50004091120B5091130B6091140B7091150B36
:104C60008EE494E0DED74091160B5091170B6091C3
:104C7000180B7091190B8BE494E0D3D7E6E1F2E0C6
:104C800007C08091C00085FFFCCF31969093C6008D
:104C900090819923B1F78091C00085FFFCCF8AE015
:104CA0008093C600FE019491E0E1F5E008C0809198
:104CB000C00085FFFCCF9093C60031969491992354
:104CC000B1F7E8E9F3E0949108C08091C00085FF56
:104CD000FCCF9093C600319694919923B1F78091BF
:104CE000C00085FFFCCF8AE08093C600FE0194914E
:104CF000E0E1F5E008C08091C00085FFFCCF909313
:104D0000C600319694919923B1F740910E0B5091C2
:104D10000F0B6091100B7091110B8FE893E081D70E
:104D20004091260B5091270B6091280B7091290B15
:104D30008CE893E076D74091DA0A5091DB0A6091D3
:104D4000DC0A7091DD0A89E893E07DD740911A0B67
:104D500050911B0B60911C0B70911D0B86E893E02A
:104D600060D740911E0B50911F0B6091200B7091EA
:104D7000210B83E893E055D74091220B5091230BF0
:104D80006091240B7091250B80E893E04AD7E6E10F
:104D9000F2E007C08091C00085FFFCCF3196909370
:104DA000C60090819923B1F78091C00085FFFCCFA8
:104DB0008AE08093C600FE019491E0E1F5E008C02E
:104DC0008091C00085FFFCCF9093C60031969491EE
:104DD0009923B1F7EEE6F3E0949108C08091C0000A
:104DE00085FFFCCF9093C600319694919923B1F73B
:104DF0008091C00085FFFCCF8AE08093C600FE0151
:104E00009491E0E1F5E008C08091C00085FFFCCFFF
:104E10009093C600319694919923B1F74091B308CD
:104E20005091B4086091B5087091B60885E693E09A
:104E3000F8D64091B7085091B8086091B9087091C0
:104E4000BA0882E693E0EDD64091BB085091BC08C9
:104E50006091BD087091BE088FE593E0E2D6E6E16F
:104E6000F2E007C08091C00085FFFCCF319690939F
:104E7000C60090819923B1F78091C00085FFFCCFD7
:104E80008AE08093C600FE019491E0E1F5E008C05D
:104E90008091C00085FFFCCF9093C600319694911D
:104EA0009923B1F7E1E5F3E0949108C08091C00047
:104EB00085FFFCCF9093C600319694919923B1F76A
:104EC0008091C00085FFFCCF8AE08093C600FE0180
:104ED0009491E0E1F5E008C08091C00085FFFCCF2F
:104EE0009093C600319694919923B1F74091620452
:104EF00050916304609164047091650487E493E0C9
:104F000090D66091660470916704809168049091D6
:104F100069040E94278CAB01BC0184E493E081D634
:104F200060916A0470916B0480916C0490916D049F
:104F30000E94338CAB01BC0181E493E072D6E6E1C0
:104F4000F2E007C08091C00085FFFCCF31969093BE
:104F5000C60090819923B1F78091C00085FFFCCFF6
:104F60008AE08093C600DF91CF9108951F920F923F
:104F70000FB60F920BB60F9211242F933F934F93BE
:104F80008F939F93EF93FF934091C600E0910806A3
:104F9000F091090631969F012F77307031978091FB
:104FA0000A0690910B062817390739F0E857FA4F8F
:104FB00040833093090620930806FF91EF919F915B
:104FC0008F914F913F912F910F900BBE0F900FBE7D
:104FD0000F901F9018959A01AB01203081EE380791
:104FE00080E0480780E0580749F182E08093C000E4
:104FF00060E079E08DE390E00E9424EE21503040A3
:1050000040405040CA01B90122E030E040E050E0A9
:105010000E9424EE3093C5002093C4008091C1000B
:1050200080618093C1008091C10088608093C1003D
:105030008091C10080688093C10008951092C000E3
:1050400020E130E0E7CF20910A0630910B068091F5
:105050000806909109068217930719F42FEF3FEF86
:105060000EC0F901E857FA4F80812F5F3F4F2F772D
:10507000307030930B0620930A06282F30E0C901C8
:10508000089580910A0690910B06909309068093EB
:105090000806089508952F923F924F925F926F9263
:1050A0007F928F929F92AF92BF92CF92DF92EF92B8
:1050B000FF920F931F93DF93CF93CDB7DEB7A097E7
:1050C0000FB6F894DEBF0FBECDBF1C016A017B0195
:1050D000411551056105710541F440E350E060E080
:1050E00070E020E030E08BD055C088249924540132
:1050F000422E55246624772401E010E00C0F1D1F7A
:10510000080D191DC701B601A30192010E9402EE0C
:10511000F80160830894811C911CA11CB11CC7017B
:10512000B601A30192010E9402EEC901DA016C01ED
:105130007D01C114D104E104F104F1F681E0E82E0F
:10514000F12CEC0EFD1EE80CF91C3E010894611CCC
:10515000711CD501C4010197A109B1096C01C818DE
:10516000D90815C0F601EE0DFF1D40814A3010F43C
:10517000405D01C0495C552747FD5095652F752F4F
:10518000C10120E030E03BD00894E108F1086E1442
:105190007F0441F7A0960FB6F894DEBF0FBECDBFD7
:1051A000CF91DF911F910F91FF90EF90DF90CF9003
:1051B000BF90AF909F908F907F906F905F904F9037
:1051C0003F902F9008952115310539F48091C0004A
:1051D00085FFFCCF4093C60008955DCFEF92FF920C
:1051E0000F931F939A01E62EFF2400E010E0B80110
:1051F000A701E9DF1F910F91FF90EF900895EF92C3
:10520000FF920F931F93CF93DF93EC017A018B01F1
:105210002115310539F48091C00085FFFCCFE09263
:10522000C60019C02A303105A9F477FF0FC04DE23E
:1052300050E060E070E020E030E0E1DF10950095A4
:10524000F094E094E11CF11C011D111DCE01B80188
:10525000A7012AE020DFDF91CF911F910F91FF90EE
:10526000EF900895EF92FF920F931F937B019A01A5
:105270000027F7FC0095102FB801A701C0DF1F9190
:105280000F91FF90EF9008950F931F938C014DE0C5
:1052900050E060E070E020E030E0B1DFC8014AE0BB
:1052A00050E060E070E020E030E0A9DF1F910F9156
:1052B0000895CF92DF92EF92FF920F931F938C018C
:1052C0009A016B01EE24FF24B701A6017CDFC8011F
:1052D000DBDF1F910F91FF90EF90DF90CF9008954B
:1052E0009F92AF92BF92CF92DF92EF92FF920F9375
:1052F0001F93CF93DF93EC017A018B01922ECB01A8
:10530000BA0120E030E040E050E00E94FEE988234E
:1053100064F4CE014DE250E060E070E020E030E067
:105320006EDF17FB109517F91095AA2420E030E0E6
:1053300040E05FE30BC0CA01B90120E030E040E289
:1053400051E40E9405EA9B01AC01A394A91498F3CF
:10535000C801B7010E9425E97B018C010E9472EA15
:105360005B016C010E949EEA9B01AC01C801B70180
:105370000E9424E97B018C01CE01B601A5012AE03F
:1053800030E021DF992099F1E7E1F2E007C0809158
:10539000C00085FFFCCF31969093C6009081992381
:1053A000B1F725C0C801B70120E030E040E251E488
:1053B0000E94DEEC7B018C010E946DEA5B016C01B6
:1053C000CC24B7FCC094DC2CCE01B601A5012AE0A8
:1053D00030E015DFC601B5010E94A0EA9B01AC01D7
:1053E000C801B7010E9424E97B018C019A9499209D
:1053F000C9F6DF91CF911F910F91FF90EF90DF9051
:10540000CF90BF90AF909F9008956ACF0895EF928C
:10541000FF920F931F93CF93DF93EC01E09028044A
:10542000F090290400912A0410912B04688179815D
:105430008A819B81A80197010E940CEC181624F424
:10544000E882F9820A831B83E0902C04F0902D04FB
:1054500000912E0410912F046C817D818E819F819B
:10546000A80197010E940CEC181624F4EC82FD822E
:105470000E831F83E0903004F090310400913204D9
:1054800010913304688579858A859B85A8019701E9
:105490000E940CEC181624F4E886F9860A871B870C
:1054A000DF91CF911F910F91FF90EF900895809120
:1054B000FB0808950F931F93CF93DF9381309105DD
:1054C000A9F46F5F7F4F09F052C08EE096E00E9412
:1054D00030228CEF98E00E94A47F8FEF98E00E942A
:1054E000A47F82E099E00E94A47F41C0892B09F04B
:1054F0003EC06F5F7F4FD9F58DE095E09093D9075F
:105500008093D8078091DF07882321F08CED97E006
:105510000E94E472C4E9D7E00DE015E005C06F9782
:1055200086E0CE35D80751F0198308838F81882310
:10553000B1F3CE0104960E94E472F1CF8DE095E0C4
:10554000998388838F81882321F0CE0104960E945D
:10555000E4728DE095E090933E0680933D06809145
:105560004406882321F081E496E00E94E472DF91F2
:10557000CF911F910F91089580E090E06FEF7FEF42
:1055800099CF81E090E06FEF7FEF94CFEF92FF92A1
:105590000F931F939B01AC018091A208882321F1F6
:1055A000CA01B90120E030E040E05FE30E94DEEC98
:1055B0007B018C0120E030E040E050E00E94FEE9F9
:1055C000882391F0C801B701A80197010E94DEEC81
:1055D0009B01AC01CA012BED3FE049E450E40E947D
:1055E000DEEC9B01AC0104C020E030E040E85FE36A
:1055F00060E070E080E89FE30E9405EA1F910F9150
:10560000FF90EF90089560911804709119048091B3
:105610001A0490911B04BADF609320047093210454
:10562000809322049093230460911C0470911D04C4
:1056300080911E0490911F04A9DF6093240470934D
:105640002504809326049093270408950E94FD8BDF
:105650008091FB08882309F03AC081E08093FB0821
:105660008091070990910809A0910909B0910A0950
:1056700080930B0990930C09A0930D09B0930E0928
:10568000E9E0F5E0949108C08091C00085FFFCCF6F
:105690009093C600319694919923B1F7EEE1F5E02D
:1056A000949108C08091C00085FFFCCF9093C60004
:1056B000319694919923B1F78091C00085FFFCCF7A
:1056C0008AE08093C60086E195E00C9431D4089579
:1056D000CF93DF93F8940E94FD8B5F9A1092D708C6
:1056E0008A9A1092D8088FB7F89490910801916027
:1056F000909308018FBF1092D908129A479A8CE0B4
:1057000060E00E94D4E3E9E0F5E0949108C0809164
:10571000C00085FFFCCF9093C600319694919923E9
:10572000B1F7E5EAF5E0949108C08091C00085FFEB
:10573000FCCF9093C600319694919923B1F7809154
:10574000C00085FFFCCF8AE08093C60084E995E025
:105750000E943FD47894C5E0D0E008C068EC70E0C7
:1057600080E090E00E9431E20E948FD421978FEF79
:10577000CF3FD80799F7F894FFCF0E9423E26093B8
:105780001109709312098093130990931409E09101
:105790004009F0914109EE5BF64F80818823A9F41E
:1057A000E4ECF5E0949108C08091C00085FFFCCF47
:1057B0009093C600319694919923B1F78091C000DF
:1057C00085FFFCCF8AE08093C60008950E9423E203
:1057D000609311097093120980931309909314092F
:1057E00008956F927F928F929F92AF92BF92CF92C5
:1057F000DF92EF92FF920F931F93F82E60911F0993
:10580000709120098091210990912209209123090A
:105810003091240940912509509126090E9419ECE4
:105820003B014C0100D000D00DB71EB70F5F1F4FDA
:105830006091100470911104882777FD8095982F4E
:105840000E94A0EA20914C0430914D0440914E04F6
:1058500050914F040E94DEEC20E030E040E752E43B
:105860000E9405EA20E030E048EC52E40E9405EA9C
:105870005B016C01F8016082718282829382F48202
:105880008091EE08858383EA98E06BE279E04FE14E
:1058900059E020E001E032E0E32E0E948758809139
:1058A0002B0990912C09A0912D09B0912E0980937C
:1058B000A3089093A408A093A508B093A60880918C
:1058C0002F0990913009A0913109B091320980934C
:1058D000A7089093A808A093A908B093AA0880915C
:1058E000330990913409A0913509B091360980931C
:1058F000AB089093AC08A093AD08B093AE0880912C
:10590000370990913809A0913909B0913A098093EB
:10591000AF089093B008A093B108B093B2088DB7C8
:105920009EB706960FB6F8949EBF0FBE8DBF0E941D
:1059300023E26093110970931209809313099093E5
:1059400014091F910F91FF90EF90DF90CF90BF90BF
:10595000AF909F908F907F906F900895CF92DF923D
:10596000EF92FF920F931F93E0902804F090290488
:1059700000912A0410912B0460912B0970912C093D
:1059800080912D0990912E09A80197010E940CEC9D
:10599000181644F4E0922B09F0922C0900932D097B
:1059A00010932E09E0902C04F0902D0400912E0409
:1059B00010912F0460912F09709130098091310965
:1059C00090913209A80197010E940CEC181644F43A
:1059D000E0922F09F09230090093310910933209B7
:1059E000E0903004F09031040091320410913304BF
:1059F000609133097091340980913509909136098D
:105A0000A80197010E940CEC181644F4E0923309A7
:105A1000F092340900933509109336090E9423E26D
:105A200060931109709312098093130990931409DC
:105A30006091A3087091A4088091A5089091A60890
:105A400020912B0930912C0940912D0950912E095C
:105A50000E94FEE9882309F07AC06091A70870913E
:105A6000A8088091A9089091AA0820912F09309147
:105A7000300940913109509132090E94FEE9882392
:105A800009F065C060914C0470914D0480914E0402
:105A900090914F0420E030E040E752E40E9405EA94
:105AA0007B018C018BE299E06FE279E043E359E0FE
:105AB00027E339E0EEEECE2EE8E0DE2E0E94D9623A
:105AC00080912B0990912C09A0912D09B0912E095C
:105AD0008093A3089093A408A093A508B093A60868
:105AE00080912F0990913009A0913109B09132092C
:105AF0008093A7089093A808A093A908B093AA0838
:105B00008091330990913409A0913509B0913609FB
:105B10008093AB089093AC08A093AD08B093AE0807
:105B20008091370990913809A0913909B0913A09CB
:105B30008093AF089093B008A093B108B093B208D7
:105B40001F910F91FF90EF90DF90CF90089560919B
:105B5000100470911104882777FD8095982F0E947A
:105B6000A0EA20914C0430914D0440914E04509194
:105B70004F040E94DEEC20E030E040E752E40E9457
:105B800005EA20E030E048EC52E488CF8CE096E073
:105B900078DAE7ECF5E0949108C08091C00085FFC9
:105BA000FCCF9093C600319694919923B1F7409120
:105BB0000709509108096091090970910A094F5F1E
:105BC0005F4F6F4F7F4F8CE096E02AE030E017DBAD
:105BD0008091C00085FFFCCF8AE08093C600CDCDC8
:105BE000409140095091410920E630E0B901469FBB
:105BF0009001479F300D569F300D1124682F772755
:105C000067FD7095C901845B964F0E9478129C01D4
:105C100090934B0980934A0980E0232B09F081E09F
:105C20000895FC01949108C08091C00085FFFCCFCD
:105C30009093C600319694919923B1F78CE096E049
:105C400022E030E0E2CBFC01949108C08091C000DA
:105C500085FFFCCF9093C600319694919923B1F7BC
:105C60008CE096E02AE030E0AECA2F923F924F924D
:105C70005F926F927F928F929F92AF92BF92CF92DC
:105C8000DF92EF92FF920F931F93DF93CF9300D099
:105C900000D0CDB7DEB79E838D838330910508F0A9
:105CA000CAC1FC01E359F74FD4908C01000F111FBA
:105CB000000F111FF801ED55F74F80E090E0A0E0D4
:105CC000B0E080839183A283B38383EA98E067EA9C
:105CD00078E04BEA58E02FEA38E00E94D35DED818E
:105CE000FE81EE0FFF1FEC5CFB4F0190F081E02D79
:105CF000F7FD0EC0CF01880F991F8E0F9F1F065C06
:105D00001B4FD8016D917C918450974F0E946D80FC
:105D1000AD80BE80AA0CBB1CAA0CBB1CF501E059CF
:105D2000F74FE590F590059114916D2D772767FD5C
:105D30007095882777FD8095982F0E94A0EA698347
:105D40007A838B839C83FBE2CF2EF9E0DF2ECA0C93
:105D5000DB1CC801B70120E030E040EC5FE30E94AB
:105D6000DEEC29813A814B815C810E94DEECF601F8
:105D70006083718382839383F501E050FC4F6081DF
:105D800071818281938160934C0470934D04809360
:105D90004E0490934F0420E030E040E752E40E942C
:105DA00005EA7B018C018BE299E06FE279E043E345
:105DB00059E027E339E0EEEECE2EE8E0DE2E0E9439
:105DC000D9620E94D18380910D06882301F18D81D3
:105DD0000E949D830E94A0EAF501E251F54F2081C7
:105DE0003181428153810E9405EA9B01AC018FEB16
:105DF00098E0A80EB91EC901DA01F50180839183EC
:105E0000A283B38387E698E0A901BD010ADF0E945F
:105E1000D1836D807E80660C771C660C771CA3EAAC
:105E20002A2EA8E03A2E260C371C80E090E0A0E055
:105E3000B0E0F10180839183A283B38383EA98E089
:105E400067EA78E04BEA58E02FEA38E00E94D35D39
:105E5000F301E458F74F85909590A590B490FBE23C
:105E60004F2EF9E05F2E460C571CC501B401905827
:105E700029813A814B815C810E94DEECD2016D93D5
:105E80007D938D939C93139760914C0470914D0476
:105E900080914E0490914F0420E030E040E752E4BE
:105EA0000E9405EA7B018C018BE299E06FE279E0C8
:105EB00043E359E027E339E0EEEECE2EE8E0DE2EB4
:105EC0000E94D9620E94D183C501B401A501940149
:105ED0000E9425E929813A814B815C810E94DEEC98
:105EE000F2016083718382839383F301E050FC4F5E
:105EF000608171818281938120E030E040E05FE346
:105F00000E94DEEC60934C0470934D0480934E0429
:105F100090934F0420E030E040E752E40E9405EA0D
:105F20007B018C018BE299E06FE279E043E359E079
:105F300027E339E00E94D9620E94D183F301E85738
:105F4000F74F6591759185919491F301ED54F74F59
:105F5000A080B180C280D380A60195010E9425E96E
:105F60007B018C01CB01D801F10180839183A28355
:105F7000B383F301EC56F74F659175918591949138
:105F80002BEC822E28E0922E860C971CA601950100
:105F90000E9425E9D4016D937D938D939C93139773
:105FA000F301E056F74F6591759185919491E8E280
:105FB000F4E06E0E7F1EA60195010E9425E9D30133
:105FC0006D937D938D939C931397C701D801F20134
:105FD00080839183A283B38380E090E0A0E0B0E06F
:105FE00080934C0490934D04A0934E04B0934F04BF
:105FF0000E94BE82ED81FE81E952F74F81E08083ED
:10600000AD81BE81AA0FBB1FFD01EC5CFB4F01906F
:10601000F081E02DF7FD0FC0CF01880F991F8E0F83
:106020009F1FAA0FBB1FA45CBB4F6D917C91845036
:10603000974F0E946D8026960FB6F894DEBF0FBE74
:10604000CDBFCF91DF911F910F91FF90EF90DF9027
:10605000CF90BF90AF909F908F907F906F905F9008
:106060004F903F902F90089580914A0990914B094D
:10607000019660E070E04AE050E00C94C41080911A
:106080004A0990914B09019660E070E00C94670F0B
:10609000CF93DF93EC018091EE088093060984E5AD
:1060A0009FDD882309F480C0EADF0E9472EA262F70
:1060B00060930609623008F477C0E0E1F5E094915E
:1060C00008C08091C00085FFFCCF9093C600319638
:1060D00094919923B1F7CD36D105C1F0CE36D105D3
:1060E00044F4C836D105C1F0C936D10509F04DC018
:1060F00010C0CA3DD10539F0CD3DD10509F045C0EC
:10610000E9E1F2E03FC0E0E3F2E031C0E7E4F2E0D1
:1061100023C0EEE5F2E015C0E5E7F2E007C08091AC
:10612000C00085FFFCCF31969093C60090819923E3
:10613000B1F72BC08091C00085FFFCCF31969093C2
:10614000C60090819923B1F720C08091C00085FFDF
:10615000FCCF31969093C60090819923B1F715C07A
:106160008091C00085FFFCCF31969093C60090814E
:106170009923B1F70AC08091C00085FFFCCF31960A
:106180009093C60090819923B1F78CE096E0622F3E
:1061900040E050E023D88091C00085FFFCCF8AE02A
:1061A0008093C60081E001C080E0DF91CF91089527
:1061B000AF92BF92CF92DF92EF92FF920F931F9315
:1061C000CF93DF9323EAE22E28E0F22ECBE2D9E050
:1061D00000E010E0F801EB53FB4F808101DD8823E4
:1061E00031F14DDF5B016C01F801E456F74F80811E
:1061F000882311F061E002C060913B0970E08827BC
:1062000077FD8095982F0E94A0EAF70120813181C7
:10621000428153810E94DEEC9B01AC01C601B501B5
:106220000E9425E9688379838A839B8309C0F701EB
:1062300080819181A281B38188839983AA83BB8362
:106240000F5F1F4F84E090E0E80EF91E24960430A3
:10625000110509F0BFCF86E4C3DC8823D9F00FDF36
:106260007B018C0160933C0970933D0980933E094A
:1062700090933F0920E030E040E050E00E940CECB9
:10628000181644F4E0924C04F0924D0400934E042E
:1062900010934F04DF91CF911F910F91FF90EF90DA
:1062A000DF90CF90BF90AF90089582DF89E498DCB3
:1062B000882351F0E4DE60931F09709320098093D6
:1062C0002109909322090CC080E090E0A0E0B0E0AA
:1062D00080931F0990932009A0932109B09322096C
:1062E0008AE47EDC882351F0CADE60932309709330
:1062F00024098093250990932609089580E090E071
:10630000A0E0B0E08093230990932409A09325098D
:10631000B093260908952F923F924F925F926F9209
:106320007F928F929F92AF92BF92CF92DF92EF9225
:10633000FF920F931F93DF93CF93CDB7DEB76E9786
:106340000FB6F894DEBF0FBECDBF70E6A72EB12CFE
:10635000E3EDF8E094906AE0762E8824839414C2EA
:106360002D3071F02A3321F48091D00A882341F036
:106370008091D10A9091D20A8F3591050CF4DAC13F
:10638000E091D10AF091D20A309709F408C3A091A4
:10639000D30AB091D40AAA9D7001AB9DF00CBA9DAE
:1063A000F00C1124EE0DFF1DE45BF64F108280917E
:1063B000D00A882309F0B9C11092D00AAE5BB64F5B
:1063C0001C928701045B164FC8016EE470E00E94C6
:1063D00078129C01009709F4F6C090934B098093C2
:1063E0004A092F5F3F4F201B310B2E0D3F1DC90166
:1063F000845B964F60E070E04AE050E00E94C41079
:106400006093D50A7093D60A8093D70A9093D80ADE
:10641000C0900709D0900809E0900909F0900A0996
:10642000A70196012F5F3F4F4F4F5F4F62177307D2
:106430008407950709F461C38091D30A9091D40A27
:106440009C012A9DC0012B9D900D3A9D900D112419
:10645000845B964F6FEE79E00E942A12892B09F037
:106460004CC3E9E0F5E0949108C08091C00085FF3D
:10647000FCCF9093C600319694919923B1F7ECEB41
:10648000F9E0949108C08091C00085FFFCCF909303
:10649000C600319694919923B1F78CE096E0B7014C
:1064A000A6012AE030E00E94FF288091C00085FF0D
:1064B000FCCF73C0FE264F5FFC01E40FF11DE45BCF
:1064C000F64FE081EA32B1F730934B0920934A0945
:1064D000C901019660E070E00E94670F0E946DEABA
:1064E0002F2D30E02617370709F45CC0E9E0F5E00E
:1064F000949108C08091C00085FFFCCF9093C600A6
:10650000319694919923B1F7EDE9F9E0949108C09F
:106510008091C00085FFFCCF9093C6003196949186
:106520009923B1F740910709509108096091090931
:1065300070910A098CE096E02AE030E00E94FF2882
:106540008091C00085FFFCCF28C0E9E0F5E0949180
:1065500008C08091C00085FFFCCF9093C6003196A3
:1065600094919923B1F7E3E7F9E0949108C0809101
:10657000C00085FFFCCF9093C6003196949199237B
:10658000B1F78CE096E0B701A6012AE030E00E9466
:10659000FF288091C00085FFFCCF8AE08093C60071
:1065A000F5DA4AC08091D50A9091D60AA091D70A0F
:1065B000B091D80A8093070990930809A09309091C
:1065C000B0930A093EC0C8016AE270E00E947812E6
:1065D000009709F436C0E9E0F5E0949108C0809195
:1065E000C00085FFFCCF9093C6003196949199230B
:1065F000B1F7E9E4F9E0949108C08091C00085FF0B
:10660000FCCF9093C600319694919923B1F74091B5
:106610000709509108096091090970910A098CE0F5
:1066200096E02AE030E00E94FF288091C00085FFBC
:10663000FCCF8AE08093C6001092D20A1092D10A51
:106640007BC28091D30A9091D40A8A9D70018B9D60
:10665000F00C9A9DF00C11248701045B164FC801C1
:1066600067E470E00E9478129C01009791F190938A
:106670004B0980934A092F5F3F4F201B310B2E0D92
:106680003F1DC901845B964F60E070E00E94670F78
:106690000E946DEA64307105E0F48091FB08882364
:1066A000C1F0992DE3EDF8E008C08091C00085FFAE
:1066B000FCCF9093C600319694919923B1F78091C5
:1066C000C00085FFFCCF7092C6008BEC98E00E9462
:1066D00031D48091D30A9091D40AFC01EA9DC00183
:1066E000EB9D900DFA9D900D1124845B964F6CE804
:1066F00072E00E948312009711F40E94682B80912F
:10670000D30A9091D40A019664E070E00E94EFED04
:106710009093D40A8093D30A80910F099091100925
:1067200001969093100980930F091092D20A10924B
:10673000D10A2AC02B3311F48092D00A8091CF0A5B
:10674000883211F48092D00A8091D00A8823E1F433
:106750002091D10A3091D20A8091D30A9091D40A23
:106760008A9DF0018B9DF00D9A9DF00D1124E20F92
:10677000F31FE45BF64F8091CF0A80832F5F3F4F7A
:106780003093D20A2093D10A80910806909109068D
:1067900020910A0630910B06821B930B8F77907025
:1067A000892B09F4C4C180910F09909110090497B5
:1067B0000CF0BDC18CE096E00E942328282F809326
:1067C000CF0A8A3009F0CCCDDBCD8091D10A9091EF
:1067D000D20A892B09F0B0C180910F09909110095C
:1067E000892B09F038C11092D90A35C14D3099F082
:1067F000433211F04A3321F48091D00A882359F0B2
:106800008091D10A9091D20A8F35910524F42F5F9F
:106810003F4F09F0F5C020919108309192084091C6
:106820009308509194088091890890918A08A091CA
:106830008B08B0918C08281739074A075B0708F4C2
:10684000A1C0932DE8EBF8E008C08091C00085FF5F
:10685000FCCF9093C600319694919923B1F7809123
:10686000C00085FFFCCF2092C6000E9423E2609307
:10687000F7087093F8088093F9089093FA0820912C
:10688000F3083091F4084091F5085091F608621B26
:10689000730B840B950B28EE33E040E050E00E9430
:1068A00002EEF22EE32ED42EC52E2DB73EB7285081
:1068B00030400FB6F8943EBF0FBE2DBF0DB71EB7C8
:1068C0000F5F1F4FEDB7FEB7B282A182F80153826E
:1068D00042826F2D7E2D842F952F20E13EE040E0F7
:1068E00050E00E9402EEF801358324836F2D7E2D47
:1068F0008D2D9C2D2CE330E040E050E00E9402EE14
:10690000CA01B9012CE330E040E050E00E9402EE01
:10691000F801778366830E94B012982DE0E1F5E0DC
:106920002DB73EB7285F3F4F0FB6F8943EBF0FBE5E
:106930002DBF08C08091C00085FFFCCF9093C6009A
:10694000319694919923B1F7F50107C08091C00069
:1069500085FFFCCF31969093C60090819923B1F7C3
:106960008091C00085FFFCCF2092C600C5010E9427
:1069700045D48EE096E00E945C218EE096E061E0D6
:106980000E94001A8091CF0A833211F49092D90AA2
:106990002091D10A3091D20A2115310519F41092B3
:1069A000D00ACAC08091D30A9091D40A869DF00182
:1069B000879DF00D969DF00D1124E20FF31FE45B0F
:1069C000F64F1082FC01EE5BF64F908220910F098A
:1069D000309110092F5F3F4F3093100920930F091A
:1069E000019664E070E00E94EFED9093D40A8093EA
:1069F000D30A1092D00A1092D20A1092D10A40C043
:106A00004B3311F49092D00A8091CF0A883211F45E
:106A10009092D00A8091D00A882391F52091D10AD2
:106A20003091D20A8091D30A9091D40A869DF001C8
:106A3000879DF00D969DF00D1124E20FF31FE45B8E
:106A4000F64F8091CF0A80832F5F3F4F3093D20A59
:106A50002093D10A15C050E6652E712C9924939489
:106A6000E8EBF8E034904AE0242E5E010894A11C83
:106A7000B11C3CEA432E38E0532EE0E1F5E084906F
:106A80002091910830919208409193085091940878
:106A90008091890890918A08A0918B08B0918C0808
:106AA000281739074A075B0708F046C080910F098D
:106AB0009091100904970CF03FC08091D90A882367
:106AC000D9F58091E4079091E507A091E607B09190
:106AD000E7078093910890939208A0939308B0934E
:106AE00094088CED97E00E9484759C01482F809358
:106AF000CF0A8A3009F07ACE8ECE8091D30A909157
:106B0000D40A8A9D80018B9D100D9A9D100D112431
:106B1000C801845B964F6AE270E00E9478129C0183
:106B2000009709F412CDFF2440E0C801C5CC809144
:106B30001006882309F049CE6E960FB6F894DEBF92
:106B40000FBECDBFCF91DF911F910F91FF90EF90BE
:106B5000DF90CF90BF90AF909F908F907F906F907D
:106B60005F904F903F902F9008950F931F93CF9376
:106B7000DF938CEF98E06BE070E00E9470818FEF04
:106B800098E066E070E00E94708182E099E065E044
:106B900070E00E947081C4E3D4E00CE314E028812B
:106BA000398137FD0CC0C901880F991F820F931FCF
:106BB000F801608171818450974F0E946D80229608
:106BC0000C5F1F4FF4E0CA33DF0749F7DF91CF9125
:106BD0001F910F910895BC0180910F0990911009A8
:106BE00004970CF070C02091D30A3091D40A80E64B
:106BF00090E0AC01249FC001259F900D349F900D23
:106C00001124845B964F0E94F311E0E1F5E094912A
:106C100008C08091C00085FFFCCF9093C6003196DC
:106C200094919923B1F7E0EFFAE0949108C0809134
:106C3000C00085FFFCCF9093C600319694919923B4
:106C4000B1F72091D30A3091D40A80E690E0289FD2
:106C5000F001299FF00D389FF00D1124E45BF64FF1
:106C600007C08091C00085FFFCCF31969093C6008D
:106C700090819923B1F7EEEEFAE0949108C08091EB
:106C8000C00085FFFCCF9093C60031969491992364
:106C9000B1F78091C00085FFFCCF8AE08093C600E9
:106CA000C901019664E070E00E94EFED9093D40A70
:106CB0008093D30A80910F099091100901969093C7
:106CC000100980930F090895BC0180910F099091DC
:106CD000100904970CF070C02091D30A3091D40AA7
:106CE00080E690E0AC01249FC001259F900D349F69
:106CF000900D1124845B964F0E948C12E0E1F5E028
:106D0000949108C08091C00085FFFCCF9093C6008D
:106D1000319694919923B1F7EDEFFAE0949108C080
:106D20008091C00085FFFCCF9093C600319694916E
:106D30009923B1F72091D30A3091D40A80E690E0EC
:106D4000289FF001299FF00D389FF00D1124E45B7E
:106D5000F64F07C08091C00085FFFCCF319690931D
:106D6000C60090819923B1F7EBEFFAE0949108C047
:106D70008091C00085FFFCCF9093C600319694911E
:106D80009923B1F78091C00085FFFCCF8AE0809302
:106D9000C600C901019664E070E00E94EFED909397
:106DA000D40A8093D30A80910F099091100901961B
:106DB0009093100980930F0908958091CC0A9091C7
:106DC000CD0A892BE9F48091CE0A8823C9F08091FD
:106DD00010068823A9F081E090E09093CD0A80937B
:106DE000CC0A81E992E070DF86E992E06DDF86E906
:106DF00092E06ADF86E992E067DF86E992E064CF9D
:106E00000895DF92EF92FF920F931F93D82E8091F7
:106E10000F099091100903970CF47DDA0E9423E288
:106E2000E0901509F09016090091170910911809C2
:106E300020911109309112094091130950911409C0
:106E4000621B730B840B950BE616F70608071907F0
:106E500038F4E114F1040105110511F00E94682BCA
:106E60000E9423E2E0901909F0901A0900911B0991
:106E700010911C09209111093091120940911309B8
:106E800050911409621B730B840B950BE616F706E1
:106E900008071907C0F4E114F1040105110599F080
:106EA00010929610109295101092981010929710C0
:106EB00010929A10109299101092F0081092EF0808
:106EC0008CE992E001DF8091480490914904A091FF
:106ED0004A04B0914B040097A105B105A9F10E94A5
:106EE00023E2209111093091120940911309509128
:106EF0001409621B730B840B950B2091480430918D
:106F0000490440914A0450914B042617370748071B
:106F10005907D0F49091B60D8091B70D9817A1F450
:106F2000DD2091F45F9A1092D7088A9A1092D808BF
:106F30009FB7F894809108018160809308019FBFFA
:106F40001092D908129A479A4A9916C020911D09A1
:106F500030911E092F5F3F4F30931E0920931D096A
:106F600080911006882341F0215137422CF025DF13
:106F700010921E0910921D090E94F85F1F910F9137
:106F8000FF90EF90DF9008952F923F924F925F9283
:106F90006F927F928F929F92AF92BF92CF92DF9229
:106FA000EF92FF920F931F93DF93CF93CDB7DEB78E
:106FB000EE970FB6F894DEBF0FBECDBF87E40E94F8
:106FC000F02D882309F434C55AD80E946DEA6A313D
:106FD000710509F49CC06B3171059CF46230710538
:106FE000B1F16330710524F4772334F50C940E5617
:106FF00063307105C1F16430710511F00C940E56C7
:107000003EC06A35710509F4BEC46B35710554F490
:107010006B31710509F401C26C31710511F00C94EA
:107020000E566EC36B35710509F4B1C46C3571052C
:1070300011F00C940E56B0C48091FB08882311F017
:107040000C940E56B5D80E94AE2C0C940E5680911E
:10705000FB08882311F00C940E5627D981E00E947A
:10706000F12B0C940E568091FB08882311F00C94A0
:107070000E561BD980E00E94F12B0C940E568EE523
:1070800098E00E9431D480E50E94F02D882321F4FD
:10709000EE24FF24870106C00E943F300E9472EA5E
:1070A0007B018C0183E50E94F02D882361F00E9412
:1070B0003F3020E030E04AE754E40E94DEEC0E94DA
:1070C00072EA7B018C010E94D1830E9423E25B0162
:1070D0006C01AE0CBF1CC01ED11E0E9423E2609347
:1070E000110970931209809313099093140906C033
:1070F0000E94CF9080E085DE0E948FD40E9423E220
:107100006A157B058C059D0598F30C940E5681E05D
:1071100080930D0680914C0490914D04A0914E04F3
:10712000B0914F048093460990934709A093480972
:10713000B093490980911004909111049093A10893
:107140008093A00884E690E090931104809310044B
:107150000E9423E26093110970931209809313092E
:107160009093140981E00E94C5828091A3089091B8
:10717000A408A091A508B091A60880932B0990932C
:107180002C09A0932D09B0932E098091A708909106
:10719000A808A091A908B091AA0880932F099093FC
:1071A0003009A0933109B09332098091AB089091D6
:1071B000AC08A091AD08B091AE08809333099093CC
:1071C0003409A0933509B09336098091AF089091A6
:1071D000B008A091B108B091B2088093370990939C
:1071E0003809A0933909B0933A0980E090E0A0E013
:1071F000B0E080934C0490934D04A0934E04B09360
:107200004F0488E50E94F02D882361F489E50E94EF
:10721000F02D882339F48AE50E94F02D882311F49B
:1072200081E001C080E080935004882329F488E540
:107230000E94F02D882321F080E090E00E94352EFE
:1072400080915004882329F489E50E94F02D882339
:1072500021F081E090E00E94352E88E50E94F02D1B
:107260008823D9F00E94343061157105810591059C
:10727000A1F00E943F302091B3083091B4084091B2
:10728000B5085091B6080E9425E96093A308709351
:10729000A4088093A5089093A60889E50E94F02D84
:1072A0008823D9F00E94343061157105810591055C
:1072B000A1F00E943F302091B7083091B80840916A
:1072C000B9085091BA080E9425E96093A708709305
:1072D000A8088093A9089093AA0880915004882355
:1072E00029F48AE50E94F02D882321F082E090E0C5
:1072F0000E94352E8AE50E94F02D8823D9F00E9445
:1073000034306115710581059105A1F00E943F306F
:107310002091BB083091BC084091BD085091BE0837
:107320000E9425E96093AB087093AC088093AD0888
:107330009093AE0883EA98E067EA78E04BEA58E079
:107340002FEA38E00E94D35D8091BF089091C00879
:10735000A091C108B091C2088093A3089093A4089B
:10736000A093A508B093A6088091C3089091C40883
:10737000A091C508B091C6088093A7089093A8086B
:10738000A093A908B093AA088091C7089091C80853
:10739000A091C908B091CA088093AB089093AC083B
:1073A000A093AD08B093AE0883EA98E067EA78E06E
:1073B0004BEA58E02FEA38E00E94D35D80E00E945B
:1073C000C5828091460990914709A0914809B091E2
:1073D000490980934C0490934D04A0934E04B093BC
:1073E0004F048091A0089091A1089093110480937C
:1073F00010040E9423E26093110970931209809394
:107400001309909314090E94BE8285EB92E00E94BA
:1074100045D410920D060C940E5680914C04909118
:107420004D04A0914E04B0914F048093460990936F
:107430004709A0934809B09349098091100490919D
:1074400011049093A1088093A00884E690E09093A3
:107450001104809310040E9423E260931109709339
:107460001209809313099093140981E00E94C58248
:107470008091A3089091A408A091A508B091A608B6
:1074800080932B0990932C09A0932D09B0932E097A
:107490008091A7089091A808A091A908B091AA0886
:1074A00080932F0990933009A0933109B09332094A
:1074B0008091AB089091AC08A091AD08B091AE0856
:1074C0008093330990933409A0933509B09336091A
:1074D0008091AF089091B008A091B108B091B20826
:1074E0008093370990933809A0933909B0933A09EA
:1074F00080E090E0A0E0B0E080934C0490934D04D5
:10750000A0934E04B0934F0488E50E94F02D882389
:1075100061F489E50E94F02D882339F48AE50E9400
:10752000F02D882311F481E001C080E080935004A5
:10753000882329F488E50E94F02D882321F080E03B
:1075400090E00E94352E80915004882329F489E52B
:107550000E94F02D882321F081E090E00E94352EDA
:1075600088E50E94F02D8823A1F00E943F302091F1
:10757000BF083091C0084091C1085091C2080E94D4
:1075800025E96093A3087093A4088093A5089093BD
:10759000A60889E50E94F02D8823A1F00E943F30C3
:1075A0002091C3083091C4084091C5085091C60885
:1075B0000E9425E96093A7087093A8088093A90802
:1075C0009093AA0880915004882329F48AE50E94A8
:1075D000F02D882321F082E090E00E94352E8AE58C
:1075E0000E94F02D8823D9F00E9434306115710576
:1075F00081059105A1F00E943F302091BB08309198
:10760000BC084091BD085091BE080E9425E96093D6
:10761000AB087093AC088093AD089093AE0883EAF2
:1076200098E067EA78E04BEA58E02FEA38E00E94F9
:10763000D35D8091BF089091C008A091C108B0911E
:10764000C2088093A3089093A408A093A508B093C0
:10765000A6088091C3089091C408A091C508B09174
:10766000C6088093A7089093A808A093A908B09390
:10767000AA088091C7089091C808A091C908B09144
:10768000CA088093AB089093AC08A093AD08B09360
:10769000AE0883EA98E067EA78E04BEA58E02FEA20
:1076A00038E00E94D35D80E00E94C5828091460947
:1076B00090914709A0914809B091490980934C04E1
:1076C00090934D04A0934E04B0934F048091A00872
:1076D0009091A10890931104809310040E9423E2DA
:1076E0006093110970931209809313099093140900
:1076F0000E94BE8286EC92E00E9445D40C940E5605
:1077000080914C0490914D04A0914E04B0914F048F
:107710008093460990934709A0934809B09349097B
:1077200080911004909111049093A1088093A00877
:1077300084E690E090931104809310040E9423E269
:10774000609311097093120980931309909314099F
:1077500081E00E94C5828091A3089091A408A09125
:10776000A508B091A60880932B0990932C09A093AB
:107770002D09B0932E098091A7089091A808A09197
:10778000A908B091AA0880932F0990933009A0937B
:107790003109B09332098091AB089091AC08A09167
:1077A000AD08B091AE088093330990933409A0934B
:1077B0003509B09336098091AF089091B008A09137
:1077C000B108B091B2088093370990933809A0931B
:1077D0003909B0933A0980E090E0A0E0B0E08093EE
:1077E0004C0490934D04A0934E04B0934F0488E54D
:1077F0000E94F02D882361F489E50E94F02D8823F2
:1078000039F48AE50E94F02D882311F481E001C04B
:1078100080E080935004882329F488E50E94F02DAD
:10782000882321F080E090E00E94352E8091500462
:10783000882329F489E50E94F02D882321F081E036
:1078400090E00E94352E88E50E94F02D8823D9F023
:107850000E9434306115710581059105A1F00E94E7
:107860003F302091B3083091B4084091B508509151
:10787000B6080E9425E96093A3087093A40880933A
:10788000A5089093A60889E50E94F02D8823D9F0D9
:107890000E9434306115710581059105A1F00E94A7
:1078A0003F302091B7083091B8084091B908509105
:1078B000BA080E9425E96093A7087093A8088093EE
:1078C000A9089093AA0880915004882329F48AE596
:1078D0000E94F02D882321F082E090E00E94352E56
:1078E0008AE50E94F02D8823D9F00E94343061157A
:1078F000710581059105A1F00E943F302091BB08E0
:107900003091BC084091BD085091BE080E9425E905
:107910006093AB087093AC088093AD089093AE0869
:1079200083EA98E067EA78E04BEA58E02FEA38E02B
:107930000E94D35D80E00E94C582809146099091AB
:107940004709A0914809B091490980934C0490934C
:107950004D04A0934E04B0934F048091A0089091E1
:10796000A10890931104809310040E9423E2609375
:1079700011097093120980931309909314090E94BE
:10798000BE820C940E5610923B090C940E5681E068
:1079900080933B090C940E5685E40E94F02D8823B9
:1079A00011F40E94D18353EAE52E58E0F52E43EB03
:1079B000C42E48E0D42E00E010E0F801EB53FB4F5A
:1079C00080810E94F02D882331F1033061F40E9400
:1079D0003F30F70160837183828393838FEA98E05D
:1079E0000E94B65D18C00E943F30F60120813181AF
:1079F000428153810E9425E9F7016083718382836C
:107A0000938383EA98E067EA78E04BEA58E02FEA4C
:107A100038E00E94D35D0F5F1F4F24E030E0E20E9C
:107A2000F31EC20ED31E0430110539F60C940E5607
:107A30008DE40E94F02D882311F40C94B2540E941E
:107A40003F300E946DEA6237710511F40C9493483F
:107A5000633771050CF0A7C06F31710509F442C49A
:107A6000603271050CF049C06631710509F4B8C285
:107A70006731710524F56131710509F469C262311C
:107A8000710574F477FF02C00C940E5662307105D4
:107A90000CF46DC16330710511F00C940E5613C2D5
:107AA0006431710509F466C2653171050CF092C24A
:107AB0006231710511F00C940E560C944F476A31E7
:107AC000710509F4C4C26B3171054CF4683171055C
:107AD00009F4A7C2693171050CF0B3C287C26C31D9
:107AE000710509F4D9C26C3171050CF4CFC26E3145
:107AF000710511F00C940E560AC36535710511F429
:107B00000C94B147663571051CF56135710511F4AA
:107B10000C942847623571057CF46A32710509F4CA
:107B200090C46035710511F40C941B4760327105E7
:107B300011F00C940E562FC36335710511F40C949B
:107B40004A476435710514F00C944F470C9446472E
:107B50006936710509F4F4C46A36710584F46C352C
:107B6000710511F40C94E7476836710509F4B3C444
:107B70006635710511F00C940E560C94CC476B369B
:107B8000710511F40C9415476B36710514F40C94BF
:107B9000E4466D36710509F410C66037710511F0C1
:107BA0000C940E56B8C4623E710511F40C948D4CC1
:107BB000633E71050CF063C0683C710511F40C94D0
:107BC0001C4A693C71053CF56837710511F40C9449
:107BD00088496937710584F46537710511F40C948F
:107BE0007D486737710509F4BEC06337710511F030
:107BF0000C940E560C946D486C38710509F48FC4C2
:107C00006E3B710509F4C4C76937710511F00C9416
:107C10000E560C948D496D3C710511F40C94224B59
:107C20006E3C71058CF46B3C710511F40C94E14AC7
:107C30006C3C710514F00C94004B693C710511F01B
:107C40000C940E560C94BE4A6A3D710511F40C94C6
:107C5000A14B6B3D71053CF46E3C710511F00C9429
:107C60000E560C94824B6C3D710511F40C94514CE2
:107C70006D3D710511F00C940E560C94624C31E080
:107C8000673F730711F40C94FF4E41E0683F74079F
:107C900084F551E06F32750711F40C94B44E81E015
:107CA000603378079CF491E06C32790711F40C94FE
:107CB000A34DE1E06D327E0711F40C94DC4D685168
:107CC000714011F00C940E560C94E84C21E0653F85
:107CD000720711F40C94F74E31E0663F730714F00D
:107CE0000C94FC4E6059714011F00C940E560C949B
:107CF000F44E52E06B35750711F40C94945482E005
:107D00006C3578079CF492E06935790711F40C948E
:107D10003252E2E06A357E0714F00C9489546855BB
:107D2000724011F00C940E560C94075023E063350A
:107D3000720711F40C94024F33E0643573073CF47E
:107D40006C55724011F00C940E560C94985453E0FC
:107D5000603A750709F48DC2675E734011F00C94A8
:107D60000E560C949B54E3EDF2E00C94994900916B
:107D70004A0910914B090E5F1F4F80E50E94F02DBC
:107D8000882329F4AA24BB246501EE240EC00E9496
:107D90003F300E9472EA5B016C01EE2461157105AF
:107DA0008105910511F0EE24E39483E50E94F02D06
:107DB000882311F4FF2414C00E943F3020E030E0FB
:107DC0004AE754E40E94DEEC0E9472EA5B016C0117
:107DD000FF24611571058105910511F0FF24F394CD
:107DE000C8016AE270E00E947812FC01009721F05D
:107DF000108202C00F5F1F4FF80180818032D1F3E3
:107E0000EE2041F4FF2031F4882321F0C8010E94C4
:107E100045D404C08CE498E00E9431D481E00E94F3
:107E200055980E94D1830E9423E2609311097093B8
:107E300012098093130990931409A114B104C10489
:107E4000D104F9F00E9423E27B018C01EA0CFB1CB7
:107E50000C1D1D1D0E9423E26E157F0580079107F2
:107E600010F00C9411560E945F98882311F00C9426
:107E700011560E94CF9080E00E9401370E948FD45B
:107E8000E9CF0E945D98882311F40C940E5607C028
:107E90000E94CF9080E00E9401370E948FD40E9400
:107EA0005F988823A9F380911006882331F08AE334
:107EB00098E00E9431D40C940E568DE298E00E9416
:107EC00031D40C940E5680914A0990914B09039637
:107ED0006AE270E00E947812FC01009709F01082BB
:107EE00080914A0990914B0903960E9445D481E004
:107EF0000E9455980E94D1830E9423E26093110949
:107F00007093120980931309909314090E945D984D
:107F1000882311F40C940E5607C00E94CF9080E085
:107F20000E9401370E948FD40E945F988823A9F392
:107F300080911006882331F08BE198E00E9431D4C3
:107F40000C940E568EE098E00E9431D40C940E569C
:107F50008DEF97E00E9431D45F988A989FB7F8948C
:107F6000809108018E7F809308019FBF12984798E7
:107F70000C940E56EDEEF7E0949108C08091C0008D
:107F800085FFFCCF9093C600319694919923B1F769
:107F90008091C00085FFFCCF8AE08093C6008EE010
:107FA00096E00E94E121EFEDF7E0949108C0809106
:107FB000C00085FFFCCF9093C60031969491992321
:107FC000B1F78091C00085FFFCCF8AE08093C600A6
:107FD0000C940E568EE096E00E9420190C940E56DA
:107FE0008EE096E00E9443150C940E5680914A094B
:107FF00090914B0904966AE270E00E947812FC01AD
:10800000009709F0108260914A0970914B096C5FEA
:108010007F4F8EE096E041E021E00E94D01D0C945D
:108020000E568EE096E00E9447150E9423E2609370
:10803000F3087093F4088093F5089093F6080C9475
:108040000E568EE096E00E944E150C940E568091CE
:108050001106882311F40C940E5683E50E94F02D2E
:10806000882311F40C940E560E943430AB01BC01ED
:1080700040939108509392088093930870939408CA
:108080008CED97E00E94CD710C940E568EE096E038
:108090000E9408170C940E5680914A0990914B0942
:1080A00004966AE270E00E9478128C01009709F150
:1080B000209140093091410980E690E0AC01249F75
:1080C000C001259F900D349F900D1124845B964F25
:1080D0006EE470E00E94781260E270E00E94781214
:1080E0009C012F5F3F4F30934B0920934A09F801C1
:1080F000108260914A0970914B096C5F7F4F8EE04E
:1081000096E040E021E00E94D01D0C940E56809134
:108110001106882311F40C940E568EE096E060E070
:108120000E947A1680914A0990914B0904966AE25E
:1081300070E00E9478128C01009709F120914009AB
:108140003091410980E690E0AC01249FC001259F59
:10815000900D349F900D1124845B964F6EE470E077
:108160000E94781260E270E00E9478129C012F5FFA
:108170003F4F30934B0920934A09F80110826091D8
:108180004A0970914B096C5F7F4F8EE096E00E9428
:1081900062170C940E5680911006882311F00E94ED
:1081A000D183E0904A09F0904B0924E030E0E20EE0
:1081B000F31EC7016AE270E00E9478128C01C701C9
:1081C00061E270E00E947812009721F07C0108942F
:1081D000E11CF11C0115110511F0F801108280E578
:1081E0000E94F02D182F80914A0990914B09E816B2
:1081F000F90608F410E080911106882311F40C941C
:108200000E5621E021278EE096E0B70141E00E9462
:10821000D01D83E50E94F02D8823B9F080914A0992
:1082200090914B098E159F0580F40E943430AB016C
:10823000BC014093910850939208809393087093E7
:1082400094088CED97E00E94CD718EE096E00E943C
:108250004715112311F00C940E560E9423E26093EF
:10826000F3087093F4088093F5089093F6080C9443
:108270000E5680914A0990914B0905966AE270E08A
:108280000E9478128C01009709F1209140093091E9
:10829000410980E690E0AC01249FC001259F900D2C
:1082A000349F900D1124845B964F6EE470E00E9421
:1082B000781260E270E00E9478129C012F5F3F4FBD
:1082C00030934B0920934A09F801108260914A09C2
:1082D00070914B096B5F7F4F8EE096E00E94DA2130
:1082E0000C940E560E9423E26093F7087093F808EE
:1082F0008093F9089093FA082091F3083091F408DC
:108300004091F5085091F608621B730B840B950B96
:1083100028EE33E040E050E00E9402EEF22EE32E21
:10832000D42EC52E2DB73EB7285030400FB6F89446
:108330003EBF0FBE2DBF0DB71EB70F5F1F4FCE0143
:108340008196EDB7FEB79283818380ED97E0F801C7
:10835000938382836F2D7E2D842F952F2CE330E025
:1083600040E050E00E9402EEF801358324836F2D37
:108370007E2D8D2D9C2D2CE330E040E050E00E94BE
:1083800002EEF801778366830E94B012E0E1F5E027
:1083900094912DB73EB7285F3F4F0FB6F8943EBF7C
:1083A0000FBE2DBF08C08091C00085FFFCCF909309
:1083B000C600319694919923B1F7FE01B19607C09A
:1083C0008091C00085FFFCCF31969093C6009081CC
:1083D0009923B1F78091C00085FFFCCF8AE080939C
:1083E000C600CE0181960E9445D480914A0B882315
:1083F00011F40C940E5610924A0B8091EE08082F3F
:1084000010E0000F111F0B561F4EF80160817181A3
:10841000882777FD8095982F0E94A0EA2091550427
:108420003091560440915704509158040E940CEC2E
:10843000181614F00C940E56F801118210820C9448
:108440000E5683E50E94F02D882311F40C940E56ED
:108450000E943F300E946DEA7B018C016B0180E538
:108460000E94F02D882369F0F7FC0BC0FFEFEF1698
:10847000F10409F034F40E943F300E946DEA8B0150
:1084800002C00DE010E0E9ECF4E0808191818017FA
:10849000910711F40C940E56329625E0E930F2075C
:1084A000A1F70430110529F4D092F008C092EF082A
:1084B00004C017FF02C00C940E56802F61E00E948A
:1084C000D4E3802F6C2D0E9487E4802FB6010E9498
:1084D000F6E20C940E5688E690E00E94483088231D
:1084E00011F00C940E5683E50E94F02D882379F04C
:1084F0000E943F3020910609022F10E0000F111F4B
:108500000B561F4E0E946DEAF801718360830E9432
:10851000FC8B0C940E560E94682B0C940E5683E52F
:108520000E94F02D882311F40C940E560E943F30C7
:108530000E946DEA70939A10609399100C940E56F5
:1085400089E690E00E944830882311F00C940E5682
:10855000EAECF7E0949108C08091C00085FFFCCF61
:108560009093C600319694919923B1F7E091060952
:10857000F0E0EE0FFF1FEE0FFF1FE156FF4E4081B0
:108580005181628173818CE096E021E030E00E94AD
:10859000052AE7ECF7E0949108C08091C00085FFC0
:1085A000FCCF9093C600319694919923B1F7E09156
:1085B0000609F0E0EE0FFF1FEB56FF4E6081718160
:1085C000882777FD8095982F0E94A0EAAB01BC0117
:1085D0008CE096E021E030E00E94052AE3ECF7E031
:1085E000949108C08091C00085FFFCCF9093C60095
:1085F000319694919923B1F74091A9105091AA1006
:108600006091AB107091AC108CE096E021E030E00E
:108610000E94052AE0ECF7E0949108C08091C00028
:1086200085FFFCCF9093C600319694919923B1F7C2
:108630006091991070919A10882777FD8095982FF6
:108640000E94A0EAAB01BC018CE096E021E030E0A2
:108650000E94052A05E9C02E00E1D02E1FE9E12E77
:1086600010E1F12E00E010E0EDEBF7E09490EBEB81
:10867000F7E0A490E8EBF7E0B490992DEDEBF7E08C
:1086800008C08091C00085FFFCCF9093C600319652
:1086900094919923B1F78CE096E0B8014AE050E05C
:1086A0000E9432299A2DEBEBF7E008C08091C000C0
:1086B00085FFFCCF9093C600319694919923B1F732
:1086C000F70140815181628173818CE096E021E065
:1086D00030E00E94052A9B2DE8EBF7E008C080916E
:1086E000C00085FFFCCF9093C600319694919923EA
:1086F000B1F7F601619171916F01882777FD80953F
:10870000982F0E94A0EAAB01BC018CE096E021E02A
:1087100030E00E94052A0F5F1F4F24E030E0E20E98
:10872000F31E0230110509F0A8CFE4EBF7E09491B5
:1087300008C08091C00085FFFCCF9093C6003196A1
:1087400094919923B1F7809106090E94418BBC0155
:108750008CE096E04AE050E00E943229EFEAF7E030
:10876000949108C08091C00085FFFCCF9093C60013
:10877000319694919923B1F78FEF9FEF0E94418B2F
:10878000BC018CE096E04AE050E00E943229ECEE19
:10879000F2E007C08091C00085FFFCCF3196909336
:1087A000C60090819923B1F78091C00085FFFCCF6E
:1087B0008AE08093C6000C943A568DE690E00E94C1
:1087C0004830882311F00C940E568FE997E00E94F0
:1087D00031D410924A0B83E50E94F02D882399F042
:1087E0000E943F3020910609022F10E0000F111F58
:1087F0000B561F4E0E946DEAF8017183608381E081
:108800008093470416C082E50E94F02D882389F0EA
:108810000E943F3020910609022F10E0000F111F27
:108820000B561F4E0E946DEAF8017183608310920F
:10883000470483E50E94F02D882351F00E943F30C9
:108840006093550470935604809357049093580492
:1088500082E40E94F02D882351F00E943F30609303
:10886000510470935204809353049093540486E40B
:108870000E94F02D882369F00E943F3060935904D4
:1088800070935A0480935B0490935C0481E080931E
:108890004A0B0E94FC8B0E9423E24B015C01209159
:1088A0000609022F10E010920509000F111FF801B0
:1088B000EB56FF4E60817181882777FD8095982F58
:1088C0000E94A0EA000F111F01561F4EF8012081DF
:1088D0003181428153810E940CEC18161CF481E016
:1088E000809305091092F108CC24CA94DC2C7601FF
:1088F000ECE9F7E05490E8E9F7E06490E4E9F7E0A8
:1089000074905AE0452E1BC1952DECE9F7E008C0A4
:108910008091C00085FFFCCF9093C6003196949162
:108920009923B1F7E0910609F0E0EE0FFF1FEE0F7B
:10893000FF1FE156FF4E40815181628173818CE0BF
:1089400096E021E030E00E94052A962DE8E9F7E064
:1089500008C08091C00085FFFCCF9093C60031967F
:1089600094919923B1F7609106098CE096E070E04C
:108970004AE050E00E943229972DE4E9F7E008C070
:108980008091C00085FFFCCF9093C60031969491F2
:108990009923B1F7F7FE03C0EDEEF2E028C00E9484
:1089A00023E2A70196012854344F4F4F5F4F261BF7
:1089B000370B480B590BCA01B90128EE33E040E0F0
:1089C00050E00E9402EE8CE096E0BA01A9012AE094
:1089D00030E00E94E3288091C00085FFFCCF0EC0EC
:1089E0008091C00085FFFCCF31969093C6009081A6
:1089F0009923B1F78091C00085FFFCCF4092C6005B
:108A00000E9423E24B015C010E94CF9080E00E9413
:108A100001370E948FD4FFEFCF16FFEFDF06FFEF85
:108A2000EF06FFEFFF0609F052C080910509E091C3
:108A30000609882331F1F0E08F01000F111F000FAC
:108A4000111F01561F4EEE0FFF1FEB56FF4E6081A8
:108A50007181882777FD8095982F0E94A0EA20E0F9
:108A600030E040E85FE30E9424E99B01AC01F8019B
:108A700060817181828193810E940CEC87FF58C0D4
:108A80005EC0F0E08F01000F111F000F111F015693
:108A90001F4EEE0FFF1FEB56FF4E6081718188273E
:108AA00077FD8095982F0E94A0EA20E030E040E812
:108AB0005FE30E9425E99B01AC01F80160817181AF
:108AC000828193810E94FEE9181694F538C0F7FC64
:108AD00036C0E0910609F0E08F01000F111F000F72
:108AE000111F01561F4EEE0FFF1FEB56FF4E608108
:108AF0007181882777FD8095982F0E94A0EA9B01BD
:108B0000AC01F80160817181828193810E9424E926
:108B10000E946DEA97FF07C09095809570956195CA
:108B20007F4F8F4F9F4F64307105810591053CF059
:108B30000E9423E2AC01CB01DA016C017D0180913E
:108B4000F108882311F00C941656FFEFCF16FFEFB3
:108B5000DF06FFEFEF06FFEFFF0669F0F7FE02C04A
:108B60000C9416560E9423E26C197D09685B7B40C9
:108B700010F00C9416560E9423E2681979098A09AC
:108B80009B09695E73408040904008F0BDCE3CCFA9
:108B900088E797E00E9431D483E50E94F02D882376
:108BA00061F00E943F300E946DEA70939A106093CA
:108BB000991081E0809347040FC082E50E94F02D58
:108BC000882351F00E943F300E946DEA70939A1002
:108BD00060939910109247040E9423E27B018C015C
:108BE0001092F108109205096091991070919A10F5
:108BF000882777FD8095982F0E94A0EA2091A910E0
:108C00003091AA104091AB105091AC100E940CEC26
:108C100018160CF083C081E0809305097FC00E9484
:108C200023E26E197F09800B910B695E73408040CF
:108C3000904008F46BC0E091EE08F0E0EE0FFF1FEB
:108C4000EE0FFF1FE156FF4E40815181628173811B
:108C50009B2DE5E7F7E008C08091C00085FFFCCFC1
:108C60009093C600319694919923B1F78CE096E0E9
:108C700022E030E00E94052A9C2DE1E7F7E008C0E1
:108C80008091C00085FFFCCF9093C60031969491EF
:108C90009923B1F76091EE088CE096E070E04AE02D
:108CA00050E00E9432299D2DEDE6F7E008C080914A
:108CB000C00085FFFCCF9093C60031969491992314
:108CC000B1F74091A9105091AA106091AB1070912A
:108CD000AC108CE096E021E030E00E94052AECEE3A
:108CE000F2E007C08091C00085FFFCCF31969093E1
:108CF000C60090819923B1F78091C00085FFFCCF19
:108D0000A092C6000E9423E27B018C010E94CF90BA
:108D100080E00E9401370E948FD40BC0E5E7F7E0A6
:108D2000B490E1E7F7E0C490EDE6F7E0D4906AE0B4
:108D3000A62E809105098823E1F08091F10888230F
:108D4000C1F46091991070919A10882777FD8095F1
:108D5000982F0E94A0EA2091A9103091AA1040916A
:108D6000AB105091AC100E940CEC18160CF457CFBD
:108D70001BC06091991070919A10882777FD80959B
:108D8000982F0E94A0EA2091A9103091AA1040913A
:108D9000AB105091AC100E94FEE988232CF4809116
:108DA0004704882309F43BCF80E697E00E9431D442
:108DB0000E9423E2609311097093120980931309B2
:108DC000909314090C940E5683E50E94F02D88238D
:108DD00021F10E943F3020E030E040E050E00E946E
:108DE000FEE988231CF460E070E011C00E943F306F
:108DF00020E030E04FE753E40E940CEC18161CF41E
:108E00006FEF70E004C00E943F300E946DEA7093E3
:108E1000F0086093EF080C940E568FEF90E090935B
:108E2000F0088093EF080C940E561092F008109200
:108E3000EF080C940E56269A2E9881E080934604F3
:108E400083E597E00E9431D40E948FD40C940E5693
:108E50000E94FD8B0E94D183129A479A0E94E08360
:108E60001092F0081092EF0868EE73E080E090E056
:108E70000E9431E2269A2E9A1092460486E497E0E8
:108E80000E9431D40E948FD40C940E5610929F08E9
:108E90000C940E5681E080939F080C940E5683E547
:108EA0000E94F02D8823A1F00E943F3020E030E0A6
:108EB0004AE754E40E94DEEC0E9472EA60934804A0
:108EC0007093490480934A0490934B040C940E567B
:108ED00088E50E94F02D882311F00C942F5689E527
:108EE0000E94F02D882311F00C942F568AE50E94E1
:108EF000F02D882311F00C942F5685E40E94F02D5C
:108F0000882311F00C942F560E94D183129A479A0D
:108F10000E94E0830C940E565F9A1092D70889E560
:108F20000E94F02D882319F08A9A1092D8088AE5B9
:108F30000E94F02D882351F09FB7F894809108018A
:108F40008160809308019FBF1092D90885E40E9438
:108F5000F02D882311F40C940E56129A479A0C9413
:108F60000E5683E50E94F02D882311F40C940E56C2
:108F70000E943F3020E030E04AE754E40E94DEECFB
:108F80000E9472EA6093150970931609809317097D
:108F9000909318090C940E5683E50E94F02D8823B7
:108FA00011F40C940E560E943F3020E030E04AE766
:108FB00054E40E94DEEC0E9472EA609319097093F7
:108FC0001A0980931B0990931C090C940E565EEEAF
:108FD000652E5AE0752E4EED242E4AE0342E3AE2EC
:108FE000432E3BE0532E88249924F401EB53FB4F8E
:108FF00080810E94F02D882309F45DC053E085161E
:1090000009F052C00E943F305B016C0120E030E06B
:1090100040EA51E40E94FEE988230CF03FC0F301CE
:109020006081718182819381A60195010E9405EA88
:109030007B018C016091220B7091230B8091240B9A
:109040009091250BA80197010E94DEEC6093220B02
:109050007093230B8093240B9093250BF101608177
:10906000718182819381A80197010E94DEECF10158
:109070006083718382839383F20160817181828135
:1090800093810E949EEAA80197010E94DEEC0E9453
:1090900072EAF2016083718382839383F301A08279
:1090A000B182C282D38207C00E943F30F301608345
:1090B0007183828393830894811C911C24E030E0A7
:1090C000620E731E220E331E420E531E34E08316B0
:1090D000910409F08ACF0C940E56E1E7F6E09491E2
:1090E00008C08091C00085FFFCCF9093C6003196E8
:1090F00094919923B1F70C940E5680914A0990915E
:109100004B0905966AE270E00E947812FC01009714
:1091100009F0108280914A0990914B0905960E94AE
:1091200045D40C940E56EEE6F6E0949108C080917A
:10913000C00085FFFCCF9093C6003196949199238F
:10914000B1F74091A3085091A4086091A5087091CF
:10915000A6088CE096E022E030E00E94052AEAE6CC
:10916000F6E0949108C08091C00085FFFCCF9093F9
:10917000C600319694919923B1F74091A708509178
:10918000A8086091A9087091AA088CE096E022E0F6
:1091900030E00E94052AE6E6F6E0949108C080914E
:1091A000C00085FFFCCF9093C6003196949199231F
:1091B000B1F74091AB085091AC086091AD08709147
:1091C000AE088CE096E022E030E00E94052AE2E65C
:1091D000F6E0949108C08091C00085FFFCCF909389
:1091E000C600319694919923B1F74091AF08509100
:1091F000B0086091B1087091B2088CE096E022E06E
:1092000030E00E94052AE7E5F6E0949108C08091DD
:10921000C00085FFFCCF9093C600319694919923AE
:10922000B1F780E00E949D830E94A0EA2091EE0A9F
:109230003091EF0A4091F00A5091F10A0E9405EA3C
:10924000AB01BC018CE096E022E030E00E94052AF0
:10925000E3E5F6E0949108C08091C00085FFFCCF63
:109260009093C600319694919923B1F781E00E94C2
:109270009D830E94A0EA2091F20A3091F30A409166
:10928000F40A5091F50A0E9405EAAB01BC018CE09A
:1092900096E022E030E00E94052AEFE4F6E09491A7
:1092A00008C08091C00085FFFCCF9093C600319626
:1092B00094919923B1F782E00E949D830E94A0EAD5
:1092C0002091F60A3091F70A4091F80A5091F90A74
:1092D0000E9405EAAB01BC018CE096E022E030E0A0
:1092E0000E94052AECEEF2E007C08091C00085FFE5
:1092F000FCCF31969093C60090819923B1F780916D
:10930000C00085FFFCCF8AE08093C6000C940E5607
:1093100080E00E94C5820C940E5681E00E94C582B6
:109320000C940E568091C00085FFFCCF319690932F
:10933000C60090819923B1F78091C00085FFFCCFD2
:109340008AE08093C600E7E4F6E0949108C080913B
:10935000C00085FFFCCF9093C6003196949199236D
:10936000B1F7659B03C0EFEEF2E00AC0E4EFF2E074
:1093700007C08091C00085FFFCCF31969093C60056
:1093800090819923B1F78091C00085FFFCCF8AE0DE
:109390008093C600EFE3F6E0949108C08091C0008E
:1093A00085FFFCCF9093C600319694919923B1F735
:1093B0008091030180FF03C0EFEEF2E00AC0E4EF0A
:1093C000F2E007C08091C00085FFFCCF31969093FA
:1093D000C60090819923B1F78091C00085FFFCCF32
:1093E0008AE08093C600E7E3F6E0949108C080919C
:1093F000C00085FFFCCF9093C600319694919923CD
:10940000B1F74B9B03C0EFEEF2E00AC0E4EFF2E0ED
:1094100007C08091C00085FFFCCF31969093C600B5
:1094200090819923B1F78091C00085FFFCCF8AE03D
:109430008093C6000C940E568091EE088093060926
:1094400084E50E94F02D882329F10E943F300E947C
:1094500072EA609306096230E8F0E0E1F5E0949189
:1094600008C08091C00085FFFCCF9093C600319664
:1094700094919923B1F7EEEFF2E007C08091C0001C
:1094800085FFFCCF31969093C60090819923B1F768
:109490000C940E5684E40E94F02D882311F40C9451
:1094A0000E560E943F3020E030E040E050E00E9445
:1094B000FEE9882319F41092A2085CC08091060985
:1094C000082F10E00E943F30000F111F000F111FE6
:1094D000085E1B4FF8016083718382839383E09061
:1094E0001804F090190400911A0410911B04C8018B
:1094F000B70120E030E040E050E00E94FEE9882320
:1095000051F40F2EF0E0EF2EF0E0FF2EF0E40F2FDD
:10951000F0E41F2FF02DE0921804F092190400934C
:109520001A0410931B04E0901C04F0901D04009199
:109530001E0410911F04C801B70120E030E040E094
:1095400050E00E94FEE9882351F40F2EF0E0EF2E48
:10955000F0E0FF2EF0E40F2FF0E41F2FF02DE0924B
:109560001C04F0921D0400931E0410931F0481E05C
:109570008093A2080E94032B0C940E5605EC14E075
:109580008EEFE82E8AE0F82EF80180810E94F02DFF
:10959000882349F00E943F300E9472EAF7016083FD
:1095A0007183828393830F5F1F4F24E030E0E20ECC
:1095B000F31E34E0093C130739F70E948B5D0C94CD
:1095C0000E5605EC14E0BEEDEB2EBAE0FB2EF801D2
:1095D00080810E94F02D882339F00E943F30F701EE
:1095E00060837183828393830F5F1F4F24E030E099
:1095F000E20EF31E34E0093C130749F70C940E56B3
:1096000083E50E94F02D882351F00E943F30609343
:10961000120B7093130B8093140B9093150B84E52E
:109620000E94F02D882311F40C940E560E943F30B6
:109630006093160B7093170B8093180B9093190B74
:109640000C940E5683E50E94F02D882351F00E9461
:109650003F3060930E0B70930F0B8093100B909321
:10966000110B84E50E94F02D882351F00E943F30B9
:109670006093260B7093270B8093280B9093290BF4
:1096800082E40E94F02D882361F00E943F300E9406
:1096900072EA6093DA0A7093DB0A8093DC0A909393
:1096A000DD0A88E50E94F02D882351F00E943F30AA
:1096B00060931A0B70931B0B80931C0B90931D0BE4
:1096C0008AE50E94F02D882351F00E943F3060937C
:1096D0001E0B70931F0B8093200B9093210B85E43E
:1096E0000E94F02D882311F40C940E560E943F30F6
:1096F0006093220B7093230B8093240B9093250B84
:109700000C940E5605EC14E0A3EBEA2EA8E0FA2E1A
:10971000F80180810E94F02D882339F00E943F30AB
:10972000F70160837183828393830F5F1F4F24E06F
:1097300030E0E20EF31E34E0083C130749F70C94C6
:109740000E568AED90E00E944830882311F00C9468
:109750000E5688E50E94F02D882389F08091060935
:10976000082F10E00E943F30000F111F000F111F43
:109770000252174FF801608371838283938389E5D6
:109780000E94F02D882389F080910609082F10E0AF
:109790000E943F30000F111F000F111F0A51174F79
:1097A000F8016083718382839383E0E1F5E0949113
:1097B00008C08091C00085FFFCCF9093C600319611
:1097C00094919923B1F7E7E2F6E0949108C0809173
:1097D000C00085FFFCCF9093C600319694919923E9
:1097E000B1F71092060940C08091C00085FFFCCF00
:1097F00011969093C6009C919923B1F7F0E0EE0F7B
:10980000FF1FEE0FFF1FE252F74F4081518162812F
:1098100073818CE096E022E030E00E94052AE5E1C9
:10982000F3E007C08091C00085FFFCCF3196909394
:10983000C60090819923B1F7E0910609F0E0EE0FA0
:10984000FF1FEE0FFF1FEA51F74F408151816281E8
:1098500073818CE096E022E030E00E94052A80913E
:1098600006098F5F80930609E0910609E23018F03F
:10987000ECEEF2E00AC0A7E1B3E0BDCF8091C000FA
:1098800085FFFCCF31969093C60090819923B1F764
:109890008091C00085FFFCCF8AE08093C6000C94C5
:1098A0000E5683E50E94F02D882311F40C940E5679
:1098B0000E943F300E946DEA70931104609310047F
:1098C0000C940E5683E50E94F02D882311F40C941D
:1098D0000E560E943F300E946DEA7B018C0184E5A8
:1098E0000E94F02D882399F08DED90E00E94483081
:1098F000882311F00C940E56E0910609F0E0EE0F6B
:10990000FF1FEC5EFB4FF182E0820C940E56F0924A
:109910001304E09212040C940E5680E50E94F02D80
:10992000882311F40C940E560E943F300E946DEA79
:109930007B0183E50E94F02D882319F40FEF1FEFC0
:1099400005C00E943F300E946DEA8B01C80101965C
:10995000039710F00C940E56E9ECF4E080819181AD
:109960008E159F0511F40C940E56329625E0E930C1
:10997000F207A1F7F7FE02C00C940E560E94D183A5
:10998000DE2C8E2D60E00E94D4E33FEF0F3F1307E3
:1099900031F00130110551F000E010E011C08E2DC2
:1099A0000E94B9E400E010E0892B51F401E010E0DE
:1099B00007C00E94CF9080E00E9401370E948FD4A0
:1099C0008D2D0E94B9E48017910799F70C940E56DB
:1099D00080E50E94F02D882321F4EE24EA94FE2CE9
:1099E00005C00E943F300E946DEA7B0183E50E9422
:1099F000F02D882309F44FC00E943F3043E0E41665
:109A0000F10488F48701000F111F0E0D1F1D045073
:109A1000174F0E946DEA9B01AC01C801B9010E9479
:109A20006D800C940E56E0E1F5E0949108C08091B1
:109A3000C00085FFFCCF9093C60031969491992386
:109A4000B1F7E9E1F3E007C08091C00085FFFCCFEA
:109A500031969093C60090819923B1F78CE096E0FF
:109A6000B7014AE050E00E943229E0E2F3E007C08B
:109A70008091C00085FFFCCF31969093C600908105
:109A80009923B1F78091C00085FFFCCF8AE08093D5
:109A9000C6000C940E56F7FE02C00C940E56EEE271
:109AA000F3E007C08091C00085FFFCCF3196909312
:109AB000C60090819923B1F7E1E3F3E007C08091FC
:109AC000C00085FFFCCF31969093C600908199230A
:109AD000B1F78CE096E0B7014AE050E00E943229ED
:109AE000E9E3F3E007C08091C00085FFFCCF319629
:109AF0009093C60090819923B1F7C701880F991FF1
:109B00008E0D9F1D8450974F0E941980BC018CE0E0
:109B100096E04AE050E00E943229ECEEF2E007C005
:109B20008091C00085FFFCCF31969093C600908154
:109B30009923B1F78091C00085FFFCCF8AE0809324
:109B4000C6000C940E5683E50E94F02D882321F464
:109B5000BEE6CB2ED12C05C00E943F300E946DEA9C
:109B60006B0180E50E94F02D882319F468EE73E004
:109B700004C00E943F300E946DEA7B010027F7FC81
:109B80000095102F1C141D048CF485E2B60120E012
:109B900030E040E050E00E94EFE5C801B7010E94CC
:109BA00031E285E20E947BE50C940E56C801B701B4
:109BB0000E9431E20C940E5680E50E94F02D88231D
:109BC00051F00E943F30609362047093630480936D
:109BD00064049093650489E40E94F02D882361F069
:109BE0000E943F300E94218C60936604709367044A
:109BF000809368049093690484E40E94F02D882384
:109C000061F00E943F300E942D8C60936A04709333
:109C10006B0480936C0490936D0483E40E94F02D98
:109C2000882351F00E943F3060936E0470936F045C
:109C300080937004909371040E941E8BEEE2F3E017
:109C400007C08091C00085FFFCCF31969093C6007D
:109C500090819923B1F7ECE3F3E007C08091C00055
:109C600085FFFCCF31969093C60090819923B1F780
:109C700040916204509163046091640470916504A2
:109C80008CE096E022E030E00E94052AE0E4F3E078
:109C900007C08091C00085FFFCCF31969093C6002D
:109CA00090819923B1F76091660470916704809167
:109CB0006804909169040E94278CAB01BC018CE080
:109CC00096E022E030E00E94052AE4E4F3E007C0D9
:109CD0008091C00085FFFCCF31969093C6009081A3
:109CE0009923B1F760916A0470916B0480916C04C0
:109CF00090916D040E94338CAB01BC018CE096E026
:109D000022E030E00E94052AE8E4F3E007C08091F9
:109D1000C00085FFFCCF31969093C60090819923B7
:109D2000B1F740916E0450916F046091700470918E
:109D300071048CE096E022E030E00E94052AECEE0F
:109D4000F2E007C08091C00085FFFCCF3196909370
:109D5000C60090819923B1F78091C00085FFFCCFA8
:109D60008AE08093C6005AC785E40E94F02D8823BC
:109D700019F4CC24DD2412C00E943F300E946DEA09
:109D80006B0177FF0BC00F2EF0E0EF2EF0E0FF2EFF
:109D9000FCE80F2FF2E41F2FF02D0AC00F2EF0E089
:109DA000EF2EF0E0FF2EF6E10F2FF3E41F2FF02D42
:109DB00083E50E94F02D882321F00E943F307B0133
:109DC0008C0183E40E94F02D882319F425E030E013
:109DD00005C00E943F300E946DEA9B01C801B70197
:109DE000A6010E9458931AC70E94D18317C70E94E8
:109DF000CC220E948E2412C70E94CC220FC70E9440
:109E00008E240CC78AE50E94F02D882309F4B8C07F
:109E10000E943F307B018C0120E030E040E751ECB4
:109E20000E940CEC88230CF44EC0C801B70120E05E
:109E300030E040EA50EC0E94FEE918160CF443C0F2
:109E4000D801C701B0588093DA089093DB08A0933B
:109E5000DC08B093DD08E0E1F5E0949108C0809162
:109E6000C00085FFFCCF9093C60031969491992352
:109E7000B1F7EBE1F6E0949108C08091C00085FF56
:109E8000FCCF9093C600319694919923B1F78091BD
:109E9000C00085FFFCCF8AE08093C600ECEEF2E0C4
:109EA00007C08091C00085FFFCCF31969093C6001B
:109EB00090819923B1F78091C00085FFFCCF8AE0A3
:109EC0008093C600ABC6E0E1F5E0949108C08091B4
:109ED000C00085FFFCCF9093C600319694919923E2
:109EE000B1F7E2E1F6E0949108C08091C00085FFEF
:109EF000FCCF9093C600319694919923B1F7EAE094
:109F0000F6E0949108C08091C00085FFFCCF90934B
:109F1000C600319694919923B1F78CE096E061EFF9
:109F20007FEF4AE050E00E943229E2E0F6E09491AF
:109F300008C08091C00085FFFCCF9093C600319689
:109F400094919923B1F78CE096E06BEF7FEF4AE0B4
:109F500050E00E943229ECEEF2E007C08091C00090
:109F600085FFFCCF31969093C60090819923B1F77D
:109F70008091C00085FFFCCF8AE08093C6004EC66A
:109F8000E0E1F5E0949108C08091C00085FFFCCF2E
:109F90009093C600319694919923B1F7E6EFF5E0DE
:109FA000949108C08091C00085FFFCCF9093C600BB
:109FB000319694919923B1F78091C00085FFFCCF31
:109FC0008AE08093C6004091DA085091DB086091E6
:109FD000DC087091DD0870588CE096E022E030E0FB
:109FE0000E94052AECEEF2E007C08091C00085FFD8
:109FF000FCCF31969093C60090819923B1F7809160
:10A00000C00085FFFCCF8AE08093C60007C6A09001
:10A01000A308B090A408C090A508D090A608A98A6B
:10A02000BA8ACB8ADC8AE090A708F090A808009151
:10A03000A9081091AA08ED8AFE8A0F8B188F20912B
:10A04000AB083091AC084091AD085091AE08298F13
:10A050003A8F4B8F5C8F8091AF089091B008A091A0
:10A06000B108B091B2088D8F9E8FAF8FB8A3A9822F
:10A07000BA82CB82DC82ED82FE820F831887298729
:10A080003A874B875C878D879E87AF87B88B85E43F
:10A090000E94F02D882369F0ED8CFE8C0F8D18A1A5
:10A0A0000E943F309B01AC01C801B7010E9425E925
:10A0B0000AC06D8D7E8D8F8D98A120E030E040E943
:10A0C00050E40E9424E96D8F7E8F8F8F98A360915A
:10A0D0004C0470914D0480914E0490914F0420E007
:10A0E00030E040E752E40E9405EA7B018C01CE019A
:10A0F0004196BE016B5E7F4FAE01475E5F4F9E0192
:10A10000235E3F4FAEEECA2EA8E0DA2E0E94D9623F
:10A110008AE50E94F02D882359F0E98CFA8C0B8D8A
:10A120001C8D0E943F309B01AC01C801B70108C0E3
:10A13000698D7A8D8B8D9C8D20E030E040E251E47A
:10A140000E9425E9698F7A8F8B8F9C8F60914C04D8
:10A1500070914D0480914E0490914F0420E030E0C6
:10A1600040E752E40E9405EA7B018C01CE01419652
:10A17000BE016B5E7F4FAE01475E5F4F9E01235E67
:10A180003F4FFEEECF2EF8E0DF2E0E94D96288E529
:10A190000E94F02D882389F0E988FA880B891C89B0
:10A1A0000E943F309B01AC01C801B7010E9425E924
:10A1B000698B7A8B8B8B9C8B08C080E090E0AFE240
:10A1C000B3E4898B9A8BAB8BBC8B89E50E94F02D15
:10A1D000882339F00E943F306D8B7E8B8F8B988F58
:10A1E00008C080E090E0A2E5B3E48D8B9E8BAF8B3E
:10A1F000B88F60914C0470914D0480914E04909101
:10A200004F0420E030E040E752E40E9405EA7B0181
:10A210008C01CE014196BE016B5E7F4FAE01475E61
:10A220005F4F9E01235E3F4FEEEECE2EE8E0DE2E26
:10A230000E94D9628CE40E94F02D882369F0ED8C95
:10A24000FE8C0F8D18A10E943F309B01AC01C8010C
:10A25000B7010E9425E90AC06D8D7E8D8F8D98A172
:10A2600020E030E048EC52E40E9424E96D8F7E8FBC
:10A270008F8F98A360914C0470914D0480914E048F
:10A2800090914F0420E030E040E752E40E9405EA5C
:10A290007B018C01CE014196BE016B5E7F4FAE010A
:10A2A000475E5F4F9E01235E3F4FBEEECB2EB8E070
:10A2B000DB2E0E94D9620E94D183129A479A64E6EB
:10A2C00070E080E090E00E9431E285EE95E00E942F
:10A2D0003FD410E019C01F5F0E94CF9081E00E9420
:10A2E00001370E948FD4112379F4389A409A63E0A1
:10A2F00070E080E090E00E9431E2409863E070E01E
:10A3000080E090E00E9431E20E945F98882319F378
:10A310008CE40E94F02D882369F0ED8CFE8C0F8D6B
:10A3200018A10E943F309B01AC01C801B7010E94F7
:10A3300024E90AC06D8D7E8D8F8D98A120E030E0DC
:10A3400048EC52E40E9425E96D8F7E8F8F8F98A391
:10A350008D8D9E8DAF8DB8A18093AF089093B0087E
:10A36000A093B108B093B2088FEA98E00E94B65D5E
:10A37000A9E14A2E512C4C0E5D1EFDE16F2E712C71
:10A380006C0E7D1E60914C0470914D0480914E04C2
:10A3900090914F0420E030E040E752E40E9405EA4B
:10A3A0007B018C01CE014196BE016B5E7F4FA20105
:10A3B0009301EEEECE2EE8E0DE2E0E94D96215E08B
:10A3C000812E912C8C0E9D1E60914C0470914D0439
:10A3D00080914E0490914F0420E030E040E752E439
:10A3E0000E9405EA7B018C015E010894A11CB11C4E
:10A3F000C501B401A20193010E94D962B9E04B2EBC
:10A40000512C4C0E5D1E60914C0470914D04809156
:10A410004E0490914F0420E030E040E752E40E9467
:10A4200005EA7B018C01C501B401A20193010E94E0
:10A43000D96260914C0470914D0480914E049091CA
:10A440004F0420E030E040E752E40E9405EA7B013F
:10A450008C01C501B401A2019E01235F3F4F0E9400
:10A46000D962DCC38091F208882309F04CC2A09025
:10A47000A308B090A408C090A508D090A608A9820F
:10A48000BA82CB82DC82E090A708F090A808009105
:10A49000A9081091AA08ED82FE820F8318872091E7
:10A4A000AB083091AC084091AD085091AE082987B7
:10A4B0003A874B875C878091AF089091B008A09154
:10A4C000B108B091B2088D879E87AF87B88BA98AF3
:10A4D000BA8ACB8ADC8AED8AFE8A0F8B188F298F85
:10A4E0003A8F4B8F5C8F8D8F9E8FAF8FB8A385E493
:10A4F0000E94F02D882369F0ED84FE840F85188971
:10A500000E943F309B01AC01C801B7010E9425E9C0
:10A510000AC06D857E858F85988920E030E040E90E
:10A5200050E40E9424E96D877E878F87988B609125
:10A530004C0470914D0480914E0490914F0420E0A2
:10A5400030E040E752E40E9405EA7B018C01CE0135
:10A550000196BE016B5F7F4FAE01475F5F4F9E016B
:10A56000235F3F4FAEEECA2EA8E0DA2E0E94D962DA
:10A570008AE50E94F02D882359F0E984FA840B853E
:10A580001C850E943F309B01AC01C801B70108C087
:10A5900069857A858B859C8520E030E040E251E436
:10A5A0000E9425E969877A878B879C8760914C0494
:10A5B00070914D0480914E0490914F0420E030E062
:10A5C00040E752E40E9405EA7B018C01CE0101962E
:10A5D000BE016B5F7F4FAE01475F5F4F9E01235F00
:10A5E0003F4FFEEECF2EF8E0DF2E0E94D96288E5C5
:10A5F0000E94F02D882389F0E980FA800B811C816C
:10A600000E943F309B01AC01C801B7010E9425E9BF
:10A6100069837A838B839C8308C080E090E0AFE2FB
:10A62000B3E489839A83AB83BC8389E50E94F02DD0
:10A63000882339F00E943F306D837E838F83988713
:10A6400008C080E090E0A2E5B3E48D839E83AF83F1
:10A65000B88760914C0470914D0480914E049091A4
:10A660004F0420E030E040E752E40E9405EA7B011D
:10A670008C01CE010196BE016B5F7F4FAE01475F3B
:10A680005F4F9E01235F3F4FEEEECE2EE8E0DE2EC1
:10A690000E94D9628CE40E94F02D882369F0ED8439
:10A6A000FE840F8518890E943F309B01AC01C801D0
:10A6B000B7010E9425E90AC06D857E858F8598893E
:10A6C00020E030E048EC52E40E9424E96D877E8768
:10A6D0008F87988B85E0882E912C8C0E9D1E09E02B
:10A6E000602E712C6C0E7D1E1DE0412E512C4C0EE7
:10A6F0005D1E60914C0470914D0480914E049091C8
:10A700004F0420E030E040EF52E40E9405EA7B0174
:10A710008C015E010894A11CB11CC501B401A30108
:10A720009201BEEECB2EB8E0DB2E0E94D9620E94D1
:10A73000D183129A479A8CE493E00E9464360E9477
:10A74000CF9081E00E9401370E948FD48FE593E083
:10A750000E9464368091EE088F5F8093EE086D85CD
:10A760007E858F85988920E030E042E053E40E94A6
:10A7700025E96D877E878F87988BC501B401A3017A
:10A7800092010F2EF0E0EF2EF0E0FF2EF0E20F2FFF
:10A79000F1E41F2FF02D0E94D9628CE40E94F02D6D
:10A7A000882369F0ED84FE840F8518890E943F306C
:10A7B0009B01AC01C801B7010E9424E90AC06D8564
:10A7C0007E858F85988920E030E048EC52E40E9435
:10A7D00025E96D877E878F87988B8D8D9E8DAF8DB8
:10A7E000B8A18093AF089093B008A093B108B0933C
:10A7F000B2088FEA98E00E94B65D8091AF08909110
:10A80000B008A091B108B091B2088D879E87AF873C
:10A81000B88BA9E04A2E512C4C0E5D1EFDE06F2E28
:10A82000712C6C0E7D1E60914C0470914D048091D2
:10A830004E0490914F0420E030E040EF51E40E943C
:10A8400005EA7B018C01CE010196BE016B5F7F4F53
:10A85000A2019301EEEECE2EE8E0DE2E0E94D96238
:10A8600091E1A92EB12CAC0EBD1E85E1882E912C54
:10A870008C0E9D1E60914C0470914D0480914E048D
:10A8800090914F0420E030E040E752E40E9405EA56
:10A890007B018C01C501B401A20193010E94D96220
:10A8A00009E1402E512C4C0E5D1E60914C047091BC
:10A8B0004D0480914E0490914F0420E030E040EF31
:10A8C00052E40E9405EA7B018C01C501B401A2019A
:10A8D00093010E94D96260914C0470914D04809163
:10A8E0004E0490914F0420E030E040EF52E40E948B
:10A8F00005EA7B018C01C501B401A2019E01235E22
:10A900003F4F0E94D9628091F2088F5F8093F208D6
:10A9100085C11092F2081092CD0A1092CC0A82E6FC
:10A9200093E00E9464367AC181E08093CE0A76C1BA
:10A930001092CE0A73C11092FB080E945A9880911F
:10A940000B0990910C09A0910D09B0910E0980930B
:10A95000070990930809A0930909B0930A090E9476
:10A96000C62D5CC184E50E94F02D882309F40BC13B
:10A970000E943F300E9472EA262F609306096230DF
:10A98000B8F1E0E1F5E0949108C08091C00085FF46
:10A99000FCCF9093C600319694919923B1F7E3E7E9
:10A9A000F3E007C08091C00085FFFCCF3196909303
:10A9B000C60090819923B1F78CE096E0622F40E0C9
:10A9C00050E00E94EE28E5E7F3E007C08091C00068
:10A9D00085FFFCCF31969093C60090819923B1F703
:10A9E0008091C00085FFFCCF8AE08093C60016C12D
:10A9F00086E40E94F02D882311F4EE241EC00E94EC
:10AA00003F307B018C0160933C0970933D0980933A
:10AA10003E0990933F0920E030E040E050E00E9482
:10AA20000CEC181644F4E0924C04F0924D040093A0
:10AA30004E0410934F04EE24E39490910609809104
:10AA4000EE08981709F473C0ABE2B9E0E3EAF8E066
:10AA500080E101900D928150E1F72091EE08C22E25
:10AA6000DD24CC0CDD1CCC0CDD1CF601E252F74FD2
:10AA70006091A3087091A4088091A5089091A60800
:10AA800020813181428153810E9424E9F09006099E
:10AA90000F2D10E0000F111F000F111FF801E252DF
:10AAA000F74F20813181428153810E9425E96093D3
:10AAB000A3087093A4088093A5089093A60886EE37
:10AAC00098E0C80ED91E6091A7087091A8088091DF
:10AAD000A9089091AA08F601208131814281538111
:10AAE0000E9424E90A51174FF801208131814281E7
:10AAF00053810E9425E96093A7087093A80880936A
:10AB0000A9089093AA08F092EE0883EA98E067EA11
:10AB100078E04BEA58E02FEA38E00E94D35DEE205F
:10AB200031F08091FB08882311F40E94AE2CE0E103
:10AB3000F5E0949108C08091C00085FFFCCF909310
:10AB4000C600319694919923B1F7E6E8F3E007C087
:10AB50008091C00085FFFCCF31969093C600908114
:10AB60009923B1F76091EE088CE096E070E04AE03E
:10AB700050E00E9432298091C00085FFFCCF8AE01E
:10AB80008093C6004BC0E0E1F5E0949108C080914D
:10AB9000C00085FFFCCF9093C60031969491992315
:10ABA000B1F7E2EDF5E0949108C08091C00085FF17
:10ABB000FCCF9093C600319694919923B1F72091E0
:10ABC00040093091410980E690E0289FF001299FDB
:10ABD000F00D389FF00D1124E45BF64F07C0809113
:10ABE000C00085FFFCCF31969093C60090819923D9
:10ABF000B1F7E0EDF5E0949108C08091C00085FFC9
:10AC0000FCCF9093C600319694919923B1F780912F
:10AC1000C00085FFFCCF8AE08093C6000E94BD2B58
:10AC200029C080E00E9455980C94533F87E897E034
:10AC30000E9431D40E9423E26093F3087093F408D9
:10AC40008093F5089093F6080E9423E2609311091F
:10AC5000709312098093130990931409DFCF0E9417
:10AC6000D18388E50E94F02D882311F00C948C4745
:10AC70000C948F47EE960FB6F894DEBF0FBECDBF93
:10AC8000CF91DF911F910F91FF90EF90DF90CF90C8
:10AC9000BF90AF909F908F907F906F905F904F90FC
:10ACA0003F902F900895CF93DF9380910F0990915B
:10ACB0001009039714F40E948B318EE096E060E057
:10ACC0000E94001A80910F0990911009892B09F4B4
:10ACD0006AC080910E06882309F44DC02091400976
:10ACE0003091410980E690E0289FE001299FD00D36
:10ACF000389FD00D1124C45BD64FCE0169E07AE0B5
:10AD00000E942A12892BE1F48EE096E0BE010E9497
:10AD1000931680910F06882371F5E6E0FAE094918E
:10AD200008C08091C00085FFFCCF9093C60031968B
:10AD300094919923B1F78091C00085FFFCCF17C093
:10AD40008EE096E060E00E947A16E4EFF9E09491DC
:10AD500008C08091C00085FFFCCF9093C60031965B
:10AD600094919923B1F78091C00085FFFCCF8AE0D0
:10AD70008093C60002C00E94C43780910F09909151
:10AD8000100901979093100980930F098091400951
:10AD900090914109019664E070E00E94EFED90937C
:10ADA0004109809340090E94CF9080E00E940137C2
:10ADB0000E94748A0E948FD4DF91CF910895809170
:10ADC0001006882341F04A9906C088E993E00E9462
:10ADD00064360C94DD360895F2DF269A2E988CE0C6
:10ADE00096E040E950ED63E070E00E94EB27E8EE6A
:10ADF000FAE0949108C08091C00085FFFCCF909349
:10AE0000C600319694919923B1F78091C00085FFD7
:10AE1000FCCF8AE08093C60040E155E0FA019491AE
:10AE200008C08091C00085FFFCCF9093C60031968A
:10AE300094919923B1F784B7282F80FF15C0E0EED5
:10AE4000FAE0949108C08091C00085FFFCCF9093F8
:10AE5000C600319694919923B1F78091C00085FF87
:10AE6000FCCF8AE08093C60021FF15C0E0EDFAE038
:10AE7000949108C08091C00085FFFCCF9093C600DC
:10AE8000319694919923B1F78091C00085FFFCCF52
:10AE90008AE08093C60022FF15C0EFEBFAE09491A0
:10AEA00008C08091C00085FFFCCF9093C60031960A
:10AEB00094919923B1F78091C00085FFFCCF8AE07F
:10AEC0008093C60023FF15C0EFEAFAE0949108C012
:10AED0008091C00085FFFCCF9093C600319694917D
:10AEE0009923B1F78091C00085FFFCCF8AE0809361
:10AEF000C60025FF15C0EFE9FAE0949108C08091E3
:10AF0000C00085FFFCCF9093C600319694919923A1
:10AF1000B1F78091C00085FFFCCF8AE08093C60026
:10AF200014BEE8E9FAE0949108C08091C00085FF62
:10AF3000FCCF9093C600319694919923B1F7E2E942
:10AF4000FAE0949108C08091C00085FFFCCF9093F7
:10AF5000C600319694919923B1F78091C00085FF86
:10AF6000FCCF8AE08093C600FA019491E0E1F5E01D
:10AF700008C08091C00085FFFCCF9093C600319639
:10AF800094919923B1F7E2E8FAE0949108C0809196
:10AF9000C00085FFFCCF9093C60031969491992311
:10AFA000B1F7EDE6FAE0949108C08091C00085FF0A
:10AFB000FCCF9093C600319694919923B1F7E1E6C6
:10AFC000FAE0949108C08091C00085FFFCCF909377
:10AFD000C600319694919923B1F7EAE4FAE094918E
:10AFE00008C08091C00085FFFCCF9093C6003196C9
:10AFF00094919923B1F78091C00085FFFCCF8AE03E
:10B000008093C600EFE3FAE0949108C08091C000FD
:10B0100085FFFCCF9093C600319694919923B1F7A8
:10B02000E3E3FAE0949108C08091C00085FFFCCF73
:10B030009093C600319694919923B1F78091C00006
:10B0400085FFFCCF8AE08093C600FA019491E0E18D
:10B05000F5E008C08091C00085FFFCCF9093C6004A
:10B06000319694919923B1F7E4E2FAE0949108C003
:10B070008091C00085FFFCCF9093C60031969491DB
:10B080009923B1F70E94C97ABC018CE096E04AE0AE
:10B0900050E00E943229EDE0FAE0949108C08091DE
:10B0A000C00085FFFCCF9093C60031969491992300
:10B0B000B1F78CE096E068E672E04AE050E00E946A
:10B0C00032298091C00085FFFCCF8AE08093C600C2
:10B0D00010924209109243091092440910924509B6
:10B0E0000E94CC220E948E240E948E8FA5D70E949F
:10B0F000CE820E94B5350E9462D580E197E220E9B8
:10B1000031E0F9013197F1F70197D9F708952F92BE
:10B110003F924F925F926F927F928F929F92AF92E7
:10B12000BF92CF92DF92EF92FF920F931F93DF9324
:10B13000CF93CDB7DEB7CD56D0400FB6F894DEBF73
:10B140000FBECDBF6F969FAF8EAF6F97A1967FAFAB
:10B150006EAFA1972A01A2962FAFA297A3960FAF29
:10B16000A397A496EFAEA497A896ACAEBDAECEAE14
:10B17000DFAEA897E22EFF24EE0CFF1CEE0CFF1CA6
:10B18000FC01EE0DFF1D20813181428153816D96BE
:10B190002CAF3DAF4EAF5FAF6D97A2014E0D5F1D5F
:10B1A00069965FAF4EAF6997DA016D907D908D9093
:10B1B0009C906D966CAD7DAD8EAD9FAD6D97A401ED
:10B1C00093010E9425E969AF7AAF8BAF9CAF10E085
:10B1D000000F111F000F111F6F96EEADFFAD6F979F
:10B1E000E00FF11F208131814281538167962CAF9E
:10B1F0003DAF4EAF5FAF6797A201400F511F6396FF
:10B200005FAF4EAF6397DA01AD90BD90CD90DC900B
:10B2100067966CAD7DAD8EAD9FAD6797A60195012C
:10B220000E9425E96DAB7EAB8FAB98AFA496BFAD06
:10B23000A497EB2FF0E0EE0FFF1FEE0FFF1F6F96AE
:10B24000AEADBFAD6F97AE0FBF1F2D913D914D912C
:10B250005C9161962CAF3DAF4EAF5FAF6197A19609
:10B260004EAD5FADA197E40FF51F608171818281C2
:10B27000938161962CAD3DAD4EAD5FAD61970E945F
:10B2800024E969AB7AAB8BAB9CABA196AEADBFADFD
:10B29000A1971C966D917D918D919C911F972D96F4
:10B2A0006CAF7DAF8EAF9FAF2D976F96AEADBFAD3C
:10B2B0006F971C962D913D914D915C911F9729960A
:10B2C0002CAF3DAF4EAF5FAF2997A401930150580B
:10B2D0002DA73EA74FA758ABB601A501705849A7A7
:10B2E0005AA76BA77CA7A1966EAD7FADA197E60E7E
:10B2F000F71ED7018D919D910D90BC91A02D2596A3
:10B300008CAF9DAFAEAFBFAF2597BC01CD0129ADCE
:10B310003AAD4BAD5CAD0E9424E91B012C01A19616
:10B32000EEADFFADA1970E0F1F1FD8012D913D91DE
:10B330004D915C9121962CAF3DAF4EAF5FAF219701
:10B34000CA01B9012DA93EA94FA958AD0E9424E90F
:10B350005B016C016DA57EA58FA598A9A60195013D
:10B360000E94DEEC7B018C0169A57AA58BA59CA5CA
:10B37000A20191010E94DEEC9B01AC01C801B70162
:10B380000E9424E93B014C016DA57EA58FA598A9DB
:10B39000A20191010E94DEEC7B018C0169A57AA5D6
:10B3A0008BA59CA5A60195010E94DEEC9B01AC013A
:10B3B000C801B7010E9425E99B01AC01C401B3019A
:10B3C0000E9498E95B016C0120E030E040E050E031
:10B3D0000E94FEE9882354F4C601B5012BED3FE03D
:10B3E00049EC50E40E9425E95B016C01C957DF4F2D
:10B3F0008881C758D040882351F0C601B5012BED94
:10B400003FE049EC50E40E9424E95B016C016D9639
:10B410006CAD7DAD8EAD9FAD6D9725962CAD3DADE0
:10B420004EAD5FAD25970E94FEE9882321F5679612
:10B430006CAD7DAD8EAD9FAD679721962CAD3DADCA
:10B440004EAD5FAD21970E94FEE98823A1F4C601AD
:10B45000B50120E030E040E050E00E94FEE98823A2
:10B4600051F4C601B5012BED3FE049EC50E40E94D8
:10B4700025E95B016C01C601B501CD57DF4F28817D
:10B4800039814A815B81C358D0400E94DEEC29A9F2
:10B490003AA94BA95CA95F770E9419EC7B018C014A
:10B4A0002FE632E143E85AE30E94FEE987FDF4C14A
:10B4B000C801B7010E94DBEA0E9472EA78A76FA375
:10B4C000672B21F4E1E0F0E0F8A7EFA32FA138A566
:10B4D000B90180E090E00E949EEA7B018C01C601E8
:10B4E000B501A80197010E9405EA6BA37CA38DA377
:10B4F0009EA369A97AA98BA99CA9A80197010E947A
:10B5000005EA6F8F78A389A39AA32D966CAD7DADC4
:10B510008EAD9FAD2D9729962CAD3DAD4EAD5FAD57
:10B5200029970E9424E9A80197010E9405EA6B8FE0
:10B530007C8F8D8F9E8F6BA17CA18DA19EA120E021
:10B5400030E040E05FEB0E94DEEC2BA13CA14DA17E
:10B550005EA10E94DEEC20E030E040E85FE30E9464
:10B5600025E96F8B788F898F9A8FA4963FADA4972A
:10B57000E32FF0E0EE0FFF1FEE0FFF1F9E012F5F86
:10B580003F4FE20FF31F61964CAD5DAD6EAD7FADE9
:10B59000619740835183628373836F96AEADBFAD75
:10B5A0006F971C964D915D916D917C911F974D8782
:10B5B0005E876F87788B41E050E05A8B498B662419
:10B5C000A2967FADA297672F70E0660F771F660F78
:10B5D000771FC901860F971FAA969FAF8EAFAA97B4
:10B5E000A396BFADA397AB2FB0E0AA0FBB1FAA0FC6
:10B5F000BB1F21E030E02C0F3D1F2A0F3B1FAC96F4
:10B600003FAF2EAFAC97AE96FFAFEEAFAE9719C17E
:10B6100038E136150CF446C06DA57EA58FA598A916
:10B620002BA13CA14DA15EA10E94DEEC7B018C010F
:10B6300069A57AA58BA59CA52F89388D498D5A8D32
:10B640000E94DEEC9B01AC01C801B7010E9425E914
:10B650007B018C016DA57EA58FA598A92F89388DBA
:10B66000498D5A8D0E94DEEC5B016C0169A57AA5BB
:10B670008BA59CA52BA13CA14DA15EA10E94DEEC57
:10B680009B01AC01C601B5010E9424E96DA77EA70C
:10B690008FA798AB6394C701D80189A79AA7ABA7D6
:10B6A000BCA765C049895A89BA0180E090E00E9430
:10B6B0009EEA2BA13CA14DA15EA10E94DEEC7B0184
:10B6C0008C01C8010E9402EA6B8B7C8B8D8B9E8B58
:10B6D000B701C8010E9441ED3B014C016996AEAD36
:10B6E000BFAD6997ED90FD900D911C9117FB1095E2
:10B6F00017F910956396EEADFFAD6397208031800A
:10B7000042805380C801B7012B893C894D895E89ED
:10B710000E94DEEC5B016C01C201B101A401930146
:10B720000E94DEEC9B01AC01C601B5010E9425E937
:10B730006DA77EA78FA798ABC801B701A40193019D
:10B740000E94DEEC7B018C01C201B1012B893C8996
:10B750004D895E890E94DEEC9B01AC01C801B701F6
:10B760000E9424E969A77AA78BA79CA7662469ADE4
:10B770007AAD8BAD9CAD2DA53EA54FA558A90E94D5
:10B7800025E9AA96AEADBFADAA976D937D938D9333
:10B790009C9313976DA97EA98FA998AD29A53AA569
:10B7A0004BA55CA50E9425E9AC96EEADFFADAC972C
:10B7B0006083718382839383AE96AEADBFADAE9747
:10B7C0006D917D918D919C912F8D38A149A15AA1A8
:10B7D0000E9425E9AE96EEADFFADAE976083718312
:10B7E000828393836D857E858F8598892B8D3C8D93
:10B7F0004D8D5E8D0E9425E96D877E878F87988BA2
:10B80000CE0101960E94072ACE010196BE016B5F10
:10B810007F4FAE01475F5F4F9E01235F3F4FA8966A
:10B82000ECACFDAC0EAD1FADA897F8E8CF2ED12C37
:10B83000CC0EDD1EBED629893A892F5F3F4F3A8B49
:10B84000298B49895A896FA178A54617570708F4AB
:10B85000DFCEA1964EAD5FADA197485F5F4FA19639
:10B860002EAD3FADA197245F3F4FA1968EAD9FAD0A
:10B87000A197DC011496A196BFAFAEAFA197BD0111
:10B88000A896ECACFDAC0EAD1FADA897E8E8CE2EA7
:10B89000D12CCC0EDD1E8DD6C359DF4F0FB6F894D8
:10B8A000DEBF0FBECDBFCF91DF911F910F91FF90F3
:10B8B000EF90DF90CF90BF90AF909F908F907F9050
:10B8C0006F905F904F903F902F9008953F924F92CE
:10B8D0005F926F927F928F929F92AF92BF92CF9220
:10B8E000DF92EF92FF920F931F93CF93DF9380919C
:10B8F0004A0B882309F4F6C08090550490905604B2
:10B90000A0905704B09058046091951070919610D3
:10B91000882777FD8095982F0E94A0EA20E030E0EC
:10B9200040E050E40E9425E9A50194010E94FEE94F
:10B9300087FDD8C03090B70D0F2EF0E04F2EF0E00D
:10B940005F2EF0E06F2EF0E07F2EF02DCDE4D0E002
:10B9500058C0232D30E02C9FF0012D9FF00D3C9F0F
:10B96000F00D1124E25BF44F80819181A281B381BB
:10B970000097A105B10581F484819581A681B781E5
:10B980000097A105B10541F480859185A285B38515
:10B990000097A105B10591F12C9F60012D9FD00C5E
:10B9A0003C9FD00C11248EE49BE0C80ED91EF601FA
:10B9B00064857585868597850E94A0EA7B018C0148
:10B9C000F60160897189828993890E949EEA9B01B0
:10B9D000AC01C801B7010E9405EAF60122A133A11A
:10B9E00044A155A10E94DEEC7B018C01A3019201D0
:10B9F0000E940CEC181614F4270138013394F7E078
:10BA00003F228091B60D381609F0A3CFC301B201D1
:10BA10002091590430915A0440915B0450915C0488
:10BA20000E94DEEC9B01AC01C501B4010E9425E936
:10BA30007B018C01A50194010E94FEE987FD02C0F3
:10BA4000470158011091510400915204F0905304A1
:10BA5000E0905404C501B401212F302F4F2D5E2DED
:10BA60000E940CEC181634F4812F902FAF2DBE2DB0
:10BA70004C015D014090CC0D5090CD0D6090CE0DED
:10BA80007090CF0DC301B201A50194010E940CEC8E
:10BA90001816C4F4C501B40120E037ED43EA5CE3B5
:10BAA0000E94DEEC7B018C01C301B20128E431EE7F
:10BAB0004AE75FE30E94DEECA80197010E9425E9B6
:10BAC0004B015C018092CC0D9092CD0DA092CE0DD9
:10BAD000B092CF0DC501B4010E946DEA709396102B
:10BAE00060939510DF91CF911F910F91FF90EF9090
:10BAF000DF90CF90BF90AF909F908F907F906F908E
:10BB00005F904F903F9008958091B60D9091B70D42
:10BB1000891B877008950F931F93CF93DF93C0E025
:10BB2000D0E08E01065D144FFE01E250F54F6081BA
:10BB30007181828193810E949EEAFE01E251F54F5C
:10BB400020813181428153810E94DEEC0E9472EAA1
:10BB5000F80160837183828393832496C031D10579
:10BB600001F7DF91CF911F910F910895FC01608142
:10BB70007181828193812091FA0A3091FB0A409170
:10BB8000FC0A5091FD0A0E94DEEC0E94AEEC60932C
:10BB9000460B7093470B8093480B9093490B86E4B8
:10BBA0009BE00C948C838F929F92AF92BF92CF9226
:10BBB000DF92EF92FF920F931F93FC018B015A01CA
:10BBC000490160817181828193812091EE0A3091D7
:10BBD000EF0A4091F00A5091F10A0E94DEEC0E94B7
:10BBE000AEEC3AE3C32E3BE0D32E60933A0B709356
:10BBF0003B0B80933C0B90933D0BF801608171816E
:10BC0000828193812091F20A3091F30A4091F40AE3
:10BC10005091F50A0E94DEEC0E94AEEC24E0E22E88
:10BC2000F12CEC0CFD1C60933E0BF70171838283B9
:10BC30009383F50160817181828193812091F60A5D
:10BC40003091F70A4091F80A5091F90A0E94DEEC0F
:10BC50000E94AEEC8601085F1F4F6093420BF80113
:10BC6000718382839383F4016081718182819381E6
:10BC70002091FA0A3091FB0A4091FC0A5091FD0A8A
:10BC80000E94DEEC0E94AEECF6013C966093460BFF
:10BC9000718382839383C601B701A8019F010E942B
:10BCA000528380E090E0A0E0B0E08093B80D9093E4
:10BCB000B90DA093BA0DB093BB0D8093BC0D9093BA
:10BCC000BD0DA093BE0DB093BF0D8093C00D90939A
:10BCD000C10DA093C20DB093C30D8093C40D90937A
:10BCE000C50DA093C60DB093C70D8093C80D90935A
:10BCF000C90DA093CA0DB093CB0D1F910F91FF906A
:10BD0000EF90DF90CF90BF90AF909F908F9008956D
:10BD10008F929F92AF92BF92CF92DF92EF92FF925B
:10BD20000F931F93CF93DF93EC016B01009709F4FE
:10BD30005CC08FA9882309F058C0EEA0FFA008A519
:10BD400019A5FB01B6A0A7A090A481A4C801B701C2
:10BD50002B2D3A2D492D582D0E94FEE988230CF0F9
:10BD600044C0C801B701A80197010E94DEEC7B0125
:10BD70008C016AA97BA98CA99DA9905820E030E08C
:10BD800040E050EC0E94DEEC2EA53FA548A959A941
:10BD90000E94DEEC9B01AC01C801B7010E9425E9BD
:10BDA0000E944BED7B018C016B2D7A2D892D982DF6
:10BDB0009701A8010E94FEE9882324F4EB2CFA2CB9
:10BDC000092D182D6B2D7A2D892D982D9701A801FD
:10BDD0000E94FEE9882349F0C701D801F60186A335
:10BDE00097A3A0A7B1A781E086ABDF91CF911F9168
:10BDF0000F91FF90EF90DF90CF90BF90AF909F900A
:10BE00008F900895EF92FF920F931F93CF93DF933C
:10BE1000F090B70D00E010E020E030E04DE4E42EBB
:10BE200011C0FE9CE0011124C25BD44FC901B801CE
:10BE3000AE016EDF8F2D8F5F883009F480E0F82E21
:10BE400098018E018091B60DF81659F7C901B80115
:10BE500040E050E05DDFDF91CF911F910F91FF90A7
:10BE6000EF900895AF92BF92CF92DF92EF92FF9240
:10BE70000F931F93CF93DF93EB018A016115710537
:10BE800009F466C04115510509F462C0DAA4CBA4D7
:10BE9000BCA4ADA46EA17FA188A599A52D2D3C2D94
:10BEA0004B2D5A2D0E94FEE9882309F451C08FA919
:10BEB000882309F043C0F801E6A0F7A000A511A56A
:10BEC0006D2D7C2D8B2D9A2DA80197010E940CECD5
:10BED0001816A4F5C801B701A80197010E94DEEC6D
:10BEE0007B018C016AA97BA98CA99DA9905820E0AF
:10BEF00030E040E050EC0E94DEEC2EA53FA548A9C2
:10BF000059A90E94DEEC9B01AC01C801B7010E9457
:10BF100025E90E944BED7B018C016D2D7C2D8B2D35
:10BF20009A2D9701A8010E94FEE9882324F4ED2CA4
:10BF3000FC2C0B2D1A2DC701D80104C08D2D9C2D72
:10BF4000AB2DBA2D8EA39FA3A8A7B9A781E08EAB76
:10BF5000DF91CF911F910F91FF90EF90DF90CF90E5
:10BF6000BF90AF900895CF92DF92EF92FF920F9320
:10BF7000DF93CF930F920F92CDB7DEB78091B60DBE
:10BF80008FB7F894F090B70D8FBF8091B60D90E009
:10BF900008968F199109877090700497FCF00091B2
:10BFA000B60D03500770CC24DD2440E050E06DE472
:10BFB000E62E12C0802F002309F488E0082F0150DC
:10BFC0000E9DC0011124825B944F9A838983B60130
:10BFD00049DFA601C980DA800F1561F70F900F9035
:10BFE000CF91DF910F91FF90EF90DF90CF90089568
:10BFF0006091EF089091B70D8091B60D9817B9F048
:10C000004091B70D242F30E08DE490E0289FF0019F
:10C01000299FF00D389FF00D1124EA56F44F6081EE
:10C0200002C04F5F47708091B60D4817D1F784E08A
:10C0300070E00E94F6E24ACC1092B60D1092B70D55
:10C0400080E1EAE3FBE0DF011D928A95E9F780E0F9
:10C0500090E0A0E0B0E08093BC0D9093BD0DA09364
:10C06000BE0DB093BF0D8093C00D9093C10DA093F2
:10C07000C20DB093C30D8093C40D9093C50DA093D2
:10C08000C60DB093C70D8093C80D9093C90DA093B2
:10C09000CA0DB093CB0D8093B80D9093B90DA093BA
:10C0A000BA0DB093BB0D08952F923F924F925F92BD
:10C0B0006F927F928F929F92AF92BF92CF92DF92B8
:10C0C000EF92FF920F931F93DF93CF93CDB7DEB71D
:10C0D00066970FB6F894DEBF0FBECDBF9E8B8D8BDB
:10C0E0006A017B0148015901DC01D8966D917D916F
:10C0F0008D919C91DB970E949EEA698B7A8B8B8B4A
:10C100009C8BA70196010E94DEEC0E94EBE90E9445
:10C1100072EA6D837E838F83988769897A898B8998
:10C120009C89A50194010E94DEEC0E94EBE90E942B
:10C1300072EA69837A838B839C832D813E814F8150
:10C140005885283731054105510540F448E750E04E
:10C1500060E070E04D835E836F83788769817A81C8
:10C160008B819C81683771058105910540F488E7D2
:10C1700090E0A0E0B0E089839A83AB83BC83AD8973
:10C18000BE89AC5BBF4FAD90BD90CD90DC90139756
:10C19000A454B040BE8BAD8B6D817E818F8198851C
:10C1A0000E949EEA6D877E878F87988BC601B501B6
:10C1B0000E94A0EA1B012C0120E030E040E050E0AA
:10C1C0000E94FEE9882321F4E0E070E060E028C0EE
:10C1D00069897A898B899C899B01AC010E94DEEC7C
:10C1E0007B018C016D857E858F8598899B01AC01D3
:10C1F0000E94DEEC9B01AC01C801B7010E9424E95A
:10C200007B018C01C201B101A20191010E9425E9CB
:10C210009B01AC01C801B7010E9405EAE62F692F16
:10C220002E2F372F482F562FB901CA010E94EBE954
:10C230000E946DEA3B014C0169817A818B819C816E
:10C240000E949EEA69877A878B879C876627772773
:10C25000CB016A197B098C099D090E94A0EA5B0148
:10C260006C0120E030E040E050E00E94FEE98823CD
:10C2700021F4E0E070E060E028C069857A858B8574
:10C280009C859B01AC010E94DEEC7B018C016989DD
:10C290007A898B899C899B01AC010E94DEEC9B0111
:10C2A000AC01C801B7010E9424E97B018C01C601E1
:10C2B000B501A60195010E9425E99B01AC01C801C9
:10C2C000B7010E9405EAE62F692F2E2F372F482F3E
:10C2D000562FB901CA010E94DBEAED89FE89A088C8
:10C2E000B188C288D38886017501E618F708080965
:10C2F00019090E946DEAA8019701261B370B480B0C
:10C30000590B57FF71C0C201B10120E030E040E09D
:10C3100050E00E94FEE9882321F4E0E070E060E054
:10C3200044C0C201B101A20191010E9425E97B0133
:10C330008C01C601B5010E949EEA9B01AC01C801B7
:10C34000B7010E94DEEC7B018C016D857E858F85B7
:10C3500098899B01AC010E94DEEC9B01AC01C801F5
:10C36000B7010E9424E97B018C0169857A858B8560
:10C370009C859B01AC010E94DEEC9B01AC01C801D5
:10C38000B7010E9425E97B018C01C201B10120E0C7
:10C3900030E040E850E40E94DEEC9B01AC01C801B3
:10C3A000B7010E9405EAE62F692F2E2F372F482F5D
:10C3B000562FB901CA010E94EBE90E946DEAAC0157
:10C3C000CB01DA013C014D0197FE03C066247724BE
:10C3D00043016A147B048C049D0410F0350146016E
:10C3E00020E030E040E050E09FB7F8946D897E890E
:10C3F000645B7F4FDB018C91AC54B040BE8BAD8B46
:10C40000882321F5FD01648A758A868A978A260D1C
:10C41000371D481D591D58962D933D934D935C93A0
:10C420005B972D813E814F815885DC962D933D93FE
:10C430004D935C93DF97A05CBF4F29813A814B817C
:10C440005C812D933D934D935C9313979FBF6696AC
:10C450000FB6F894DEBF0FBECDBFCF91DF911F9115
:10C460000F91FF90EF90DF90CF90BF90AF909F9093
:10C470008F907F906F905F904F903F902F90089596
:10C480004F925F927F928F929F92AF92BF92CF9284
:10C49000DF92EF92FF920F931F93CF93DF937090F1
:10C4A000B70DC0E0D0E07DE4472E512C45C0209769
:10C4B000A9F18EA9882361F4849CF001859CF00D7C
:10C4C000949CF00D1124E25BF44F86A9882331F18E
:10C4D000EAA0FBA00CA11DA16EA17FA188A599A532
:10C4E000A80197010E9405EA5B016C01849CF001A0
:10C4F000859CF00D949CF00D1124E25BF44F66A135
:10C5000077A180A591A5A80197010E9405EA8B015A
:10C510009C01CE01B601A501C7DD1EAA739488E077
:10C52000781609F47724849CE001859CD00D949CB6
:10C53000D00D1124C25BD44F872C992487FC909492
:10C540008091B60D90E08816990609F0B0CF20973B
:10C55000E9F0EAA0FBA00CA11DA16EA17FA188A516
:10C5600099A5A80197010E9405EA5B016C016DEC99
:10C570007CEC8CE49DE3A80197010E9405EA8B0105
:10C580009C01CE01B601A5018FDD1EAADF91CF91DE
:10C590001F910F91FF90EF90DF90CF90BF90AF90E1
:10C5A0009F908F907F905F904F900895DCDC2ADC05
:10C5B00067CF2F923F924F925F926F927F928F92AE
:10C5C0009F92AF92BF92CF92DF92EF92FF920F9322
:10C5D0001F93DF93CF93CDB7DEB7CC59D0400FB6C2
:10C5E000F894DEBF0FBECDBF5C014B013A012901BB
:10C5F000C756DF4FE882C959D040C656DF4FF88290
:10C60000CA59D040C556DF4F0883CB59D040C456D5
:10C61000DF4F1883CC59D040E796DFAECEAEE79718
:10C620008091B60D8F5F883009F480E0282F332782
:10C6300027FD309538A72FA307C00E94CF9080E038
:10C640000E9401370E948FD48091B70D90E04FA1D6
:10C6500058A58417950789F36091EE0A7091EF0A47
:10C660008091F00A9091F10AE5966CAF7DAF8EAFA4
:10C670009FAFE597D5012D913D914D915C910E9421
:10C68000DEEC0E94AEECCD57DF4F6883C358D0403C
:10C69000CC57DF4F7883C458D040CB57DF4F8883C7
:10C6A000C558D040CA57DF4F9883C658D040209114
:10C6B000F20A3091F30A4091F40A5091F50AE1969A
:10C6C0002CAF3DAF4EAF5FAFE197CA01B901D401C6
:10C6D0002D913D914D915C910E94DEEC0E94AEEC5B
:10C6E000C957DF4F6883C758D040C857DF4F78839A
:10C6F000C858D040C757DF4F8883C958D040C65765
:10C70000DF4F9883CA58D0402091F60A3091F70A3B
:10C710004091F80A5091F90AAD962CAF3DAF4EAF5B
:10C720005FAFAD97CA01B901D3012D913D914D91F4
:10C730005C910E94DEEC0E94AEECC557DF4F68832F
:10C74000CB58D040C457DF4F7883CC58D040C35724
:10C75000DF4F8883CD58D040C257DF4F9883CE58E3
:10C76000D0402091FA0A3091FB0A4091FC0A509186
:10C77000FD0AA9962CAF3DAF4EAF5FAFA997CA0196
:10C78000B901D2012D913D914D915C910E94DEEC59
:10C790000E94AEECC157DF4F6883CF58D040C057DE
:10C7A000DF4F7883C059D040CF56DF4F8883C159BF
:10C7B000D040CE56DF4F9883C259D0408091B60DFD
:10C7C000E82FF0E0A596FFAFEEAFA5978DE490E0DF
:10C7D0009F01289FF001299FF00D389FF00D112433
:10C7E000E25BF44FE45BFF4F1082EC54F040409169
:10C7F0003A0B50913B0B60913C0B70913D0BA39613
:10C800004CAF5DAF6EAF7FAFA397CD57DF4F888141
:10C810009981AA81BB81C358D040841B950BA60B7C
:10C82000B70B6F968CAF9DAFAEAFBFAF6F978083E6
:10C830009183A283B383B7FF0BC0B095A095909569
:10C8400081959F4FAF4FBF4F80839183A283B38366
:10C8500020913E0B30913F0B4091400B5091410B8A
:10C860006B962CAF3DAF4EAF5FAF6B97C957DF4FA5
:10C87000688179818A819B81C758D040621B730B84
:10C88000840B950B67966CAF7DAF8EAF9FAF6797AC
:10C890008DE490E0A596AEADBFADA597A89FF00141
:10C8A000A99FF00DB89FF00D1124E25BF44F67963D
:10C8B0002CAD3DAD4EAD5FAD679724833583468388
:10C8C000578357FF0DC0DA01C901B095A095909527
:10C8D00081959F4FAF4FBF4F84839583A683B783C6
:10C8E0004091420B5091430B6091440B7091450B6A
:10C8F00063964CAF5DAF6EAF7FAF6397C557DF4FA9
:10C9000088819981AA81BB81CB58D040841B950B2B
:10C91000A60BB70B2F968CAF9DAFAEAFBFAF2F97C7
:10C920008DE490E0A596AEADBFADA597A89FF001B0
:10C93000A99FF00DB89FF00D1124E25BF44F2F96E4
:10C940002CAD3DAD4EAD5FAD2F972087318742872F
:10C95000538757FF0DC0DA01C901B095A095909596
:10C9600081959F4FAF4FBF4F80879187A287B38735
:10C970002090460B3090470B4090480B5090490B4D
:10C98000C157DF4F488159816A817B81CF58D040A0
:10C9900042195309640975092B964CAF5DAF6EAF10
:10C9A0007FAF2B97E091EE08F0E0EE0FFF1FEE0F48
:10C9B000FF1FE05EFB4F608171818281938127962A
:10C9C0006CAF7DAF8EAF9FAF27978091120490918F
:10C9D000130423969FAF8EAF23972B966CAD7DAD3E
:10C9E0008EAD9FAD2B9797FF07C090958095709562
:10C9F00061957F4F8F4F9F4F0E94A0EA27962CADE5
:10CA00003DAD4EAD5FAD27970E94DEEC0E946DEA12
:10CA10002396AEADBFAD23979D01442737FD4095CA
:10CA2000542F0E94B0ED24E630E040E050E00E9438
:10CA300024EE8DE490E0A5966EAD7FADA597689F3E
:10CA4000F001699FF00D789FF00D1124E25BF44F27
:10CA5000DF011C96248711963C93119712964C93F4
:10CA6000129713965C93E080F180028113816480B9
:10CA7000758086809780A084B184C284D384C901E4
:10CA8000DA018A159B05AC05BD0514F4D601C50174
:10CA900086159705A805B90514F4D401C3019C01B6
:10CAA000AD018E159F05A007B10714F4A8019701E9
:10CAB0008DE490E0A596AEADBFADA597A89FB0015F
:10CAC000A99F700DB89F700D1124625B744FFB011C
:10CAD000208B318B428B538B26303105410551051C
:10CAE00010F40C94BA6EE85BFF4F8091EF089091C0
:10CAF000F008AA2797FDA095BA2F80839183A2837F
:10CB0000B383DB0190961C92CD57DF4F288139818A
:10CB10004A815B81C358D040A3968CAD9DADAEAD2C
:10CB2000BFADA397281739074A075B0724F481E0B4
:10CB3000DB0190968C93C957DF4F288139814A8158
:10CB40005B81C758D0406B966CAD7DAD8EAD9FAD0F
:10CB50006B97261737074807590794F48DE490E040
:10CB6000A596AEADBFADA597A89FF001A99FF00D0A
:10CB7000B89FF00D1124E25BF44F80A1826080A386
:10CB8000C557DF4F288139814A815B81CB58D0401E
:10CB900063966CAD7DAD8EAD9FAD6397261737075D
:10CBA0004807590794F48DE490E0A596AEADBFAD6B
:10CBB000A597A89FF001A99FF00DB89FF00D112433
:10CBC000E25BF44F80A1846080A3C157DF4F2881CE
:10CBD00039814A815B81CF58D04022153305440505
:10CBE000550594F48DE490E0A5964EAD5FADA59704
:10CBF000489FF001499FF00D589FF00D1124E25B12
:10CC0000F44F80A1886080A38DE490E0A5966EAD7E
:10CC10007FADA597689FF001699FF00D789FF00D9B
:10CC20001124E25BF44FE796AEADBFADE7978C9170
:10CC300081A3208131814281538121962CAF3DAF68
:10CC40004EAF5FAF2197211531054105510509F020
:10CC50005F988DE490E0A5964EAD5FADA597489F97
:10CC6000F001499FF00D589FF00D1124E25BF44F45
:10CC700064807580868097806114710481049104BA
:10CC800009F08A988DE490E0A5966EAD7FADA597EA
:10CC9000689FF001699FF00D789FF00D1124E25B11
:10CCA000F44FA084B184C284D384A114B104C1041C
:10CCB000D10441F09FB7F894809108018E7F809352
:10CCC00008019FBF8DE490E0A596AEADBFADA597DE
:10CCD000A89FF001A99FF00DB89FF00D1124E25B11
:10CCE000F44F84859585A685B7850097A105B10584
:10CCF00011F40C94B16E80914B0B882319F0815084
:10CD000080934B0B80914C0B882319F081508093BA
:10CD10004C0B80914D0B882319F0815080934D0B63
:10CD2000E796EEADFFADE7978081813051F081301D
:10CD300018F08230E9F40FC0129880E180934B0B19
:10CD400012C0479880E180934C0B80914B0B882355
:10CD500079F4129A0DC080E180934D0B80914B0BBA
:10CD6000882309F4129A80914C0B882309F4479A7E
:10CD700020900E0B30900F0B4090100B5090110B29
:10CD8000C756DF4F6881C959D040C656DF4F7881FA
:10CD9000CA59D040C556DF4F8881CB59D040C456C0
:10CDA000DF4F9881CC59D040A20191010E94FEE949
:10CDB00087FD16C0C756DF4F8881C959D040C65677
:10CDC000DF4F9881CA59D040C556DF4FA881CB5953
:10CDD000D040C456DF4FB881CC59D0401C012D0142
:10CDE0006F966CAD7DAD8EAD9FAD6F970E94A0EA42
:10CDF000E5962CAD3DAD4EAD5FADE5970E9405EAE1
:10CE0000C158DF4F6883CF57D040C058DF4F788379
:10CE1000C058D040CF57DF4F8883C158D040CE573D
:10CE2000DF4F9883C258D040AC01CB01DA0189832F
:10CE30009A83AB83BC8367966CAD7DAD8EAD9FADA1
:10CE400067970E94A0EAE1962CAD3DAD4EAD5FAD77
:10CE5000E1970E9405EAEC966FAFEC97ED967FAFF5
:10CE6000ED97EE968FAFEE97EF969FAFEF97AC01F1
:10CE7000CB01DA018D839E83AF83B8872F966CAD8B
:10CE80007DAD8EAD9FAD2F970E94A0EAAD962CADE3
:10CE90003DAD4EAD5FADAD970E9405EAE8966FAF30
:10CEA000E897E9967FAFE997EA968FAFEA97EB9616
:10CEB0009FAFEB97AC01CB01DA0189879A87AB87EB
:10CEC000BC872B966CAD7DAD8EAD9FAD2B970E9430
:10CED000A0EAA9962CAD3DAD4EAD5FADA9970E94DD
:10CEE00005EA27962CAD3DAD4EAD5FAD27970E946C
:10CEF000DEEC7B018C0123962EAD3FAD2397B9016B
:10CF0000882777FD8095982F0E94A0EA9B01AC01AD
:10CF1000C801B7010E94DEEC20E030E048EC52E4AA
:10CF20000E9405EA9B01AC016D877E878F87988BF5
:10CF300021966CAD7DAD8EAD9FAD219766307105AC
:10CF4000810591051CF576E0671671048104910452
:10CF5000ECF486E0A816B104C104D104BCF48DE45D
:10CF600090E0A596AEADBFADA597A89FF001A99F93
:10CF7000F00DB89FF00D1124E25BF44FDA01C90106
:10CF8000BF7786A797A7A0ABB1AB5DC0C158DF4FF5
:10CF90002881CF57D040C058DF4F3881C058D0408B
:10CFA000CF57DF4F4881C158D040CE57DF4F58810F
:10CFB000C258D040B901CA010E9495ED3B014C0115
:10CFC000EC962FADEC97ED963FADED97EE964FAD0D
:10CFD000EE97EF965FADEF97B901CA010E9495ED0C
:10CFE0005B016C01E8962FADE897E9963FADE997B4
:10CFF000EA964FADEA97EB965FADEB97B901CA01A0
:10D000000E9495ED7B018C01C401B301A60195013D
:10D010000E9425E9A80197010E9425E90E944BED95
:10D020002DE430E0A5964EAD5FADA597429FF0018F
:10D03000439FF00D529FF00D1124E25BF44F66A761
:10D0400077A780AB91AB8DE490E0A5966EAD7FADF8
:10D05000A597689FF001699FF00D789FF00D11244E
:10D06000E25BF44F86A597A5A0A9B1A989AF9AAFB5
:10D07000ABAFBCAF60E070E080E89FE329AD3AADB4
:10D080004BAD5CAD0E9405EA9B01AC01C201B10150
:10D090000E94DEEC2B013C018091B60D9091B70D02
:10D0A000A82FB0E01896A91BB109A770B070BEA355
:10D0B000ADA3A230B1050CF451C05D01CC24B7FC86
:10D0C000C094DC2CC601B5010E94A0EA20E030E04B
:10D0D00040E850E40E94FEE988230CF03FC060E085
:10D0E00074E284E799E4A30192010E9405EA0E9498
:10D0F000AEEC7B018C016091DA0A7091DB0A8091C1
:10D10000DC0A9091DD0AE616F7060807190730F5E4
:10D110006E197F09800B910B660F771F881F991F6F
:10D12000A60195010E9402EECA01B9010E949EEA81
:10D130000E94AEEC9B01AC012E0D3F1D401F511F04
:10D14000CA01B9010E949EEA9B01AC0160E074E251
:10D1500084E799E40E9405EA2B013C018DE490E00C
:10D16000A596EEADFFADA597E89F8001E99F100D54
:10D17000F89F100D1124025B144F69AD7AAD8BAD91
:10D180009CADA30192010E94DEECD80192966D93B2
:10D190007D938D939C93959750966D917D918D91F4
:10D1A0009C9153970E949EEAA30192010E94DEEC9B
:10D1B0000E94EBE90E9472EAF80160AF71AF82AFA2
:10D1C00093AFCD56DF4F1882C359D040CC56DF4FB6
:10D1D0001882C459D04020E8222E9FE3392E88249B
:10D1E0009924E1E0F0E0EC0FFD1FE80DF91DC3010B
:10D1F000B20120813181428153810E94DEECE1E164
:10D20000F0E0EC0FFD1FE80DF91D60837183828350
:10D2100093835B016C01E894D7F8F401E252F54F77
:10D22000E080F18002811381C601B501A801970158
:10D230000E940CEC1816CCF4C801B701A6019501A8
:10D240000E9405EA6B017C01CD56DF4F6881C3590E
:10D25000D040CC56DF4F7881C459D040C101A701DE
:10D2600096010E94FEE988236CF4CD56DF4F888139
:10D27000C359D040CC56DF4F9881C459D040D1011A
:10D280006C017D0124E030E0820E931E30E18316B4
:10D29000910471F0D701C601CD56DF4FC882C35942
:10D2A000D040CC56DF4F9883C459D0401D0199CF50
:10D2B000C701B60120E030E040E85FE30E94FEE9EC
:10D2C00088230CF04CC08E010F5E1F4F81E2A82E08
:10D2D000B12CAC0EBD1ED8016D917D918D919C91AC
:10D2E000A70196010E94DEECF8016193719381938E
:10D2F00091938F01EA15FB0571F78DE490E0A596F7
:10D300002EAD3FADA597289F8001299F100D389F16
:10D31000100D1124025B144FD80192966D917D91EE
:10D320008D919C919597A70196010E94DEECF801E2
:10D3300062A373A384A395A360AD71AD82AD93ADD9
:10D340000E949EEAA70196010E94DEEC0E9472EA0A
:10D35000D801D8966D937D938D939C93DB978DE444
:10D3600090E0A596EEADFFADA597E89F8001E99FFF
:10D37000100DF89F100D1124025B144FD801509628
:10D380006D917D918D919C9153970E949EEAF80139
:10D3900026A537A540A951A90E9405EA1B012C0129
:10D3A000F80180819181A281B3810097A105B10527
:10D3B00049F584819581A681B7810097A105B105C2
:10D3C00009F580859185A285B3850097A105B105F2
:10D3D000C9F4C201B1012091160B3091170B409195
:10D3E000180B5091190B0E94DEEC0E94EBE90C5BCC
:10D3F0001F4F0E9472EAD8016D937D938D939C9389
:10D40000139771C1C201B1012091120B3091130B1E
:10D410004091140B5091150B0E94DEEC0E94EBE939
:10D420000E9472EA2DE430E0A596EEADFFADA5971F
:10D43000E29F6001E39FD00CF29FD00C11242EE4F8
:10D440003BE0C20ED31EB4E46B2E712C6C0C7D1C21
:10D45000D3016D937D938D939C93139780902A0BAA
:10D4600090902B0BA0902C0BB0902D0B0E949EEA5D
:10D470007B018C01F60160817181828193810E9420
:10D48000A0EA9B01AC01C801B7010E94DEEC7B0160
:10D490008C01D60150966D917D918D919C91539701
:10D4A0000E949EEA9B01AC01C801B7010E9405EAF7
:10D4B0007B018C01C501B4010E949EEA9B01AC0175
:10D4C000C801B7010E940CEC18162CF4F3018082FD
:10D4D0009182A282B38280902E0B90902F0BA0900D
:10D4E000300BB090310B8DE490E0A5962EAD3FADA2
:10D4F000A597289F6001299FD00C389FD00C11243C
:10D500004EE45BE0C40ED51EA4E46A2E712C6C0CB4
:10D510007D1CD3016D917D918D919C910E949EEA1D
:10D520007B018C01F60164817581868197810E945F
:10D53000A0EA9B01AC01C801B7010E94DEEC7B01AF
:10D540008C01D60150966D917D918D919C91539750
:10D550000E949EEA9B01AC01C801B7010E9405EA46
:10D560007B018C01C501B4010E949EEA9B01AC01C4
:10D57000C801B7010E940CEC18162CF4F30180824C
:10D580009182A282B3828090360B9090370BA0904C
:10D59000380BB090390B8DE490E0A5962EAD3FADE1
:10D5A000A597289F6001299FD00C389FD00C11248B
:10D5B0004EE45BE0C40ED51EF4E46F2E712C6C0CAF
:10D5C0007D1CD3016D917D918D919C910E949EEA6D
:10D5D0007B018C01F60164857585868597850E949F
:10D5E000A0EA9B01AC01C801B7010E94DEEC7B01FF
:10D5F0008C01D60150966D917D918D919C915397A0
:10D600000E949EEA9B01AC01C801B7010E9405EA95
:10D610007B018C01C501B4010E949EEA9B01AC0113
:10D62000C801B7010E940CEC18162CF4F30180829B
:10D630009182A282B3828090320B9090330BA090A3
:10D64000340BB090350B8DE490E0A5962EAD3FAD38
:10D65000A597289F6001299FD00C389FD00C1124DA
:10D660004EE45BE0C40ED51EE4E46E2E712C6C0C0F
:10D670007D1CD3016D917D918D919C910E949EEABC
:10D680007B018C01F60160857185828593850E94FE
:10D69000A0EA9B01AC01C801B7010E94DEEC7B014E
:10D6A0008C01D60150966D917D918D919C915397EF
:10D6B0000E949EEA9B01AC01C801B7010E9405EAE5
:10D6C0007B018C01C501B4010E949EEA9B01AC0163
:10D6D000C801B7010E940CEC18162CF4F3018082EB
:10D6E0009182A282B3828DE490E0A5962EAD3FADEB
:10D6F000A597289F6001299FD00C389FD00C11243A
:10D700004EE45BE0C40ED51EF601EC5BFF4F60817A
:10D710007181828193810E949EEA7B018C01A2012A
:10D7200091010E9405EAD601D2966D937D938D9367
:10D730009C93D597C801B7012DEB37E346E051E440
:10D740000E94DEEC0E946DEAF601648F758F868F71
:10D75000978F60901A0B70901B0B80901C0B909011
:10D760001D0BC401B30120E030E040E05FE30E9404
:10D77000DEEC5B016C01298D3A8D4B8D5C8D2DAB00
:10D780003EAB4FAB58AF40911E0B50911F0B6091B9
:10D79000200B7091210B49AB5AAB6BAB7CABCB012F
:10D7A000BA0120E030E040E05FE30E94DEEC7B0164
:10D7B0008C016DA97EA98FA998AD9F77A8019701CB
:10D7C0000E940CEC181644F4C601B501A80197019B
:10D7D0000E94FEE9882314F4860175016D8D7E8D0B
:10D7E0008F8D98A16DA77EA78FA798AB8091220BF4
:10D7F0009091230BA091240BB091250B89A79AA798
:10D80000ABA7BCA7BC01CD0120E030E040E05FE366
:10D810000E94DEEC1B012C016DA57EA58FA598A9A9
:10D820009F77A20191010E940CEC181644F4C801E4
:10D83000B701A20191010E94FEE9882314F41701A7
:10D8400028018DE490E0A596AEADBFADA597A89F49
:10D85000F001A99FF00DB89FF00D1124E25BF44F89
:10D8600022A133A144A155A129A33AA34BA35CA3B0
:10D87000C201B1010E94FEE987FD04C029A03AA0BF
:10D880004BA05CA04DA15EA1423051050CF405C136
:10D890005091B80DCB56DF4F5883C559D040609199
:10D8A000B90DCA56DF4F6883C659D0407091BA0D82
:10D8B000C956DF4F7883C759D0408091BB0DC856F9
:10D8C000DF4F8883C859D040652FCA56DF4F788113
:10D8D000C659D040C956DF4F8881C759D040C85675
:10D8E000DF4F9881C859D04027E137EB41ED58E32D
:10D8F0000E940CEC18160CF0D0C069897A898B89CB
:10D900009C892091BC0D3091BD0D4091BE0D509170
:10D91000BF0D0E9424E99B01AC010E94DEEC7B015B
:10D920008C016D897E898F89988D2091C00D3091F1
:10D93000C10D4091C20D5091C30D0E9424E99B017D
:10D94000AC010E94DEEC9B01AC01C801B7010E9452
:10D9500025E90E944BED7B018C01A40193010E94FB
:10D960000CEC18165CF00F2EF0E06F2EF0E07F2E1E
:10D97000F0E88F2EFFE39F2EF02D08C0C401B30105
:10D98000A80197010E9405EA3B014C016DA97EA9FF
:10D990008FA998AD2091C40D3091C50D4091C60D51
:10D9A0005091C70D0E9424E97B018C01E89417F97E
:10D9B000C801B70129A93AA94BA95CA90E940CEC9E
:10D9C000181694F469A97AA98BA99CA9A8019701B2
:10D9D0000E9405EA5B016C01C401B301A601950137
:10D9E0000E94FEE9882314F4640153016DA57EA50D
:10D9F0008FA598A92091C80D3091C90D4091CA0DED
:10DA00005091CB0D0E9424E97B018C01E89417F919
:10DA1000C801B70129A53AA54BA55CA50E940CEC4D
:10DA2000181694F469A57AA58BA59CA5A801970161
:10DA30000E9405EA7B018C01C601B501A80197018E
:10DA40000E94FEE9882314F48601750169A17AA178
:10DA50008BA19CA1A80197010E94DEEC7B018C01A7
:10DA6000CB56DF4F6881C559D040CA56DF4F788109
:10DA7000C659D040C956DF4F8881C759D040C856D3
:10DA8000DF4F9881C859D040A80197010E94FEE954
:10DA900087FD19C0D801C70102C0D201C101CB5610
:10DAA000DF4F8883C559D040CA56DF4F9883C65987
:10DAB000D040C956DF4FA883C759D040C856DF4F62
:10DAC000B883C859D0408DE490E0A596AEADBFAD07
:10DAD000A597A89F8001A99F100DB89F100D112434
:10DAE000025B144FCB56DF4F8881C559D040CA56D0
:10DAF000DF4F9881C659D040C956DF4FA881C7591A
:10DB0000D040C856DF4FB881C859D040F80182A72D
:10DB100093A7A4A7B5A762A973A984A995A99058AA
:10DB200020E030E040E050EC0E94DEECD8019E9610
:10DB30002D913D914D915C91D1970E94DEEC2BE0AF
:10DB400037ED43E25BE30E9425E90E944BEDF62EA0
:10DB5000E72ED82EC92ECB56DF4F6881C559D0404D
:10DB6000CA56DF4F7881C659D040C956DF4F8881E9
:10DB7000C759D040C856DF4F9881C859D0402F2D83
:10DB80003E2D4D2D5C2D0E94FEE987FD14C0CB5625
:10DB9000DF4FF882C559D040CA56DF4FE882C659D8
:10DBA000D040C956DF4FD882C759D040C856DF4F42
:10DBB000C882C859D0408DE490E0A596EEADFFAD87
:10DBC000A597E89F8001E99F100DF89F100D112483
:10DBD000025B144FCB56DF4F8881C559D040CA56DF
:10DBE000DF4F9881C659D040C956DF4FA881C75929
:10DBF000D040C856DF4FB881C859D040F80186A33D
:10DC000097A3A0A7B1A762A173A184A195A12F2D6D
:10DC10003E2D4D2D5C2D0E94FEE918162CF081E062
:10DC2000D801D7968C9302C0F80117AA8DE490E032
:10DC3000A5962EAD3FADA597289FF001299FF00D29
:10DC4000389FF00D1124E25BF44F81E086ABACEB22
:10DC5000BDE0FE01719680E101900D928150E1F7E7
:10DC60008DE490E0A5964EAD5FADA597489F60010D
:10DC7000499FD00C589FD00C11246EE47BE0C60E57
:10DC8000D71ED6019296ED90FD900D911C9195971F
:10DC9000E092B80DF092B90D0093BA0D1093BB0D40
:10DCA00096966D917D918D919C919997A801970180
:10DCB0000E9405EA4B015C01C201B101A801970174
:10DCC0000E9405EA8B019C01C601B501A4010E94D6
:10DCD0005460BFA1B093B60DC157DF4F2881398181
:10DCE0004A815B81CF58D0402093460B3093470B3D
:10DCF0004093480B5093490BC557DF4F48815981DA
:10DD00006A817B81CB58D0404093420B5093430BA8
:10DD10006093440B7093450BC957DF4F688179813D
:10DD20008A819B81C758D04060933E0B70933F0B14
:10DD30008093400B9093410BCD57DF4F88819981A1
:10DD4000AA81BB81C358D04080933A0B90933B0B80
:10DD5000A0933C0BB0933D0B0E94D6620E94C882F8
:10DD600009C02090260B3090270B4090280B509034
:10DD7000290B06C8C456DF4F0FB6F894DEBF0FBE9E
:10DD8000CDBFCF91DF911F910F91FF90EF90DF906A
:10DD9000CF90BF90AF909F908F907F906F905F904B
:10DDA0004F903F902F900895FF920F931F93CF9322
:10DDB000DF938B010E9423E2EB01FF24FA9409C058
:10DDC0000E9423E26C1B7D0B6017710710F080E04E
:10DDD00008C0FEBC0DB407FEFDCF8EB58F3F81F7A6
:10DDE00081E0DF91CF911F910F91FF900895FC0189
:10DDF0004281242F30E0C9019595879580658CBDBF
:10DE000040FF02C080E004C080E0463009F081E0BD
:10DE10008DBD808160E00C9487E4DF92EF92FF92E9
:10DE20000F931F93CF93DF93EC01D62E79018A01D4
:10DE3000DEDFCE016CE271E0B7DF8D2D80648EBD38
:10DE40000DB407FEFDCF28E130E0D801C701022E56
:10DE500004C0B695A795979587950A94D2F78EBD7D
:10DE60000DB407FEFDCF285030408FEF283F380714
:10DE700061F7DD2011F485E906C088E0D81611F4B9
:10DE800087E801C08FEF8EBD0DB407FEFDCF8CE09B
:10DE9000D81631F48FEF8EBD0DB407FEFDCF8EB5D1
:10DEA0009FEF2FEF2EBD0DB407FEFDCF8EB587FF80
:10DEB00004C0992311F09150F5CF8B83DF91CF915E
:10DEC0001F910F91FF90EF90DF900895FC018081EA
:10DED00061E00C9487E4DC016EBDFA0120E030E0E3
:10DEE0000DB407FEFDCF80818EBD0DB407FEFDCFC2
:10DEF00081818EBD2E5F3F4F329682E02030380701
:10DF000079F70DB407FEFDCF8FEF8EBD0DB407FE80
:10DF1000FDCF8FEF8EBD0DB407FEFDCF8FEF8EBD11
:10DF20000DB407FEFDCF8EB513968C9313978F71AA
:10DF3000853011F481E0089583E111968C93119757
:10DF4000CD01C4DF80E00895CF92DF92EF92FF927F
:10DF50000F931F93CF93DF93EC017A018B0169013B
:10DF60008C81833039F059E0EE0CFF1C001F111F2B
:10DF70005A95D1F7CE0168E1A80197014EDF8823B9
:10DF800011F086E020C0CE016EEFA601A4DF882349
:10DF9000D9F0CE0168E572E007DF882311F487E14C
:10DFA00012C0CE016DE020E030E040E050E035DF0F
:10DFB000882341F48FEF8EBD0DB407FEFDCF8EB5E3
:10DFC000882371F086E18983CE0180DF80E0DF91D4
:10DFD000CF911F910F91FF90EF90DF90CF90089518
:10DFE000CE0174DF81E0F3CFBF92CF92DF92EF9248
:10DFF000FF920F931F93CF93DF93EC016B017A0194
:10E000000E9423E28B01BB24BA9409C00E9423E240
:10E01000601B710B6D52714010F081E10BC0BEBCF2
:10E020000DB407FEFDCF8EB58B838F3F79F38E3F06
:10E0300039F08FE08983CE0149DF8FEF8EBD34C088
:10E04000D7011197EF28D9F08FEF8EBD20E030E097
:10E050009FEF0BC00DB407FEFDCF8EB5F601E20FAA
:10E06000F31F80839EBD2F5F3F4F2A173B0790F31E
:10E070000DB407FEFDCF8EB5AC0DBD1D8C938FEF9B
:10E080008EBD0DB407FEFDCF8EB58FEF8EBD0DB4E6
:10E0900007FEFDCF8EB5CE0119DF8FEF8EBD0DB41B
:10E0A00007FEFDCF81E004C00DB407FEFDCF80E088
:10E0B000DF91CF911F910F91FF90EF90DF90CF9064
:10E0C000BF900895CF92DF92EF92FF920F931F932C
:10E0D000CF93DF93EC017A018B0169018C8183304E
:10E0E00039F0A9E0EE0CFF1C001F111FAA95D1F713
:10E0F000CE0161E1A801970190DE882331F084E030
:10E100008983CE01E3DE80E005C0CE01B60140E0A8
:10E1100052E06ADFDF91CF911F910F91FF90EF9056
:10E12000DF90CF900895BF92CF92DF92EF92FF924F
:10E130000F931F93CF93DF93EC01B62E1C821982AD
:10E1400048830E9423E26B01888161E00E94D4E34E
:10E15000CE01BCDE82E360E00E94D4E383E361E0B1
:10E160000E94D4E384E361E00E94D4E385E361E0AC
:10E170000E94D4E385E361E00E9487E485E08A831E
:10E1800082E58CBD1DBC80E09FEF9EBD0DB407FEF7
:10E19000FDCF8F5F8A30C9F709C00E9423E26C1956
:10E1A0007D09615D774010F081E059C0CE0160E0EB
:10E1B00020E030E040E050E030DE182F8B838130EB
:10E1C00061F7CE0168E02AEA31E040E050E025DE68
:10E1D00082FF02C01C8311C080E02FEF2EBD0DB462
:10E1E00007FEFDCF9EB58F5F8430C1F79B839A3ABF
:10E1F00011F082E034C082E08C838C81823021F087
:10E20000EE24FF2487010FC0E12CF12C012D00E446
:10E21000102F09C00E9423E26C197D09615D7740CF
:10E2200010F08AE01CC0CE0167E320E030E040E05F
:10E2300050E0F3DDCE0169E2A8019701EEDD8B83AA
:10E24000882341F78C81823019F5CE016AE320E002
:10E2500030E040E050E0E1DD882329F088E0898368
:10E26000CE0134DE20C08FEF8EBD0DB407FEFDCF92
:10E270008EB5807C803C11F483E08C8380E09FEF3E
:10E280009EBD0DB407FEFDCF2EB58F5F8330C1F765
:10E29000CE011CDE86E08B1518F488E1898303C06B
:10E2A000BA8281E001C080E0DF91CF911F910F9190
:10E2B000FF90EF90DF90CF90BF900895CF93DF93C2
:10E2C000EB01DC0190E020E03EE28C91803269F0CD
:10E2D000283029F4FE01E90FF11D30839F5FFE0114
:10E2E000E90FF11D8C9180839F5F2F5F11962B307A
:10E2F00061F7C90FD11D1882DF91CF9108950F9357
:10E300001F93CF93DF93DC01EB018A0180E090E063
:10E3100020E2FE01E80FF91F208301968B30910562
:10E32000C1F757E040E024C0622F2E3219F088E098
:10E330009BE007C05A3051F15AE048E018C032174C
:10E3400029F1FC01019634913323C9F75417F0F0F9
:10E350002132E0F02F37D0F4822F81568A3110F429
:10E36000622F6052FE01E40FF11D60834F5F119632
:10E370002C91222311F02F32B9F6F801B183A0833A
:10E3800090E08881803219F091E001C090E0892FFF
:10E39000DF91CF911F910F9108956F927F928F928D
:10E3A0009F92AF92BF92CF92DF92EF92FF920F9324
:10E3B0001F93CF93DF93EC017A018B012B812223F2
:10E3C00009F480C089899A89AB89BC89841795072B
:10E3D000A607B70708F476C085C0E114F10401056B
:10E3E000110551F41C821D821E821F821886198617
:10E3F0001A861B8681E067C0288539854A855B853A
:10E40000E98DFA8D858590E0099621503040404095
:10E41000504039014A01082E04C09694879477949D
:10E4200067940A94D2F72F5F3F4F4F4F5F4F089486
:10E43000E108F108010911095701680104C0D694E7
:10E44000C794B794A7948A95D2F70894E11CF11C5D
:10E45000011D111DA614B704C804D90428F0211504
:10E4600031054105510549F48D899E89AF89B88DE3
:10E470008C839D83AE83BF8316C0A618B708C808D7
:10E48000D90811C04C815D816E817F81898D9A8D03
:10E4900094010E945D7D0894A108B108C108D108CB
:10E4A000882331F40FC084E0882E912C8C0E9D1EA1
:10E4B000A114B104C104D10429F7E886F9860A87BA
:10E4C0001B8798CF80E0DF91CF911F910F91FF9034
:10E4D000EF90DF90CF90BF90AF909F908F907F9004
:10E4E0006F900895223009F078CFE7CFCF93DF9374
:10E4F000EC018C859D85AE85BF8540E0611141E0D2
:10E50000BC01CD010E94377B882319F420E030E064
:10E510000AC08889282F30E095E0220F331F9A9592
:10E52000E1F72A52324FC901DF91CF9108950F933D
:10E530001F93CF93DF938C01FC0183818823D9F152
:10E54000818187FF35C0C80161E0D0DFEC01009711
:10E5500091F18881853E79F1F8018381823040F420
:10E5600081899289A389B4898C8F9D8FAE8FBF8F4B
:10E57000F80185899689A789B08D9B8F8A8FCD01F7
:10E58000AA27BB279D8B8C8BE091D00DF091D10DEC
:10E59000309751F0BE016A5E7F4FCE0148961995C3
:10E5A000888D998D9B8B8A8BF80181818F778183F0
:10E5B0000E94FC7A04C081E0F801808380E0DF9152
:10E5C000CF911F910F9108950F931F938C01AFDF8F
:10E5D000F80113821F910F910895FC018381882314
:10E5E00011F0CF01F1CF0895CF93DF93FC01EB0140
:10E5F0008381882381F08250823020F48FE28883E7
:10E60000198207C0CF0160E071DF009721F0BE01E1
:10E6100055DE81E001C080E0DF91CF9108956F92D7
:10E620007F928F929F92AF92BF92CF92DF92EF92A2
:10E63000FF920F931F93DF93CF9300D00F92CDB72C
:10E64000DEB77C015A016B01DC0113968C911397A4
:10E65000813009F08EC011968C9181FF8AC09DC0D7
:10E660000097A105B10511F481E084C0F701608431
:10E67000718482849384C701B601A5018EDE88234C
:10E6800009F477C0D70159968D919C915A97A1149E
:10E69000B104C104D10489F455964D915D916D91F9
:10E6A0007C9158970E94D27D882309F462C0F701BB
:10E6B000158A168A178A108E44C0D70114964D9178
:10E6C0005D916D917C9117979E012F5F3F4F0E9446
:10E6D0005D7D882309F44DC0D7015996ED91FC91D9
:10E6E0005A9749815A816B817C818789803149F4AD
:10E6F000483FBFEF5B07B0E06B07B0E07B0748F037
:10E7000020C0483F8FEF58078FEF68078FE07807EA
:10E71000C0F4CF010E94D27D882359F1D70114960D
:10E720004D915D916D917C91179759968D919C912A
:10E730005A970FEF1FEF2FEF3FE00E94D77C8823FF
:10E74000C1F0F701A18AB28AC38AD48A8181806824
:10E750008183C701ECDE882361F0B601A5016A144C
:10E760007B048C049D0410F4B401A301C70115DEE1
:10E7700001C080E00F900F900F900F90CF91DF912C
:10E780001F910F91FF90EF90DF90CF90BF90AF90CF
:10E790009F908F907F906F900895F7018189928963
:10E7A000A389B48984179507A607B70708F058CF3F
:10E7B000E0CFCF93DF93EC0140E050E060E070E009
:10E7C0002EDF882359F0CE0161E090DEFC01009736
:10E7D00029F085EE80831B820FD701C080E0DF9196
:10E7E000CF9108952F923F924F925F926F927F92B6
:10E7F0008F929F92AF92BF92CF92DF92EF92FF9251
:10E800000F931F93CF93DF93EC012A018B81882311
:10E8100009F4B5C0898180FFB2C0C7C025014E1878
:10E820005F083B0174E0272E312C2C0E3D1E420167
:10E83000A0C0288539854A855B856FEFA62E61E0EB
:10E84000B62EA222B3228B8179018A0199E0169516
:10E850000795F794E7949A95D1F7E98DFA8D823070
:10E8600049F4428D538D648D758D4E0D5F1D601F73
:10E87000711F3FC0D480DA94DE20A114B104D9F412
:10E88000DD20C9F4211531054105510549F48D8973
:10E890009E89AF89B88D8C839D83AE83BF830BC067
:10E8A0004C815D816E817F81CF0191010E945D7DF0
:10E8B000882309F464C0E98DFA8D4C815D816E81F5
:10E8C0007F814250504060407040058404C0440F36
:10E8D000551F661F771F0A94D2F786859785A089F2
:10E8E000B189480F591F6A1F7B1F4D0D511D611DB6
:10E8F000711D80E092E08A199B09840188159905B1
:10E9000008F48C0182E00030180709F066C080919D
:10E91000D20D9091D30DA091D40DB091D50D481783
:10E9200059076A077B0709F458C08091D60F909168
:10E93000D70F9301C7DB882349F421C095012A52E0
:10E94000324FC301B901A8010E945112600E711E1D
:10E95000980140E050E088859985AA85BB85820FA3
:10E96000931FA41FB51F88879987AA87BB87801A22
:10E97000910A8114910409F05CCFA20102C04FEF0B
:10E980005FEFCA01DF91CF911F910F91FF90EF9040
:10E99000DF90CF90BF90AF909F908F907F906F90BF
:10E9A0005F904F903F902F900895A988BA88CB88A8
:10E9B000DC88E884F9840A851B859A0140E050E0F0
:10E9C000D601C5018E199F09A00BB10B2817390775
:10E9D0004A075B0708F022CF24CFCB01BA0140E001
:10E9E00046D6882309F0AACFCACFCF92DF92EF9202
:10E9F000FF920F931F93CF93DF937C01EB018A016A
:10EA0000FC018381823008F46EC080859185A285E7
:10EA1000B3858F719070A070B0700097A105B1059B
:10EA200009F061C06CC0F8011082EDE0CE2ED12C4F
:10EA3000C701BE0140E250E0D5DE9C018032910565
:10EA400021F0009709F04FC050C04881442309F4D9
:10EA50004CC0453E69F34E3259F38B858F738F302E
:10EA6000E9F501151105D1F18A8D9B8D892BB1F541
:10EA7000842F90E08F719070009781F18330910521
:10EA80006CF58C9D90018D9D300D9C9D300D112459
:10EA90002D503040F801E20FF31F898180838B8174
:10EAA00081838D8182838F818383898584838E8511
:10EAB0008583888986838A8987838C8980878E89E4
:10EAC0008187888D82878C8D83878E8D84878881CE
:10EAD00086FF04C0F801E20FF31F15868B8583FDC6
:10EAE000A7CF822F03C08FEF01C080E0DF91CF91CD
:10EAF0001F910F91FF90EF90DF90CF9008954115F7
:10EB0000510509F090CF91CFDF93CF930F92CDB7FE
:10EB1000DEB7BE016F5F7F4F41E050E063DE0197DB
:10EB200019F02FEF3FEF03C08981282F30E0C90192
:10EB30000F90CF91DF910895EF92FF920F931F9363
:10EB4000CF93DF93EC018B81823030F1E884F9843C
:10EB50000A851B85CE01D8DF97FD1EC08885998563
:10EB6000AA85BB854F96A11DB11D88879987AA8765
:10EB7000BB87A5E016950795F794E794AA95D1F77A
:10EB80002E2D30E02F703070F5E0220F331FFA95F4
:10EB9000E1F72A52324F02C020E030E0C901DF9194
:10EBA000CF911F910F91FF90EF9008950F931F93B6
:10EBB000CF93DF93EC018B018B81882309F040C058
:10EBC000FB018789803109F041C082E08B831D8A77
:10EBD0001E8A1F8A188E808D918DA0E0B0E045E0DE
:10EBE000880F991FAA1FBB1F4A95D1F7898B9A8B53
:10EBF000AB8BBC8B13C083E08B83F801428D538DAC
:10EC0000648D758D4D8B5E8B6F8B788F9E012F5E23
:10EC10003F4FC8010E942E7E882391F01A8F098FE2
:10EC200081E089831C821D821E821F8218861986BC
:10EC30001A861B861C861D861E861F86188A01C0A2
:10EC400080E0DF91CF911F910F9108958032C1F73D
:10EC5000D2CF1F93CF93DF93EC01142F262F30E0F8
:10EC6000F90175E0EE0FFF1F7A95E1F7EA52F24FD6
:10EC70008385817121F0842F827109F066C08091B3
:10EC8000D20D9091D30DA091D40DB091D50D8C875C
:10EC90009D87AE87BF87688BF90165E0EE0FFF1F88
:10ECA0006A95E1F7EA52F24F84899589A0E0B0E0D5
:10ECB000DC01992788278D8B9E8BAF8BB88F228D97
:10ECC000338DA90160E070E0482B592B6A2B7B2B18
:10ECD0004D8B5E8B6F8B788F838590E08871907001
:10ECE000009751F4848D958DA68DB78D898B9A8B65
:10ECF000AB8BBC8B81E00BC0409739F59E012F5E3A
:10ED00003F4F898D9A8DAAD78823F9F084E08B83B1
:10ED1000812F8F7089831C821D821E821F8218861C
:10ED200019861A861B8614FF16C0CE0140E050E0FB
:10ED300060E070E074DC882371F409C049895A8965
:10ED40006B897C89CE0129DB02C01B8280E0DF91C8
:10ED5000CF911F91089515FDF1CF81E0F8CFCF93AA
:10ED6000DF93EC019C012C5F3F4F898D9A8D41E030
:10ED700050E060E070E0DDD78823A1F08D899E89A6
:10ED8000AF89B88D0097A105B10559F48C819D819B
:10ED9000AE81BF818D8B9E8BAF8BB88F8981806850
:10EDA000898381E0DF91CF9108952F923F924F9216
:10EDB0005F927F928F929F92AF92BF92CF92DF929B
:10EDC000EF92FF920F931F93DF93CF9300D000D069
:10EDD000CDB7DEB76C01162F072F5E834D83DC01A4
:10EDE00013968C911397813009F069C111968C911B
:10EDF00081FF65C182C1F6014189528963897489A5
:10EE000080859185A285B38584179507A607B707E6
:10EE100029F0C601C2DA882309F451C1812F902F4D
:10EE20009C0119014D805E800FC1D6015996ED916C
:10EE3000FC915A97DA01C90149E0B695A7959795D3
:10EE400087954A95D1F774807A9478228FEF882E2F
:10EE500081E0982E82229322772009F051C08114FC
:10EE6000910409F04DC0D60114964D915D916D91BC
:10EE70007C911797411551056105710581F45596EF
:10EE80008D919D910D90BC91A02D0097A105B1058C
:10EE900059F1F60184839583A683B78331C0CF01EE
:10EEA0009E012F5F3F4F09D6882309F408C12981AD
:10EEB0003A814B815C81D6015996ED91FC915A972C
:10EEC0008789803149F4283FBFEF3B07B0E04B070B
:10EED000B0E05B0770F008C0283FEFEF3E07EFEFB0
:10EEE0004E07EFE05E0728F0C60139DF882341F4C2
:10EEF000E6C0D60114962D933D934D935C931797DE
:10EF000080E092E08819990952018415950508F46A
:10EF10005C01D6015996ED91FC915A971496ED90AB
:10EF2000FD900D911C9117978EEF9FEFAFEFBFEF04
:10EF3000E80EF91E0A1F1B1F058404C0EE0CFF1CFF
:10EF4000001F111F0A94D2F786859785A089B18981
:10EF5000E80EF91E0A1F1B1FE70CF11C011D111DF5
:10EF600090E0A91692E0B90639F58091D20D909102
:10EF7000D30DA091D40DB091D50D8E159F05A0078E
:10EF8000B10771F41092D80F8FEF9FEFAFEFBFEF83
:10EF90008093D20D9093D30DA093D40DB093D50D43
:10EFA0008091D60F9091D70FB801A70191010E94CF
:10EFB000A46F8823A9F583C08114910411F5D601AB
:10EFC00018962D913D914D915C911B9751968D9185
:10EFD0009D910D90BC91A02D281739074A075B071A
:10EFE00080F00AD3882309F46AC081E08093D80FA7
:10EFF000E092D20DF092D30D0093D40D1093D50D65
:10F0000007C0C801B70141E032D3882309F457C0D3
:10F0100094012A52324FC901B101A5010E94511237
:10F02000950140E050E0F60180859185A285B38589
:10F03000820F931FA41FB51F80879187A287B38774
:10F040002A0C3B1C4A185B08D60118962D913D915D
:10F050004D915C911B974114510409F0E6CE5196F5
:10F060008D919D910D90BC91A02D82179307A407BF
:10F07000B50748F4F601218B328B438B548B818189
:10F080008068818311C08091D00D9091D10D892B22
:10F0900059F08D819E81892B39F0D60111968C9182
:10F0A0001197806811968C93F601818183FF04C0CB
:10F0B000C6013DDA882319F04D815E8105C081E0EB
:10F0C000D6018C934FEF5FEFCA0126960FB6F894E6
:10F0D000DEBF0FBECDBFCF91DF911F910F91FF908B
:10F0E000EF90DF90CF90BF90AF909F908F907F90E8
:10F0F0005F904F903F902F90089582FD7CCE8ECEF2
:10F10000DF92EF92FF920F931F93CF93DF93EC0167
:10F1100089899A89AB89BC89805E9F4FAF41B04095
:10F1200008F06FC0CE011BDE882309F46AC064D2E8
:10F13000882309F466C0E98DFA8DEC80FD800E818C
:10F140001F818EEF9FEFAFEFBFEFE80EF91E0A1F92
:10F150001B1F058404C0EE0CFF1C001F111F0A9426
:10F16000D2F786859785A089B189E80EF91E0A1F16
:10F170001B1F81E08093D80FE092D20DF092D30D47
:10F180000093D40D1093D50D80E092E0E6EDFDE004
:10F19000DF019C011D9221503040E1F7DD24D39422
:10F1A00011C0B801A7014D0D511D611D711D809148
:10F1B000D60F9091D70F26ED3DE00E94A46F8823D3
:10F1C00001F1D394E98DFA8D8481D81650F320E0B3
:10F1D00032E040E050E0058404C0220F331F441F9A
:10F1E000551F0A94D2F789899A89AB89BC89820F05
:10F1F000931FA41FB51F898B9A8BAB8BBC8B81E0AF
:10F2000001C080E0DF91CF911F910F91FF90EF90AF
:10F21000DF9008958F929F92AF92BF92CF92DF922C
:10F22000EF92FF920F931F93CF93DF936C01EB014B
:10F23000942E852EA22E898D9A8DD6015A969C9356
:10F240008E935997CB0140E050E060E070E0A5D884
:10F25000BB2437C0CE0170DCFC01009709F48FC0DD
:10F2600055E016950795F794E7945A95D1F71E2D1A
:10F270001F708081882311F0853EC9F4BB2099F46A
:10F280002091D20D3091D30D4091D40D5091D50DD8
:10F29000D6011C962D933D934D935C931F975096EA
:10F2A0001C93BB24B3948081882359F418C0892D02
:10F2B000982DBF014BE050E00E944412009709F4E2
:10F2C0006CC0E884F9840A851B8589899A89AB8991
:10F2D000BC89E816F9060A071B0708F4BBCFA6FE8F
:10F2E0004EC0A1FE4CC0BB2049F0F6011089C601FA
:10F2F00061E0FCD8EC01009761F441C08B81823061
:10F3000009F43DC0CE01FCDE8823C9F110E0C6ED52
:10F31000DDE080E2DE011D928A95E9F7DE01292D0C
:10F32000382DC901FC018BE001900D928150E1F76D
:10F33000E091D00DF091D10D309739F0BE01625FB0
:10F340007F4FCE014096199508C081E298E2998BD3
:10F35000888B80E098E09F878E87888999899B8B2E
:10F360008A8B998F888F8E859F859F8B8E8B44D1BA
:10F37000882329F0C601612F4A2D6BDC01C080E093
:10F38000DF91CF911F910F91FF90EF90DF90CF9081
:10F39000BF90AF909F908F900895A7FEEBCFEFCFD7
:10F3A0002F923F924F925F926F927F928F929F9295
:10F3B000AF92BF92CF92DF92EF92FF920F931F9383
:10F3C000DF93CF93CDB7DEB7C654D0400FB6F894D5
:10F3D000DEBF0FBECDBF3C016B01DE01AE5BBF4F98
:10F3E00011965C934E9325962FAF25971C861F860A
:10F3F0001FA21AA66115710509F47CC0FC01838166
:10F40000882309F077C0FA0180818F32F1F08601FC
:10F41000ECE0EE2EF12CEC0EFD1E72E4A72EB12CCA
:10F42000AC0EBD1E4E010894811C911C2796FFAEA8
:10F43000EEAE279767E2262E312C2C0E3D1E2701BB
:10F4400023C01196B183A08301C0FD01A081B181C9
:10F450008C918F32B1F3D60113968C911397825011
:10F460008230A8F28E01095D1F4F59966D917C91F3
:10F470005A97C8019BDB882359F63CC0342D252DB3
:10F480008701832F922F7C01F50180819181B40146
:10F49000A5010E947F71882329F42CC03196D501E3
:10F4A000ED93FC93D501ED91FC9180818F32B1F306
:10F4B0008823B9F0C701B801A40121E0ABDE88239D
:10F4C000C9F00C151D0511F0C8017ED82796EEADC8
:10F4D000FFAD2797EE16FF0689F6C101322D292FC1
:10F4E000CFCFC301B801A40125962FAD259792DE99
:10F4F000182F01C010E0CE0187966FD8CE010C9670
:10F500006CD8812FCA5BDF4F0FB6F894DEBF0FBEF9
:10F51000CDBFCF91DF911F910F91FF90EF90DF90C2
:10F52000CF90BF90AF909F908F907F906F905F90A3
:10F530004F903F902F9008950F931F93DF93CF9399
:10F54000CDB7DEB76B970FB6F894DEBF0FBECDBF59
:10F550009C01AB0119821C828E010F5F1F4FC801F5
:10F56000B90122E01DDF882311F410E003C0C801B7
:10F5700020D9182FCE01019630D8812F6B960FB667
:10F58000F894DEBF0FBECDBFCF91DF911F910F91D9
:10F590000895DF93CF930F92CDB7DEB780916812B5
:10F5A000909169129E012F5F3F4F009719F0281B21
:10F5B000390B02C02E563241C9010F90CF91DF9115
:10F5C0000895DB010D900020E9F71197A61BB70BFA
:10F5D0000496AD01EACBDF93CF930F92CDB7DEB7A0
:10F5E00069830496BE016F5F7F4F41E050E0DDDB31
:10F5F0000F90CF91DF9108958091D80F882399F1D2
:10F600004091D20D5091D30D6091D40D7091D50DD4
:10F610008091D60F9091D70F26ED3DE00E94A46F08
:10F62000882319F14091D90F5091DA0F6091DB0FC7
:10F630007091DC0F411551056105710591F08091C4
:10F64000D60F9091D70F26ED3DE00E94A46F88233E
:10F6500061F01092D90F1092DA0F1092DB0F109216
:10F66000DC0F1092D80F81E0089580E00895DF92BA
:10F67000EF92FF920F931F937B018C01D42E809108
:10F68000D20D9091D30DA091D40DB091D50D8E15C2
:10F690009F05A007B107B9F0AFDF8823E1F08091A3
:10F6A000D60F9091D70FB801A70126ED3DE00E943B
:10F6B0006270882381F0E092D20DF092D30D009316
:10F6C000D40D1093D50DDD2011F481E005C081E04B
:10F6D0008093D80F01C080E01F910F91FF90EF90B1
:10F6E000DF9008958F929F92AF92BF92CF92DF9258
:10F6F000EF92FF920F931F93CF93DF936C01142F20
:10F700007093D70F6093D60FFC01178A82E090E0C8
:10F71000A0E0B0E080839183A283B3831092D80FDE
:10F720001092D90F1092DA0F1092DB0F1092DC0FAB
:10F730008FEF9FEFAFEFBFEF8093D20D9093D30D7C
:10F74000A093D40DB093D50D442321F4882499249B
:10F7500054013FC0453008F01CC160E070E080E01B
:10F7600090E040E084DF882309F413C1C12FD0E08A
:10F770002197FE0174E0EE0FFF1F7A95E1F7EA5240
:10F78000F24FE254FE4F8081EE5BF14090E08F77C4
:10F790009070892B09F0FDC0E653FE4F8081918166
:10F7A000A281B38184369105A105B10508F4F1C0A9
:10F7B00064E0CC0FDD1F6A95E1F7C456D04F888016
:10F7C0009980AA80BB8081149104A104B10409F43A
:10F7D000E0C0C501B40140E04ADF882309F4D9C084
:10F7E0008091E10D9091E20D8050924009F0D1C0DE
:10F7F0002091E60D222309F4CCC08091E40D909174
:10F80000E50D892B09F4C5C08091E30D882309F427
:10F81000C0C0F601228B8091E30D8483158661E0E0
:10F8200070E007C04F5FF60145874150483008F04F
:10F83000B0C0F6014585848190E09B01042E02C092
:10F84000220F331F0A94E2F78217930759F720918A
:10F85000EC0D3091ED0D2115310519F040E050E02F
:10F8600008C02091FA0D3091FB0D4091FC0D509194
:10F87000FD0DF6012583368347835087E090E40D24
:10F88000F090E50D00E010E0E80CF91C0A1D1B1DCE
:10F89000E38AF48A058B168B8091E70D9091E80D31
:10F8A000918F808F6091E60D70E080E090E00E9483
:10F8B000B0ED6E0D7F1D801F911FF601628F738F5B
:10F8C000848F958F2091E70D3091E80D55E0220F40
:10F8D000331F5A95E1F721503E4F232F33272695AA
:10F8E00040E050E0260F371F481F591F26873787F3
:10F8F000408B518B8091E90D9091EA0D009719F0A2
:10F90000A0E0B0E008C08091F60D9091F70DA091B5
:10F91000F80DB091F90D85017401E21AF30A040B98
:10F92000150BA8019701280F391F4A1F5B1FF6010D
:10F93000058404C056954795379527950A94D2F7C4
:10F940002187328743875487253FFFE03F07F0E058
:10F950004F07F0E05F0720F48CE0F601878B19C0B9
:10F96000255F3F4F4040504018F480E1F6010EC043
:10F970008091020E9091030EA091040EB091050E9D
:10F98000F601828F938FA48FB58F80E2878B81E001
:10F9900001C080E0DF91CF911F910F91FF90EF9018
:10F9A000DF90CF90BF90AF909F908F9008956F920F
:10F9B0007F928F929F92AF92BF92CF92DF92EF92FF
:10F9C000FF920F931F93CF93DF93EC015A016B01CA
:10F9D00038014901423051056105710508F45DC0E7
:10F9E00089859A85AB85BC850196A11DB11D8417BB
:10F9F0009507A607B70708F450C08F89803129F40E
:10FA0000E52EF62E072F11270CC0803209F045C0D5
:10FA10007A018B0187E016950795F794E7948A950C
:10FA2000D1F78B899C89AD89BE89E80EF91E0A1F22
:10FA30001B1FC801B70141E01ADE882371F18F89CD
:10FA4000803149F4F501F070EE0FFF1FEA52F24FDA
:10FA5000718260820DC0F501EF77F070EE0FFF1F2D
:10FA6000EE0FFF1FEA52F24F608271828282938210
:10FA70008A89823080F08D819E81AF81B885E80EC1
:10FA8000F91E0A1F1B1FE092D90FF092DA0F0093A4
:10FA9000DB0F1093DC0F81E001C080E0DF91CF919C
:10FAA0001F910F91FF90EF90DF90CF90BF90AF909C
:10FAB0009F908F907F906F900895CF92DF92EF92FA
:10FAC000FF920F931F93CF93DF93EC017A018B0189
:10FAD000690189859A85AB85BC850196A11DB11DFB
:10FAE00084179507A607B70708F452C08F8980319D
:10FAF00029F45527412F302F2F2D0CC0803209F0CB
:10FB000047C09A01AB0167E0569547953795279511
:10FB10006A95D1F78B899C89AD89BE89280F391FD9
:10FB20004A1F5B1F8091D20D9091D30DA091D40DEF
:10FB3000B091D50D281739074A075B0731F0CA0184
:10FB4000B90140E094DD882319F18F89803159F49F
:10FB5000F701F070EE0FFF1FEA52F24F80819181A2
:10FB6000A0E0B0E00EC0F701EF77F070EE0FFF1FDE
:10FB7000EE0FFF1FEA52F24F80819181A281B38183
:10FB8000BF70F60180839183A283B38381E001C0BB
:10FB900080E0DF91CF911F910F91FF90EF90DF9068
:10FBA000CF900895AF92BF92CF92DF92EF92FF92E3
:10FBB0000F931F93DF93CF9300D00F92CDB7DEB793
:10FBC0006C017A018B0182E090E0A0E0B0E0F601E8
:10FBD00080839183A283B3835E010894A11CB11C2E
:10FBE000C601B801A701950168DF882339F1C60174
:10FBF000B801A70100E010E020E030E0D8DE882363
:10FC0000E9F0E980FA800B811C81F6018789803157
:10FC100051F4F8EFEF16FFEFFF06F0E00F07F0E00A
:10FC20001F07F0F209C088EFE8168FEFF8068FEF94
:10FC300008078FE01807A0F281E001C080E00F9074
:10FC40000F900F900F90CF91DF911F910F91FF9028
:10FC5000EF90DF90CF90BF90AF9008954F925F925A
:10FC60006F927F928F929F92AF92BF92CF92DF92CC
:10FC7000EF92FF920F931F93DF93CF9300D00F92D9
:10FC8000CDB7DEB76C0149835A836B837C8339011E
:10FC9000EE24FF2487012E010894411C511C812C65
:10FCA000E2E09E2EA12CB12C49815A816B817C818E
:10FCB000C601920102DF882339F1D501C401F601A2
:10FCC000058404C0880F991FAA1FBB1F0A94D2F78E
:10FCD000E80EF91E0A1F1B1F29813A814B815C81A6
:10FCE0008789803131F4285F3F4F40405040E0F237
:10FCF00005C0285F3F4F4F4F5F40B0F2F301E082F5
:10FD0000F1820283138381E00F900F900F900F9088
:10FD1000CF91DF911F910F91FF90EF90DF90CF90E7
:10FD2000BF90AF909F908F907F906F905F904F901B
:10FD300008952F923F924F925F926F927F928F928F
:10FD40009F92AF92BF92CF92DF92EF92FF920F936A
:10FD50001F93DF93CF93CDB7DEB72F970FB6F894ED
:10FD6000DEBF0FBECDBF1C014A875B876C877D87D6
:10FD70003F872E87DC0119968D919D910D90BC9146
:10FD8000A02D0196A11DB11D8E839F83A887B987E1
:10FD9000F9010081118122813381011511052105AD
:10FDA000310549F0480159010894811C911CA11C9E
:10FDB000B11C1D8210C0D1018D909D90AD90BC9062
:10FDC0001D828A859B85AC85BD850197A105B105FE
:10FDD00011F491E09D83750164014424552432019E
:10FDE0008E010F5F1F4FF10181859285A385B48538
:10FDF000481659066A067B0608F08CC08E819F81E2
:10FE0000A885B9858C159D05AE05BF0550F4A2E007
:10FE10008A2E912CA12CB12CF2E0CF2ED12CE12CEA
:10FE2000F12CC101B701A601980147DE882309F42E
:10FE300071C089819A81AB81BC81A70196012F5F36
:10FE40003F4F4F4F5F4F0097A105B10519F0490192
:10FE50005A010DC0281939094A095B098A859B8511
:10FE6000AC85BD85281739074A075B0759F0089408
:10FE7000411C511C611C711C0894C11CD11CE11C4B
:10FE8000F11CB1CFC101A601B7010FEF1FEF2FEF9A
:10FE90003FE08DDD882391F43DC0260137010894B1
:10FEA0004108510861087108C101B301A20197011D
:10FEB00086017DDD882371F1730162018C149D043C
:10FEC000AE04BF0450F3AE85BF854D915D916D9139
:10FED0007C91411551056105710531F0C101950114
:10FEE000840165DD8823B1F0EE85FF8580829182F3
:10FEF000A282B382FD81FF2359F00894811C911CDA
:10FF0000A11CB11CD1018D929D92AD92BC92139710
:10FF100081E001C080E02F960FB6F894DEBF0FBEDF
:10FF2000CDBFCF91DF911F910F91FF90EF90DF90A8
:10FF3000CF90BF90AF909F908F907F906F905F9089
:10FF40004F903F902F900895FC018091DD0F8432F7
:10FF500090F480838F5F8093DD0F815090E0FC01EF
:10FF6000EE0FFF1FE80FF91FE252F04F88EB9BE006
:10FF70009283818308958FEF80830895FC0120810F
:10FF80002432B8F58181992787FD909548E850E0A3
:10FF9000481B590B440F551F440F551F6417750715
:10FFA00084F08281992787FD909548E552E0481BAF
:10FFB000590B440F551F440F551F641775070CF458
:10FFC000AB0142505040CA01AA2797FDA095BA2F15
:10FFD000880F991FAA1FBB1F4FB7F89430E0F90193
:10FFE000EE0FFF1FE20FF31FE252F04F9283818367
:10FFF0004FBF0895FC0180818F3F19F420E030E06D
:020000021000EC
:1000000016C090E0FC01EE0FFF1FE80FF91FE2524F
:10001000F04F2181328183E0220F331F8A95E1F76F
:10002000B4E036952795BA95E1F72E5F3F4FC901A9
:100030000895AF92BF92CF92DF92EF92FF920F930B
:100040001F938C01D7DF00D00F920196AA2797FD4E
:10005000A095BA2FF8016181772767FD709528E890
:1000600030E0261B370B220F331F220F331F44278C
:1000700037FD4095542F6281772767FD7095E8E53D
:10008000EE2EE2E0FE2EE61AF70AEE0CFF1CEE0C56
:10009000FF1C0027F7FC0095102F64EBA62EB12C57
:1000A000C12CD12CEDB7FEB7A182B282C382D4821B
:1000B000BC01CD01AA24BB2465010E94DDE80F909C
:1000C0000F900F900F90CB011F910F91FF90EF9029
:1000D000DF90CF90BF90AF900895AF92BF92CF9234
:1000E000DF92EF92FF920F931F93CF93DF93EC0178
:1000F0009B0182E0603278070CF048C077FF03C0B4
:1001000020E030E005C0653B710514F024EB30E0E1
:1001100000D00F92B901882777FD8095982F29810B
:10012000332727FD3095E8E8AE2EB12CA21AB30A8A
:10013000AA0CBB1CAA0CBB1CCC24B7FCC094DC2CA6
:10014000EA81FF27E7FDF09528E532E02E1B3F0B03
:10015000220F331F220F331F442737FD4095542FA2
:10016000EDB7FEB7218332834383548320E030E030
:1001700040E050E004EBE02EF12C012D112D0E9407
:10018000DDE89B010F900F900F900F90CE01B90109
:10019000F5DEDF91CF911F910F91FF90EF90DF90EF
:1001A000CF90BF90AF900895CF92DF92EF92FF92E1
:1001B0001F93CF93DF93EC01162F7A016901888199
:1001C000843208F080C0862F61E00E94D4E38881E9
:1001D00090E0FC01EE0FFF1FE80FF91FE252F04F15
:1001E0001F738081807C812B808380E292E08E1956
:1001F0009F0964E070E00E94EFED698380E699E07A
:100200008C199D0964E070E00E94EFED6A83A8817B
:100210008A2F6CE00E94CFED682F70E0AB01440F95
:10022000551F460F571F440F551F440F551F20E001
:1002300030E0C901840F951FFC01EE0FFF1FE80F8E
:10024000F91FE252F04F808186FD31C02F5F3F4F92
:100250002C30310571F740C01092900082E08093FD
:100260009100109295001092940088BB80937100C9
:100270001EC06230710569F41092A00082E0809384
:10028000A1001092A5001092A40089BB8093720077
:100290000EC0672B61F41092200182E0809321014F
:1002A00010922501109224018ABB809373008A2F3B
:1002B00090E0FC01EE0FFF1FE80FF91FE252F04F34
:1002C0008081806480838881DF91CF911F91FF902E
:1002D000EF90DF90CF9008956130710551F6BCCF5B
:1002E00040E252E020E639E05FCFEF92FF920F93B9
:1002F0001F93CF93DF938B017A01EC01DC01A65BA6
:10030000BF4E8C9187FF04C0FB011182108237C061
:10031000AE01440F551F4C0F5D1F440F551F440F76
:10032000551F2C91332727FD3095240F351F8091C1
:10033000DD0F90E02817390714F58C91992787FD78
:100340009095840F951FFC01EE0FFF1FE80FF91F1A
:10035000E252F04F808186FF12C08C91992787FD71
:100360009095840F951FFC01EE0FFF1FE80FF91FFA
:10037000E252F04F80818F7360E00E9487E4DE01DB
:10038000A65BBF4E8C918F5F8C93AE01440F551FBF
:100390004C0F5D1F440F551F440F551F2C913327E1
:1003A00027FD3095240F351F8091DD0F90E0281731
:1003B00039070CF04DC08C918C300CF049C0F8011D
:1003C000208131818C91992787FD9095840F951F0D
:1003D000FC01EE0FFF1FE80FF91FE252F04F818181
:1003E0009281280F391FF701318320838C9199273F
:1003F00087FD9095840F951FFC01EE0FFF1FE80FFE
:10040000F91FE252F04F808186FF2AC08C91992714
:1004100087FD9095840F951FFC01EE0FFF1FE80FDD
:10042000F91FE252F04F80818F7361E00E9487E4F0
:1004300017C080E49CE904C0F80180819181049692
:10044000F70191838083C65BDF4E8FEF888308C0FE
:10045000F80180819181049680549C4950F3ECCF3F
:10046000DF91CF911F910F91FF90EF9008951F9210
:100470000F920FB60F920BB60F9211242F933F934A
:100480004F935F936F937F938F939F93AF93BF939C
:10049000EF93FF9380E090E064E271E048E251E086
:1004A00024DFFF91EF91BF91AF919F918F917F9149
:1004B0006F915F914F913F912F910F900BBE0F90D5
:1004C0000FBE0F901F9018951F920F920FB60F92AC
:1004D0000BB60F9211242F933F934F935F936F931B
:1004E0007F938F939F93AF93BF93EF93FF9382E09C
:1004F00090E064EA70E048EA50E0F7DEFF91EF91A7
:10050000BF91AF919F918F917F916F915F914F912B
:100510003F912F910F900BBE0F900FBE0F901F9029
:1005200018951F920F920FB60F920BB60F921124CF
:100530002F933F934F935F936F937F938F939F93EB
:10054000AF93BF93EF93FF9381E090E064E970E095
:1005500048E950E0CADEFF91EF91BF91AF919F91C2
:100560008F917F916F915F914F913F912F910F905C
:100570000BBE0F900FBE0F901F9018951092811018
:10058000109283101092851008958093610408954D
:10059000EFE6F0E08081826080830895819A879AF7
:1005A000EAE0F1E08081826080830E9A3B9A579A5C
:1005B0005F9A829A8A9AE7E0F1E080818160808385
:1005C0009FB7F894E8E0F1E08081816080839FBF6D
:1005D0000A9A129A3F9A479A6D98759A53985B9A1D
:1005E000E4E0F1E080818E7F80839FB7F894E5E0BE
:1005F000F1E08081816080839FBF809A88985F9AB4
:100600001092D708869A8E988A9A1092D808EAE0B3
:10061000F1E08081886080839FB7F894EBE0F1E09F
:100620008081877F80839FBF9FB7F894E8E0F1E0E7
:100630008081816080839FBF1092D9080C9A1498A2
:10064000129A399A4198479AA1E8B0E08C918F7E2E
:100650008C938C9188608C93E0E8F0E080818D7FB2
:10066000808380818E7F808380818F73808380816F
:100670008F7C80838C91887F82608C9380E090E473
:1006800090938900809388001092850010928400D6
:10069000EFE6F0E080818260808381E080936104F6
:1006A000789408951F93FC011FB7F894808191817D
:1006B000A281B38180935B1090935C10A0935D1036
:1006C000B0935E10FB0180819181A281B381809300
:1006D0005F1090936010A0936110B0936210FA01C4
:1006E00080819181A281B381809363109093641083
:1006F000A0936510B0936610F90180819181A28169
:10070000B3818093671090936810A0936910B093A1
:100710006A101FBF1F910895FC012FB7F8948081C4
:100720009181A281B3818093671090936810A09308
:100730006910B0936A102FBF0895E82F8FB7F8940F
:10074000F0E0EE0FFF1FEE0FFF1FE55AFF4E208176
:100750003181428153818FBFB901CA0108958091CF
:100760006F008D7F80936F000CC09091B60D8091CB
:10077000B70D981731F08091B70D8F5F8770809318
:10078000B70D9091B60D8091B70D981771F7109233
:100790004E1010924D1080916F00826080936F0018
:1007A000089507C00E94CF9080E00E9401370E9408
:1007B0008FD49091B60D8091B70D981799F7089541
:1007C000F0DF5F9A1092D7088A9A1092D8089FB7E4
:1007D000F894E8E0F1E08081816080839FBF10920F
:1007E000D908129A479A08951F920F920FB60F9246
:1007F0000BB60F921124AF92BF92CF92DF92EF927D
:10080000FF920F931F932F933F934F935F936F9399
:100810007F938F939F93AF93BF93CF93DF93EF9388
:10082000FF9380914D1090914E10892B09F097C144
:100830009091B60D8091B70D981719F4E0E0F0E0B3
:1008400014C08091B70D90E02DE430E0829FF0015C
:10085000839FF00D929FF00D1124E25BF44FE45B57
:10086000FF4F81E08083EC54F040F0934E10E09312
:100870004D10309709F46DC1E45BFF4F81E0808338
:10088000EC54F04010928D1010928E1010928F1038
:100890001092901060AD71AD2CE96134720718F0C0
:1008A00060E47CE904C03EE46132730730F0769581
:1008B00067957695679584E007C047E261317407D4
:1008C00030F07695679582E08093861007C080931C
:1008D00086106032710510F460E270E06052704082
:1008E00058E060307507E8F0472F50E0440F551F7F
:1008F000440F551F495C544F9A012E5F3F4FF90139
:10090000859194919C01AA27639FC001629F810DEC
:100910009A1F06948A1F9A1F1124FA014591549137
:100920001EC0CB01969587958C7F895C904FFC010A
:1009300045915491FC01329625913491862F90E097
:1009400087709070FC012E9FC0012F9F900D3E9FDD
:10095000900D1124B3E096958795BA95E1F7481B61
:10096000590B44365105A8F4E0EAF3E007C0809142
:10097000C00085FFFCCF31969093C60090819923EB
:10098000B1F78CE096E04AE050E00E94592944E635
:1009900050E05093921040939110809186109927C7
:1009A00087FD90959093941080939310E0914D1053
:1009B000F0914E1064AD75AD70938C1060938B10F8
:1009C000FCE961347F0718F060E47CE904C02EE4A0
:1009D0006132720730F0769567957695679584E079
:1009E00007C037E26131730730F07695679582E092
:1009F0008093861008C081E0809386106032710574
:100A000010F460E270E06052704048E060307407BB
:100A1000E8F0472F50E0440F551F440F551F495C25
:100A2000544F9A012E5F3F4FF901859194919C019B
:100A3000AA27639FC001629F810D9A1F06948A1F97
:100A40009A1F1124FA01459154911EC0CB0196952D
:100A500087958C7F895C904FFC0145915491FC01F6
:100A6000329625913491862F90E087709070FC012A
:100A70002E9FC0012F9F900D3E9F900D112433E0BB
:100A8000969587953A95E1F7481B590B44365105E1
:100A9000A8F4E0EAF3E007C08091C00085FFFCCF36
:100AA00031969093C60090819923B1F78CE096E03F
:100AB0004AE050E00E94592944E650E0CA01A0E013
:100AC000B0E08093871090938810A0938910B09322
:100AD0008A105093890040938800E0914D10F09166
:100AE0004E1080899189A289B389B695A79597956B
:100AF0008795B095A095909581959F4FAF4FBF4F2B
:100B000080936B1090936C10A0936D10B0936E1047
:100B100080936F1090937010A0937110B093721027
:100B20008093731090937410A0937510B093761007
:100B30008093771090937810A0937910B0937A10E7
:100B400010927B1010927C1010927D1010927E10EB
:100B500006C080ED97E09093890080938800C09153
:100B60004D10D0914E10209709F4A1C488A1809314
:100B70007F1080FF03C0899A8FEF02C0899881E0BF
:100B800080935D0480917F1081FF03C08F988FEF69
:100B900002C08F9A81E080935E0480917F1080FF75
:100BA0003BC0809161048823B9F18CB18295869510
:100BB00087708095282F217080FF2CC08091801035
:100BC000882341F188819981AA81BB811816190671
:100BD0001A061B06FCF480915B1090915C10A091AA
:100BE0005D10B0915E1080934F1090935010A093C1
:100BF0005110B093521081E08093811088899989B7
:100C0000AA89BB8980937B1090937C10A0937D1060
:100C1000B0937E102093801080917F1081FD37C0AB
:100C200080916104882399F120910301217031E0C2
:100C3000232759F180918210882339F18C819D817D
:100C4000AE81BF81181619061A061B06F4F48091AE
:100C50005F1090916010A0916110B091621080932C
:100C6000531090935410A0935510B0935610309396
:100C7000831088899989AA89BB8980937B10909376
:100C80007C10A0937D10B0937E10209382108091F1
:100C90007F1082FF48C09FB7F89480910B0182605B
:100CA00080930B019FBF8FEF80935F04809161045D
:100CB000882309F443C089B18695869586958095E9
:100CC000282F217080FF2CC080918410882341F14F
:100CD00088859985AA85BB85181619061A061B06EC
:100CE000FCF48091631090916410A0916510B09114
:100CF00066108093571090935810A0935910B0939A
:100D00005A1081E08093851088899989AA89BB89C6
:100D100080937B1090937C10A0937D10B0937E10F5
:100D2000209384100BC08FB7F89490910B019D7F96
:100D300090930B018FBF81E080935F0480917F10BF
:100D400099A183FF07C0913011F4439A01C0169A0C
:100D50008FEF06C0913011F4439801C0169881E0DE
:100D60008093600460E082C18091C00087FF19C059
:100D70004091C600E0910806F091090631969F0166
:100D80002F773070319780910A0690910B062817C3
:100D9000390739F0E857FA4F40833093090620931A
:100DA0000806288139814A815B8180916B1090917E
:100DB0006C10A0916D10B0916E10280F391F4A1F52
:100DC0005B1F20936B1030936C1040936D10509309
:100DD0006E1012161306140615066CF5889A88898B
:100DE0009989AA89BB89281B390B4A0B5B0B209375
:100DF0006B1030936C1040936D1050936E102091D7
:100E00005B1030915C1040915D1050915E108091AC
:100E10005D04992787FD9095A92FB92F820F931F05
:100E2000A41FB51F80935B1090935C10A0935D107E
:100E3000B0935E1088982C813D814E815F818091B6
:100E40006F1090917010A0917110B0917210280FD6
:100E5000391F4A1F5B1F20936F103093701040930F
:100E600071105093721012161306140615066CF5C5
:100E70008E9A88899989AA89BB89281B390B4A0BC4
:100E80005B0B20936F103093701040937110509350
:100E9000721020915F10309160104091611050915C
:100EA000621080915E04992787FD9095A92FB92F34
:100EB000820F931FA41FB51F80935F109093601043
:100EC000A0936110B09362108E98288539854A8569
:100ED0005B858091731090917410A0917510B09102
:100EE0007610280F391F4A1F5B1F20937310309311
:100EF0007410409375105093761012161306140652
:100F00001506DCF59FB7F89480910B0188608093FB
:100F10000B019FBF88899989AA89BB89281B390B36
:100F20004A0B5B0B20937310309374104093751031
:100F300050937610209163103091641040916510A9
:100F40005091661080915F04992787FD9095A92F95
:100F5000B92F820F931FA41FB51F80936310909326
:100F60006410A0936510B09366109FB7F8948091B9
:100F70000B01877F80930B019FBF2C853D854E859C
:100F80005F858091771090917810A0917910B09141
:100F90007A10280F391F4A1F5B1F20937710309358
:100FA00078104093791050937A1012161306140695
:100FB0001506BCF589A1813011F4419A01C0149A3B
:100FC00088899989AA89BB89281B390B4A0B5B0B35
:100FD00020937710309378104093791050937A10C3
:100FE00020916710309168104091691050916A10FB
:100FF00080916004992787FD9095A92FB92F820FC2
:10100000931FA41FB51F8093671090936810A0933F
:101010006910B0936A1089A1813011F4419801C020
:10102000149880917B1090917C10A0917D10B091CC
:101030007E100196A11DB11D80937B1090937C10B2
:10104000A0937D10B0937E1020917B1030917C1086
:1010500040917D1050917E1088899989AA89BB8919
:10106000281739074A075B0730F46F5F80918610B5
:1010700068170CF479CE20917B1030917C10409150
:101080007D1050917E108C899D89AE89BF89821711
:101090009307A407B50708F4E3C0E0908710F09029
:1010A00088100091891010918A10AC8CBD8CCE8C68
:1010B000DF8CA8019701C601B501AA27279FB12D92
:1010C000389FF001489FF00D479FE00DF11D289FCC
:1010D000B00DE11DFA1F379FB00DE11DFA1F469FAD
:1010E000B00DE11DFA1F369FB10DEA1FFA1FB6952C
:1010F000EA1FFA1F11248CAD9DAD8E0F9F1F909398
:101100008C1080938B1028AD39AD4AAD5BADA0E05B
:10111000B0E0281739074A075B0720F430938C109A
:1011200020938B1060918B1070918C108CE961343E
:10113000780718F060E47CE904C09EE46132790726
:1011400030F0769567957695679584E007C0E7E27D
:1011500061317E0730F07695679582E08093861046
:1011600008C081E0809386106032710510F460E25F
:1011700070E060527040F8E060307F07E8F0472F81
:1011800050E0440F551F440F551F495C544F9A01BE
:101190002E5F3F4FF901859194919C01AA27639F8F
:1011A000C001629F810D9A1F06948A1F9A1F112405
:1011B000FA01459154911EC0CB01969587958C7F7D
:1011C000895C904FFC0145915491FC013296259128
:1011D0003491862F90E087709070FC012E9FC001A3
:1011E0002F9F900D3E9F900D1124B3E0969587950B
:1011F000BA95E1F7481B590B44365105A8F4E0EACB
:10120000F3E007C08091C00085FFFCCF319690933A
:10121000C60090819923B1F78CE096E04AE050E057
:101220000E94592944E650E0509389004093880079
:101230009A0140E050E08091871090918810A09131
:101240008910B0918A10820F931FA41FB51F80933D
:10125000871090938810A0938910B0938A1002C1D0
:1012600020917B1030917C1040917D1050917E1028
:10127000888D998DAA8DBB8D82179307A407B5071A
:1012800008F0E4C060918D1070918E1080918F10E5
:10129000909190102C8D3D8D4E8D5F8DAA27639F70
:1012A000B12D749FF001849FF00D839FE00DF11D1F
:1012B000649FB00DE11DFA1F739FB00DE11DFA1F71
:1012C000829FB00DE11DFA1F729FB10DEA1FFA1F38
:1012D000B695EA1FFA1F112480918B1090918C1003
:1012E0008E179F0738F4C05CDF4F68817981C05446
:1012F000D04003C0BC016E1B7F0BC05CDF4F288158
:1013000039814A815B81CB01A0E0B0E0821793076D
:10131000A407B50708F4B901FCE961347F0718F0A8
:1013200060E47CE904C02EE46132720730F0769507
:1013300067957695679584E007C037E2613173075A
:1013400030F07695679582E08093861008C081E042
:10135000809386106032710510F460E270E0605294
:10136000704048E060307407E8F0472F50E0440FC9
:10137000551F440F551F495C544F9A012E5F3F4F34
:10138000F901859194919C01AA27639FC001629FF6
:10139000810D9A1F06948A1F9A1F1124FA01459104
:1013A00054911EC0CB01969587958C7F895C904F98
:1013B000FC0145915491FC01329625913491862F80
:1013C00090E087709070FC012E9FC0012F9F900DC0
:1013D0003E9F900D112423E0969587952A95E1F77D
:1013E000481B590B44365105A8F4E0EAF3E007C066
:1013F0008091C00085FFFCCF31969093C60090810C
:101400009923B1F78CE096E04AE050E00E94592918
:1014100044E650E050938900409388009A0140E0F0
:1014200050E080918D1090918E10A0918F10B0910E
:101430009010820F931FA41FB51F80938D1090935F
:101440008E10A0938F10B09390100CC080919110CB
:1014500090919210909389008093880080919310CE
:101460008093861020917B1030917C1040917D10EC
:1014700050917E10E0914D10F0914E10808991892D
:10148000A289B389281739074A075B0780F01092B1
:101490004E1010924D109091B60D8091B70D981787
:1014A00031F08091B70D8F5F87708093B70DFF91FA
:1014B000EF91DF91CF91BF91AF919F918F917F91EC
:1014C0006F915F914F913F912F911F910F91FF90DD
:1014D000EF90DF90CF90BF90AF900F900BBE0F902A
:1014E0000FBE0F901F90189580918110882349F4AA
:1014F00080918310882329F480918510882309F432
:101500009CC0E0E1F5E0949108C08091C00085FFA7
:10151000FCCF9093C600319694919923B1F7E3E7FD
:10152000F3E1949108C08091C00085FFFCCF9093B7
:10153000C600319694919923B1F780918110882348
:10154000F1F060914F107091501080915110909176
:1015500052100E94A0EA2091EE0A3091EF0A4091C9
:10156000F00A5091F10A0E9405EAAB01BC018FE636
:1015700093E10E94112E8FE593E10E9431D4809176
:1015800083108823F1F06091531070915410809172
:101590005510909156100E94A0EA2091F20A3091C5
:1015A000F30A4091F40A5091F50A0E9405EAAB0152
:1015B000BC018BE593E10E94112E8BE493E10E9424
:1015C00031D4809185108823F1F06091571070918B
:1015D00058108091591090915A100E94A0EA2091C1
:1015E000F60A3091F70A4091F80A5091F90A0E94E0
:1015F00005EAAB01BC0187E493E10E94112E87E369
:1016000093E10E9431D4E4EBF3E007C08091C00085
:1016100085FFFCCF31969093C60090819923B1F756
:101620008091C00085FFFCCF8AE08093C6001092B5
:1016300081101092831010928510089560E070E080
:101640008FE793E420916604309167044091680429
:10165000509169040E9405EADC019B01AC012093D2
:10166000D3103093D4104093D5105093D610CB01A3
:101670008093D7109093D810A093D910B093DA101C
:101680000895FC0197FF03C08091AD1003C0E2559F
:10169000FF4E808190E008952F923F924F925F928B
:1016A0006F927F928F929F92AF92BF92CF92DF9272
:1016B000EF92FF920F931F93CF93DF93EC0121E002
:1016C00030E0A901440F551F440F551FFA01E25A9B
:1016D000FB4E85919491C817D9070CF059C0B901F8
:1016E00061507040660F771F660F771FCB01805ADD
:1016F0009B4EFC0105911491625A7B4EFB01C590F3
:10170000D490FA01E05AFB4EE590F490FA01E25AC7
:10171000FB4EA590B490B801882777FD8095982F4F
:101720000E94A0EA1B012C01CC19DD09BE0188270B
:1017300077FD8095982F0E94A0EA3B014C01E01AAA
:10174000F10A0027F7FC0095102FC801B7010E948D
:10175000A0EA9B01AC01C401B3010E94DEEC7B0155
:101760008C01AC18BD08CC24B7FCC094DC2CC6019D
:10177000B5010E94A0EA9B01AC01C801B7010E941B
:1017800005EA9B01AC01C201B1010E9425E919C023
:10179000822F8F5F2F5F3F4F2D33310509F091CF9F
:1017A0008D3329F0E0E070E080E060E00CC0E0E51F
:1017B000F5E165917491882777FD8095982F0E94B7
:1017C000A0EAE62F692F2E2F372F482F562FB90169
:1017D000CA01DF91CF911F910F91FF90EF90DF90A1
:1017E000CF90BF90AF909F908F907F906F905F90C1
:1017F0004F903F902F900895089510929610109258
:1018000095101092AE102C9810929810109297107C
:101810001092AF109FB7F894E2E0F1E080818F7BE7
:1018200080839FBF10929A10109299101092AD1061
:101830009FB7F894E2E0F1E080818F7D80839FBFC5
:1018400008952CEA35EC47E25EE30C94DEEC2CEADA
:1018500035EC47E25EE30C9405EA2CEA35EC47E20E
:101860005EE30C9405EA2CEA35EC47E25EE30C9467
:10187000DEEC9FB7F894809102018F7D8093020186
:101880009FBF0E94572A882339F5E9E0F5E094913B
:1018900008C08091C00085FFFCCF9093C6003196B0
:1018A00094919923B1F7E3E9F3E1949108C0809111
:1018B000C00085FFFCCF9093C60031969491992388
:1018C000B1F78091C00085FFFCCF8AE08093C6000D
:1018D00082E893E10E943FD40C94262B1F93182F8B
:1018E0008CDF0E94572A882309F036C0E9E0F5E032
:1018F000949108C08091C00085FFFCCF9093C600F2
:10190000319694919923B1F78CE096E0612F70E0C5
:101910004AE050E00E9432298091C00085FFFCCF50
:101920008AE08093C600E4E1F4E1949108C08091DC
:10193000C00085FFFCCF9093C60031969491992307
:10194000B1F78091C00085FFFCCF8AE08093C6008C
:1019500087E094E10E943FD40E94262B1F910895B6
:101960001F920F920FB60F920BB60F9211242F9366
:101970003F934F935F936F937F938F939F93AF9317
:10198000BF93EF93FF9320917604222389F58091F2
:10199000AE108093B910882311F02C9A01C02C98B6
:1019A0008091AF108093B810882331F09FB7F894DE
:1019B00080910201806405C09FB7F8948091020174
:1019C0008F7B809302019FBF8091AD108093B710F1
:1019D000882331F09FB7F89480910201806205C09E
:1019E0009FB7F894809102018F7D809302019FBF81
:1019F0008091B910821708F42C988091B810821742
:101A000040F49FB7F894809102018F7B809302018C
:101A10009FBF8091B710821740F49FB7F8948091D0
:101A200002018F7D809302019FBF2F5F2F7720934C
:101A3000760480917704853009F48EC0863090F466
:101A4000823009F44FC0833030F48823F1F08130C4
:101A500009F0B2C029C0833009F453C0843009F0C2
:101A6000ABC06BC0883009F499C0893038F4863037
:101A700009F48EC0873009F09FC08EC0893009F408
:101A800091C08A3009F098C095C088E080937B00AF
:101A900085E480937C0080917A00806480937A0052
:101AA0000E944C9D81E01BC080917800909179004C
:101AB000A0E0B0E02091C6103091C7104091C8104E
:101AC0005091C910280F391F4A1F5B1F2093C61061
:101AD0003093C7104093C8105093C91082E0809390
:101AE00077046AC088E080937B0086E480937C0062
:101AF00080917A00806480937A000E944C9D83E0FC
:101B0000EECF8091780090917900A0E0B0E0209134
:101B1000BA103091BB104091BC105091BD10280FED
:101B2000391F4A1F5B1F2093BA103093BB1040939C
:101B3000BC105093BD1084E0D2CF88E080937B002E
:101B400085E480937C0080917A00806480937A00A1
:101B50000E944C9D85E0C3CF8091780090917900E0
:101B6000A0E0B0E02091C2103091C3104091C410A9
:101B70005091C510280F391F4A1F5B1F2093C210B8
:101B80003093C3104093C4105093C51086E0A7CF84
:101B90000E944C9D87E0A3CF88E0A1CF0E944C9D7E
:101BA00089E09DCF109277048091CA108F5F809357
:101BB000CA1002C0109277048091CA10803108F4D4
:101BC0006BC08091B0108823C1F48091C6109091B1
:101BD000C71090939C1080939B108091C21090919D
:101BE000C31090939E1080939D108091BA10909195
:101BF000BB109093A8108093A71081E08093B01041
:101C00001092CA101092C6101092C7101092C810ED
